:020000040800F2
:1000000068DF0010DD02000869DF0008E9880008E9
:1000100081DB0008A91B00088D0002080000000019
:10002000000000000000000000000000650A010858
:1000300091210008000000007DF7000869480108D0
:10004000F7020008F7020008F7020008F7020008AC
:10005000F7020008F7020008ED2900089D2A0008B1
:10006000FD2A0008492B0008F7020008CD1F0008F0
:10007000F7020008F7020008F7020008F70200087C
:1000800021200008F7020008F7020008F702000824
:10009000F7020008F7020008F7020008952B000895
:1000A000F7020008F7020008F7020008F70200084C
:1000B000F7020008DD4801085D4A0108F702000860
:1000C000F7020008F7020008F7020008F70200082C
:1000D000F7020008F7020008F7020008F70200081C
:1000E0004D2A0008F7020008F7020008F70200088E
:1000F0003DD30108F7020008F7020008F7020008E4
:10010000F7020008F70200089571010811020108C2
:10011000F7020008F70200080DAD010899D20108A6
:10012000F702000875200008C9200008F70200083F
:10013000F7020008F7020008F7020008F7020008BB
:10014000F7020008F7020008F7020008B5DF000810
:100150001D21000835210008F7020008F7020008F9
:10016000F7020008F7020008F7020008F70200088B
:10017000F7020008F7020008F7020008000000007C
:10018000F7020008F702000800F002F800F096F805
:100190000AA090E8000C82448344AAF10107DA45E2
:1001A00001D100F08BF8AFF2090EBAE80F0013F09E
:1001B000010F18BFFB1A43F001031847502A04002F
:1001C000902A04000A444FF0000C10F8013B13F091
:1001D000070408BF10F8014B1D1108BF10F8015BA0
:1001E000641E05D010F8016B641E01F8016BF9D193
:1001F00013F0080F1EBF10F8014BAD1C0C1B09D1EA
:100200006D1E58BF01F801CBFAD505E014F8016B5B
:1002100001F8016B6D1EF9D59142D6D370470000ED
:100220000023002400250026103A28BF78C1FBD8FF
:10023000520728BF30C148BF0B60704766292CF0B9
:100240002A8165292CF0278167292CF024816129D6
:100250002CF02381692900F02D81642900F02A8186
:10026000752900F027816F2900F0BE81782900F000
:10027000E5810368DB0928BF41F08001632901F0B3
:100280003280E32901F04580002070471FB52CF033
:1002900032F89DE8030000F0D9FB01F003F90400F7
:1002A000002000212BF0A0F8401C606000200021FD
:1002B0002BF084F8E0601FBD10B510BD01F087FA87
:1002C0001146FFF7E3FF23F031FF01F0B3FA03B467
:1002D000FFF7F2FF03BC01F0E3FA00000948804792
:1002E00009480047FEE7FEE7FEE7FEE7FEE7FEE718
:1002F000FEE7FEE7FEE7FEE704480549054A064B30
:1003000070470000C14801088901000868A1001079
:1003100068DF001068C0001068C0001070B50646A5
:1003200000F074FB056806F10B0020F00704B442EE
:100330009CBF002070BD2B466A68BAB11068A0420D
:1003400010D304F1080188423CBF5068586007D3BD
:100350005168101941601168091B016058601460F0
:10036000101D70BD13465268002AE7D12146284669
:1003700000F058FB0028DED170BD70B50446051FA3
:1003800000F044FB0068002C14BF446870BD002CD2
:1003900018BFAC423CBF20466468F8D301680A1815
:1003A000AA4218BF456003D12A680546114401607E
:1003B00028684119A1421CBF6C6070BD616869600A
:1003C00021680844286070BD0FB41CB5074B06AA0D
:1003D0007B4469460090059800F063FF0020694661
:1003E00000F072FF1CBC5DF814FB0000F50E00006D
:1003F00070B5044685690068C10601D5302600E065
:100400002026C00707D070BDD4E9012130469047AF
:10041000206A401C20626D1EF6D570BD70B5044682
:1004200085690078C00707D170BDD4E9012120207B
:100430009047206A401C20626D1EF6D570BD096889
:100440004A0501D540B27047C905FCD500B27047D6
:1004500009684A0501D5C0B27047C905FCD580B20C
:10046000704770B50C460546012A05D028788006ED
:1004700000D5EA69002302E0012305E05B1C9342FA
:1004800002D2E05C0028F9D1A869E618C01AA86178
:10049000286A184428622846FFF7AAFF04E0D5E935
:1004A000012114F8010B9047B442F8D32846FFF716
:1004B000B5FF70BD2DE9F04106460024106875298E
:1004C000314616A510D0FFF7BAFF002802DA4042E5
:1004D00013A507E031688A0701D512A502E0490794
:1004E00004D511A5012401E0FFF7B2FF00210A2283
:1004F00006F1240709E0B0FBF2FCB0FBF2F302FBCB
:100500001C00303078541846491C0028F3D123468B
:100510002A463046BDE8F04100F0D9BA000000009C
:100520002D0000002B000000200000002DE9FF5FDF
:1005300015468A460446DFF8AC80F8440027D8E91F
:1005400000103E46CDE9001010E03AF816106A4659
:1005500002A800F022FF411C07D02178890603D5AC
:10056000E269391891420DD80744761C207880063C
:1005700002D5E069B84205DDAE42E6DB3AF8160086
:100580000028E2D1A069C01BA0612046FFF730FF20
:10059000D8E90010CDE90010002017E03AF8181053
:1005A0006A4602A800F0F9FEB0F1FF3F81460BD089
:1005B00000250DF1080B05E0D4E901211BF8050029
:1005C00090476D1C4D45F7D308F10100B0428046BD
:1005D000E4DB206A384420622046FFF71FFFBDE8B5
:1005E000FF9F000062BF020070B5044621461068FC
:1005F000FFF72EFF002104F1240505E000F00702BB
:100600003032C0086A54491C0028F7D12068002302
:1006100008A2050708D500F02000084304D0E069CF
:10062000012305A2401EE0612046BDE8704000F0B5
:100630004EBA0000000000003000000070B5044613
:100640000D4621461068FFF703FF2188090502D5F2
:100650000F4A7A4402E00E4A7A440E32002104F135
:10066000240305E000F00F060009965D5E54491C66
:100670000028F7D120780023000704D5702D02D080
:1006800009B1022311322046BDE8704000F01FBAC4
:1006900052BE02002DE9F05F894604464FF0000A81
:1006A000DFF874B1FB44C0F820A02046E168884719
:1006B000002874D0252806D0D4E901219047206A6B
:1006C000401C2062F1E700265F462046E16888472B
:1006D0002028054607DB312D05D2781910F8200CAB
:1006E00008B10643F1E7B00701D526F00406C4F8C7
:1006F0001CA00027C4F818A02A2D09D028462AF0EB
:10070000EFFC38B304EB8708303DC8F8185019E007
:1007100059F8041B204604EB87029161E168884781
:10072000012F054618D1E069002820DA26F02006BE
:100730001DE0D8F8180000EB800005EB40003038D1
:10074000C8F818002046E168884705462AF0C8FC2A
:100750000028EED1012F0AD02E2D08D12046E168C5
:1007600088477F1C0546022F46F02006C4DBA0699F
:10077000002803DA404246F00106A061F00701D0EC
:1007800026F010066C2D0BD0682D09D04C2D39D0D9
:100790006A2D35D0742D35D07A2D33D016E038E05F
:1007A000E1682F4620468847B842054609D16C2F9C
:1007B00026D04FF48060E16806432046884705460E
:1007C00004E06C2F1AD04FF4807006430DB3A5F1EE
:1007D0004100192802D8203546F400664A462946C9
:1007E000204626604E46FFF729FD80B101280BD038
:1007F000F61D26F0070000F1080956E74020E4E75F
:100800008020D8E70020D6E706F104094DE7284606
:1008100052E7206ABDE8F09F28BE020070B5064688
:1008200000F0F8F80468054630460A22002100F07E
:100830007CFD2C6070BD40EA010310B59B070FD111
:10084000042A0DD310C808C9121F9C42F8D020BA40
:1008500019BA884201D9012010BD4FF0FF3010BDF8
:100860001AB1D30703D0521C07E0002010BD10F8C6
:10087000013B11F8014B1B1B07D110F8013B11F88C
:10088000014B1B1B01D1921EF1D1184610BD40EA4D
:100890000103024630B59B0710D14FF0013400E050
:1008A00008C208C91D1B9D4315EAC41FF8D013F0E8
:1008B000FF0102F8011B0DD01B0AF8E711F8013BFC
:1008C000002B02F8013B05D011F8013B002B02F888
:1008D000013BF3D130BD10B5431C02E010F8011B01
:1008E00071B18107FAD14FF0013202C88C1A8C43E2
:1008F00014EAC211F9D0C01A0A0603D0C01E10BDF6
:10090000C01A10BD0A0401D0801E10BD0902FCD01F
:10091000401E10BD421E12F8013F002BFBD111F802
:10092000013B002B02F8013BF9D1704710B504469A
:1009300010F0030F08BF11F0030F40F015804FF0C7
:10094000013E121FC0F20E8051F8043BA3EB0E0CC7
:100950002CEA030C1CEACE1C08BF40F8043BF0D084
:10096000A1F1040102F10402521E08DB11F8013B5F
:1009700000F8013B002BF7D1114600F064FD204642
:1009800010BD00000000000030B44FF0013C50F8F2
:10099000042B51F8043BCCFA52F4D51A20D1FCB9FF
:1009A00050F8042B51F8043BCCFA52F4D51A17D165
:1009B000B4B950F8042B51F8043BCCFA52F4D51AD0
:1009C0000ED16CB950F8042B51F8043BCCFA52F418
:1009D000D51A05D1002CDAD030BC4FF0000070479A
:1009E00029BAB1FA81F111F01801D1F12000844047
:1009F000F2D1CA40CB4012F0FF0213F0FF0330BC2B
:100A0000D01A704770477047704700000048704721
:100A100038A401200048704730A401207047704777
:100A20007047704738B504460A4600206946AFF360
:100A30000080002808BF38BD02460099204600F01B
:100A400035FD012038BD012000F092BEF8B5AFF3AE
:100A50000080054600200C46102000BF0646A8195D
:100A6000A0420DD9324669460020AFF3008007004E
:100A700008BF00F07DFE0098A04218BF0546C419CB
:100A8000FFF7C4FF05600746F01D20F00700461978
:100A9000284600F00AF8B44208BFF8BDA21B314650
:100AA0003868BDE8F84000F001BD00210160C0E9F0
:100AB000011070471020704710B5FFF7ABFF0068BA
:100AC00010BD10B50446FFF7A5FF046010BD2DE969
:100AD000F0470D4699469246044600F12408016805
:100AE000880604D5E06921F01001216000E00120B2
:100AF000A84201DD471B00E00027A1697A1902EB3B
:100B00000900081AA0612078C00602D42046FFF729
:100B10006FFC002608E0D4E901211AF8060090478E
:100B2000206A401C761C20624E45F4DB2078C0060B
:100B30000AD52046FFF75CFC06E0D4E9012130200D
:100B40009047206A401C2062381EA7F10107F4DCA0
:100B500007E0D4E9012118F805009047206A401CFD
:100B60002062281EA5F10105F3DC2046FFF756FCA4
:100B70002078000602D50220BDE8F0870120FBE7BF
:100B80002DE9FF4F0C461E464FF0FF378BB0D2E9E0
:100B90000001DDF860800A908A46C1F30A5505B964
:100BA0003D46002108464FF00000BAF1000F00F466
:100BB000400005DA00EB80004FF4400101EA5000EC
:100BC0004FEA9059B9F1010F00DDB9460A9850EA91
:100BD0004A000ED044F61050A5F2FF3545432F14BD
:100BE000B8F1000F1ED07542291E1EDDC9F10002AA
:100BF0001CE0B8F1010F4FF0000001D0302103E0FC
:100C0000F24305E02154401CB042FBDB3046002299
:100C1000002121540B99C1F80880C1E900200FB0D0
:100C2000BDE8F08FBD1B6D1CDEE74A4600DA694265
:100C300006A800F02BFD06AB93E8070003AB83E8A2
:100C4000070050460A9927F0C9FA8DE80700A0F579
:100C500000501F3800900398002D0ADD42F21F015A
:100C60004A460844002303A90390684627F032FD52
:100C700009E0A0F500504A461F38002303A903905D
:100C8000684627F03CFD8DE807000004000C03D007
:100C90004FF0FF30410800E01046B8F1000F03D0DC
:100CA0000022009215461EE0751E05D400F018FCC7
:100CB000303262556D1EF9D5B3460122084302D089
:100CC00000227F1C04E02078302801D100227F1E02
:100CD000002A099784D01DE0112D07DA00F000FCEE
:100CE000303262556D1C50EA0102F5D1084302D042
:100CF0000098C8B10EE00021681E05E0235C625C2C
:100D000063542254401E491C8142F7DBAB46A81BAA
:100D1000401E0990002004F80B000B98099AC0F8B7
:100D20000880C0E9002B7AE711264FF0000857E74A
:100D30002DE9F04F88460446D21D22F0070191B0FC
:100D4000D1E90001CDE90A0127F010FE02460B9817
:100D5000C00F01D02D2007E02068810701D52B208E
:100D600002E0202101EAC000032A099001D0072AED
:100D700005DB03464146204600F0F8FB0BE12078F6
:100D8000800601D5E06900E00620B8F1650F8146D4
:100D900006D0B8F1660F18D0B8F1670F70D131E006
:100DA0000020B9F1110F009001DB112301E009F1DE
:100DB00001030AAA01A90CA8FFF7E2FEDDE90C7005
:100DC000002609F10105834647E001204B460090CB
:100DD0004FF000470AAA01A90CA8FFF7D1FEDDE9F0
:100DE0000DB00C995D46002610B909F101000D18EF
:100DF000B9EB050003D4C0F1FF3609F10105A5EBFD
:100E000009002BE0B9F1010F01DA4FF001090020D0
:100E1000B9F1110F0090484601DD112300E00346AF
:100E20000AAA01A90CA8FFF7ABFEDDE90C704D463C
:100E300000268346207800070AD4AB4500DA5D46D9
:100E400001A8012D04DD411911F8011C302907D03A
:100E50004F4502DA17F1040F04DA012082460FE051
:100E60006D1EEEE7002F02DCED1B3E4403E0781C14
:100E7000A84200DD7D1CB81B00F1010A4FF00047BD
:100E80002078000703D4AA4501DB4FF0FF3A002188
:100E9000B7F1004F0DF143088DF8431024D0022024
:100EA0002B23002F01DA7F422D230A21021EA0F1FD
:100EB000010000DC5FB197FBF1FC97FBF1F201FB55
:100EC0001C7C17460CF1300C08F801CDEEE7A8F1B8
:100ED000010003702188090501D5452100E0652145
:100EE000A0F1010800F8011C09980FA9A1EB08075F
:100EF000FF1D00B10120411901EBEA70A1693844DE
:100F0000081A401EA0612078C00602D42046FFF7D0
:100F10006FFA099828B1D4E901219047206A401C52
:100F200020622078C00622D52046FFF761FA1EE035
:100F3000002E04DBB34502DD01A8805D00E0302017
:100F4000D4E901219047206A401C2062761CAAF156
:100F500001005FEA000A0AD100F0A4FAC068016843
:100F6000405CD4E901219047206A401C2062281E81
:100F7000A5F10105DCDC07E0D4E9012118F8010B3B
:100F80009047206A401C2062381EA7F10107F3DC5D
:100F90002046FFF743FA032011B041E62DE9F04F58
:100FA00004460D46D21D22F0070089B0D0E9009713
:100FB0004846394627F0DAFC0246F80F01D02D23C7
:100FC00007E02068810701D52B2302E0202101EAF8
:100FD000C0038DF820300BB1012000E00020032A6F
:100FE000824601D0072A04DB2946204600F0BEFADB
:100FF0003FE12078800601D40D2500E0E569C7F3C4
:101000000A560D2D49DA00214FEA175B08464FF0CA
:101010000000002F00F4400007DA00EB80004FF4DE
:10102000400100EBD07001EA60008115012901DD6B
:101030004FF0FF3100224FEA850CBCF1180F06D3A8
:101040001346ACF118004FF08052C24003E04FF459
:10105000801323FA0CF30CF10C0CBCF1200F04D319
:10106000ACF1200C09FA0CF001E007FA0CF00029B1
:101070004FF0004801DD18B90FE00ED140450CD308
:1010800019EB02095F4121B9404502D19F4329EA8A
:101090000209BBEB175F00D0761C2088000502D543
:1010A0007B48784402E07A487844193808AA30230B
:1010B00002F80A30037C0AF10101002E0AF1020A4B
:1010C00053546A4602DC4FF0300101E04FF0310129
:1010D0004FF001088DF8001002D0A6F2FF3603E0B1
:1010E00059EA470100D06B4E002D02DC2178090738
:1010F00004D54FF002082E218DF80110C4460021BE
:101100000BE0C7F303433F01C35C491C6D1E02F8AB
:101110000830052908F1010801DA002DF1DC002171
:101120000CE000EB1973491C1B786D1E082902F8AE
:1011300008304FEA091908F1010801DA002DF0DC46
:1011400021688B0602D516E0A8F10108E04505DD0F
:1011500002EB080313F8013C302BF5D0B8F1000F77
:1011600009DD02EB080313F8013C2E2B03D109071C
:1011700001D4A8F10108002D05DD3E2102F8081078
:101180006D1E08F10108407C002E02F8080008F1ED
:10119000010804DA2D20764202F8080002E02B2034
:1011A00002F808000A214FF47A70864208F101081B
:1011B0000BDB96FBF0F3303302F8083096FBF0F3CC
:1011C00008F1010800FB136601E0642E0CDB6420CB
:1011D00096FBF0F3303302F8083096FBF0F308F199
:1011E000010800FB136601E00A2E06DB96FBF1F016
:1011F000303002F8080008F1010896FBF1F001FB1D
:101200001060303002F80800A16908F1010808EB0D
:10121000050202EB0A00081AA0612078C00602D479
:101220002046FFF7E5F8216A08AE01EB0A002062CC
:1012300004E0D4E9012116F8010B9047BAF1010A44
:10124000F7D22078C00602D52046FFF7D1F86E46C7
:1012500009E016F8010B3E280FD0D4E90121904790
:10126000206A401C2062B8F10108F2D22046FFF744
:10127000D5F809B00320BDE8F08F206A2844206229
:1012800003E0D4E90121302090476D1EEBD3F8E74D
:10129000ADB4020002FCFFFF01694A1C026108783C
:1012A000704700B58FB0CDE90131002105910549A6
:1012B0007944CDE9031011466846FFF7EBF90FB00A
:1012C00000BD0000E5FFFFFF0A6802F8010B0A609D
:1012D000704710B5436913B1AFF3008001E0FFF729
:1012E000C0F8012010BD127800F124010A7000221C
:1012F0004A700122EDE711684FF0FF32E9E710B5BF
:10130000436913B1AFF3008001E0FFF70FF901204B
:1013100010BD128800F1240182840022C2840122BF
:10132000EDE711684FF0FF32E9E72DE9F04791460C
:101330000F4680460446002614F8015B2DB100F0EC
:10134000A9F80068405DC007F6D12B2D02D02D2DE5
:1013500018D0641E4A463946204600F047F927B1A6
:101360003968A14201D1C7F800804FF0020471052D
:101370000BD54042002803DDFFF74CFB0460A007BB
:10138000BDE8F08746F48066E4E70028F8DAFFF766
:1013900041FB04606FF00040F2E72DE9F041164692
:1013A0000C46054600F076F8036893F80101012821
:1013B00007D0FF2C12D8185D80B101202C70BDE839
:1013C000F081D3F807013246214603F20713C7180C
:1013D0002846BC46BDE8F041002360474FF0FF308F
:1013E000EDE710B5203AC0F00B80B1E81850A0E846
:1013F0001850B1E81850A0E81850203ABFF4F5AFE3
:101400005FEA027C24BFB1E81850A0E8185044BF3E
:1014100018C918C0BDE810405FEA827C24BF51F8AB
:10142000043B40F8043B08BF7047D20728BF31F89F
:10143000023B48BF11F8012B28BF20F8023B48BFF0
:1014400000F8012B70474FF000020429C0F0128011
:1014500010F0030C00F09581CCF1040CBCF1020FEC
:1014600018BF00F8012BA8BF20F8022BA1EB0C013C
:1014700000F087B95FEAC17C24BF00F8012B00F8B7
:10148000012B48BF00F8012B70470000004870474F
:1014900030A4012010B500F005F8001D10BD00BFFC
:1014A000499F02000048704750A40120034640684D
:1014B0008C46002818BF88423CBF03464068F8D3DA
:1014C00018681844884207D00CF1030020F0070088
:1014D000001D411A521A0146081D0A60FEF74DBF51
:1014E00030B5B0F10A0271F100034FEA900E4EEAF6
:1014F000817EB0EB0E0061EB91014FEA101E4EEAC7
:10150000017E10EB0E0041EB11114FEA102E4EEA56
:10151000016E10EB0E0041EB11214FEA104E4EEA26
:10152000014E10EB0E0041EB1141401841F100015A
:101530004FEAD00040EA41704FEAD1014FEA8104FE
:1015400044EA907410EB800544EB01046D1944EB00
:101550000404521BA3414FF0000348BF0A3200D5D8
:1015600030BD401C41F1000130BD00002DE9F041CB
:101570001F46044603260168072A01F4006004DBC5
:1015800008B116A505E016A503E008B115A500E011
:1015900015A521F010002060A069C01EA0610FB148
:1015A000401EA0612046FEF723FF4FB1D4E9012180
:1015B00038469047206A401C2062C01C206206E02A
:1015C000206AFAE7D4E9012115F8010B9047761E4D
:1015D000F8D22046FEF722FFBDE8F0814E414E00D2
:1015E0006E616E00494E4600696E66002DE9F05F3F
:1015F000824615468B4600270AF10104B946007859
:10160000302801D09DB113E014F8010B0127782890
:1016100003D0582801D045B10AE00DB1102D07D1F3
:10162000002714F8010B102502E0082500E00A2528
:101630000026B0460EE005FB080005FB06F1012779
:101640001FFA80F801EB1046B6F5803F00D3B9468B
:1016500014F8010B294600F0DFF80028EBDABBF1A3
:10166000000F05D00FB1641E00E05446CBF80040D7
:10167000B9F1000F06D0FFF7CDF902210160C81EB5
:10168000BDE8F09F48EA0640FAE700002DE9F04780
:10169000814616468AB0354878440DC88DE80D005D
:1016A00032487844801C03AC0DC884E80D0041F634
:1016B0009B300844372190FBF1F290FBF1F5A5F146
:1016C000800501FB12041B3C02D56442012000E0AE
:1016D0000020DFF898A080460027FA44AAF1BE0A4D
:1016E0000EE0E0070AD03246684607EB47010123C7
:1016F0000AEB810127F003F88DE8070064107F1CD6
:10170000002CEED1194F7F44AE3F19E0E80715D009
:1017100007EB04100DF1180A90E80E008AE80E009D
:10172000C068F04201D1981908903246012306A9F9
:1017300003A826F0E4FF03AB83E807006D10641CE8
:10174000002DE3D14FF0010332466946B8F1000F96
:1017500003A802D026F0BEFF01E026F0D0FFC9E9C1
:101760000001C9F808200AB0BDE8F08738B00200CF
:1017700010B500F06DF8BDE8104000F064B84FF00F
:10178000000200B5134694469646203922BFA0E8D1
:101790000C50A0E80C50B1F12001BFF4F7AF0907DD
:1017A00028BFA0E80C5048BF0CC05DF804EB8900CE
:1017B00028BF40F8042B08BF704748BF20F8022B11
:1017C00011F0804F18BF00F8012B70477047754625
:1017D000FFF75CFEAE4605006946534620F0070061
:1017E000854618B020B5FEF787FDBDE820404FF0D4
:1017F00000064FF000074FF000084FF0000BAC461A
:10180000ACE8C009ACE8C009ACE8C009ACE8C00964
:1018100021F007018D4670473A2800D2303820F079
:101820002002412A01D3A2F13700884201D34FF0B0
:10183000FF30704710B50446AFF300802046BDE886
:101840001040FEF744BD002801D000F029B87047D1
:1018500010B5012805D0002103A000F027F80120D1
:1018600010BD09A1F8E7000053494752544D454DBA
:101870003A204F7574206F662068656170206D6531
:101880006D6F7279000000003A2048656170206D2C
:10189000656D6F727920636F727275707465640024
:1018A00001491820ABBEFEE72600020070B50546D0
:1018B0000C460A2000E06D1C00F011F835B12878C4
:1018C0000028F8D102E0641C00F009F814B1207877
:1018D0000028F8D1BDE870400A20AFF3008008B5B9
:1018E00069468DF800000320ABBE08BD53EA020C28
:1018F00000F069802DE9F04B4FF00006002B1FBF70
:10190000B3FA83F503FA05F424FA05F65E4012BF34
:101910001643B2FA82F502FA05F4C5F120051EBF9E
:1019200022FA05FC44EA0C04203556EA044C4FEA3E
:10193000144418BF641C4FF000084FF00009904297
:1019400071EB030C39D3002919BFB1FA81F701FA01
:1019500007F6B0FA80F700FA07F6C7F120071EBFB6
:1019600020FA07FC46EA0C062037B6FBF4FCA7EB8E
:101970000507103F07F01F0BCBF120062CFA06F6E7
:101980000CFA0BFB44BFB3460026202FA4BF5E46D3
:101990004FF0000B5BEA060C08BF4FF0010B19EB90
:1019A0000B0948EB0608ABFB027C06FB02CC0BFBE9
:1019B00003CCC01B71EB0C01C1E70B46024641464C
:1019C0004846BDE8F08B13B5084318BF4FF0FF3011
:1019D0000146AFF30080BDE81C407047032A40F287
:1019E000308010F0030C00F0158011F8013BBCF1C1
:1019F000020F624498BF11F801CB00F8013B38BFD9
:101A000011F8013BA2F1040298BF00F801CB38BFE6
:101A100000F8013B11F003033FF4E3AC083AC0F0D7
:101A2000088051F8043B083A51F804CBA0E80810AC
:101A3000F5E7121D5CBF51F8043B40F8043BAFF3DF
:101A40000080D20724BF11F8013B11F801CB48BF39
:101A500011F8012B24BF00F8013B00F801CB48BF6F
:101A600000F8012B704702F0FF0343EA032242EA29
:101A70000242FFF7EABC02F0FF0343EA032242EA14
:101A80000242FFF77EBE0000002070472DE9F04FB4
:101A900081B04CF24064C2F20104D4F8100345F264
:101AA0006261C2F2010145F662721830C2F20102AF
:101AB000002526C020461CF061FDD4F81093B9F132
:101AC000000F56D048F21867C1F20007388848F274
:101AD000185B4CF278240FF2B00AC1F2000BC2F28C
:101AE000010400260AE000BF81B2B1F5807F06F153
:101AF000010624BF002038801E2E1CD01AF80610C4
:101B000082B20BF802100130218882B28A423880FA
:101B1000EAD14FF0000800BF00F07CF9B5EB582F78
:101B200003D1012808F10108F6D000F073F901286B
:101B300001D03888D8E74CF24060D9E90712C2F2E8
:101B40000100D0F820030A444FF490730027C0F836
:101B50005C22C0E9993703690327012BA0F8507272
:101B600008BFC0F8602200F514710068DAB21EF0F8
:101B70008DF94CF22121C2F20101012200200A70EC
:101B800001B0BDE8F08F00BF5B4F4B5D2053746127
:101B90007274205265636569766520555342204111
:101BA0007564696F0D0A00004AF22850C2F2010004
:101BB0000178012919D10021017041F204004AF293
:101BC0002452CEF20000C2F2010242F670230168F4
:101BD0001268C1F200031F68891A3944196000684D
:101BE00042F67421C1F2000108604EF2FF054AF28C
:101BF000FC4640F21847C0F2F5550FF22C08C2F22D
:101C00000106C4F202074FF4800400E03C60404645
:101C100000210BF017FB00BF3068A842F6D201305C
:101C2000306000BFF8E700BF427573204661756CF5
:101C30007400000021280DD0202815D10868D1F8A3
:101C4000031042F66412C1F20002C2F803101060E1
:101C50000020704742F66410C1F20000D0F8032063
:101C60000068C1F80320086000207047002070471A
:101C70004CF24060C2F20100D0F80C130020086260
:101C800042F64C204AF20052C1F20000C2F20102B8
:101C9000486100208A6170472DE9F04F91B00DF145
:101CA000040A0C46064650464021FFF768FD2268AC
:101CB00050463146FEF73AFE206801383F2803D9E6
:101CC000002011B0BDE8F08F47F6046B47F6C4560C
:101CD0004CF234284FF00009C1F2000BC1F20006AB
:101CE000C2F201080020002519E000BFC7F1400141
:101CF00008EB07003F2F88BF0021FFF7A4FB4046F9
:101D000031463A46FFF76DFB304640218BF8009094
:101D1000FFF735FD01352168A8B28142D0D91AF804
:101D200000000028F6D09BF800703B28F055DDD06D
:101D3000781CC1B240298BF80000E5D2EAE7000028
:101D400022281BD021280DD0202828D10868D1F8BE
:101D500003104AF20842C2F20102C2F803101060F6
:101D6000002070474AF20840C2F20100D0F8032078
:101D70000068C1F8032008600020704788780128B7
:101D800007D147F6A510C1F2000001210170002023
:101D9000704747F6A510C1F2000000210170002035
:101DA00070470000002070474CF24060C2F2010012
:101DB000D0F80813002008624AF2485042F69022F8
:101DC000C2F20100C1F20002486100208A6170473E
:101DD00080B54CF24061C2F20101D1F80833D1F86C
:101DE0002023586110234FF0000CC2F82402C2E9EE
:101DF0008B3C13694FF0010C012BA2F818C208BFED
:101E0000C2F82802106802F50671DAB21EF03EF838
:101E1000002080BD2DE9F04F81B04BF25355C2F246
:101E200001052878C8B948F218604CF2782BC1F245
:101E30000000C2F2010BB0F80080BBF80060B045B2
:101E400003D1002001B0BDE8F08F4CF2406AC2F22D
:101E5000010ADAF80873786A18B1032001B0BDE806
:101E6000F08F4DF2D8440120C2F2010428702046C0
:101E70004FF48071FFF783FCB0452DD2FF2E55D86B
:101E800048F21850C1F200008119C6F1FF0082B279
:101E90003F2A28BF3F20013082B24DF2D840C6F51C
:101EA0008079C2F20100A0461FFA89F4FFF796FD7F
:101EB00006F140003C2162183D2A3DD03E2A3FD029
:101EC0003F2A3FD000293FD0043962183C2A06F14E
:101ED0000406F0D1304639E02BD948F21850C1F24F
:101EE00000008119F043404482B23F2A28BF3F20BE
:101EF000013082B24DF2D840A8EB0609C2F20100CF
:101F00001FFA89F4FFF76AFD06F140003C216218D0
:101F10003D2A13D03E2A25D03F2A25D041B304398B
:101F200062183C2A06F10406F1D11EE04FF00009C8
:101F300010E04FF0000923E0701C07E0013614E0C8
:101F4000B01C03E0F01C01E04FF040094446064697
:101F5000ABF80000B0B2B0F5807F04BF0020ABF852
:101F600000000DE0023600E00336ABF8006003E04D
:101F7000ABF800004FF040094DF2D844C2F2010422
:101F8000786AE0B91FFA89F0BC613862796AB1B940
:101F900001217962DAF8202340F20113114621F879
:101FA000583F1369CAF83400D06600205466012BEC
:101FB000106708BF94661068DAB21DF067FF002052
:101FC0002870012001B0BDE8F08F00004AF22850CF
:101FD000C2F20100017801291BD1002141F2040C59
:101FE0004AF224520170CEF2000CC2F2010242F613
:101FF0007023DCF800101268C1F200031868891A17
:1020000008441860DCF8000042F67421C1F20001B7
:1020100008604CF6AC10C2F2010004F011BA0000E6
:102020004AF22850C2F20100017801291BD1002197
:1020300041F2040C4AF224520170CEF2000CC2F2BA
:10204000010242F67023DCF800101268C1F20003AE
:102050001868891A08441860DCF8000042F67421F8
:10206000C1F20001086049F62400C1F2000004F04A
:10207000E7B900004AF22850C2F2010001780129B4
:102080001BD1002141F2040C4AF224520170CEF21D
:10209000000CC2F2010242F67023DCF80010126854
:1020A000C1F200031868891A08441860DCF80000BF
:1020B00042F67421C1F2000108604CF60C20C2F215
:1020C000010004F0BDB900004AF22850C2F201003C
:1020D000017801291BD1002141F2040C4AF224525B
:1020E0000170CEF2000CC2F2010242F67023DCF85D
:1020F00000101268C1F200031868891A08441860B9
:10210000DCF8000042F67421C1F2000108604CF6D0
:102110006C20C2F2010004F093B9000080B54CF6C7
:10212000CC20C2F2010004F08BF9BDE8804001F040
:1021300029BC000080B54AF22850C2F201000178A3
:1021400001291BD1002141F2040C4AF224520170F2
:10215000CEF2000CC2F2010242F67023DCF800104D
:102160001268C1F200031868891A08441860DCF884
:10217000000042F67421C1F2000108604CF62C30D8
:10218000C2F2010004F05CF9BDE8804001F014BE29
:102190004AF22850C2F201000178012918BF7047A5
:1021A000002141F2040C4AF224520170CEF2000CDC
:1021B000C2F2010242F67023DCF800101268C1F28C
:1021C00000031868891A08441860DCF8000042F619
:1021D0007421C1F200010860704700002DE9F0434E
:1021E00081B02DED088B82B047F2F079C1F2000981
:1021F0004AF2685720F0010009F26911C2F20107A2
:10220000022808BF09F5B5713E6840F2000540F6A6
:10221000007406EB4600C1F20005C2F2000491F81A
:10222000008005EB002021464FF44072FFF7D9F8FB
:10223000701C022888BF0020386000EB400005EBCE
:10224000002120464FF44072FFF7CBF800200090A9
:10225000684620F0CFFF9DED000AB5EE400AF1EE92
:1022600010FA06D141F26F209FEDB50AC3F6832024
:102270000090B5EE001A20EE010AB0EEC00A01A8E7
:1022800027F012FC4CF22920C2F2010001784AF238
:10229000F4400029C2F201004DD101EE108AB8EEDF
:1022A000412A9FEDA81A9FEDA83A20EE011A31EEBF
:1022B000031A9FEDA63A21EE001A31EE031A21EE21
:1022C000000A9DED011A9FEDA23AB8EEC11A31EE57
:1022D000031A31EE000A9FED9F1A99F95E2190EDE5
:1022E000003A20EE010A01EE102AB8EEC11A30EED3
:1022F000034A31EE444A98A2B5EE404AF1EE10FA94
:10230000C8BF043292ED005A24EE022A22EE052ABA
:1023100032EE032AB1EE084A32EE003A31EE044AB8
:10232000B4EE443AF1EE10FA80ED002AC4BF31EE6B
:10233000400A80ED000A99F8012009F13803002ACB
:1023400008BF09F11C031A78002A04BF4FF07E521F
:10235000026011B19FED820A08E090ED001AB3EE21
:102360000E0AB4EE401AF1EE10FA03DDB0EE401A98
:1023700080ED000A42F62428C1F2000898ED008A98
:1023800038EE410AB5EE400AF1EE10FA60D09FED4A
:10239000752AB4EE418A20EE022A9FED730AF1EE0F
:1023A00010FAB0EE409AC8BFB0EE429A9FED6F2A85
:1023B0009FED6FAA31EE483AB4EE418A002600271D
:1023C00023EE022AF1EE10FAB8BFB0EE429A18E0FE
:1023D00038EE098A88ED008A0127A51928EE0A0A35
:1023E00095ED00BA10EE100A28F0C8FE00EE100AB3
:1023F000043620EE0B0AB6F5407F85ED000A00F0AA
:102400009880B5EE400AF1EE10FA07DAA01990EDC7
:10241000001AB5EE401AF1EE10FAD9DCB5EE400A1A
:10242000F1EE10FA10DDA01990ED000A0020B5EED3
:10243000400AF1EE10FAB8BF01203843C0074FF050
:102440000007C5D1C9E700BFF807C1D10027C4E71D
:102450009FED470A21EE000A10EE100A28F08EFECA
:1024600000EE100A6FF03F00211891ED101A91ED67
:10247000112A91ED123A91ED134A21EE001A22EE43
:10248000002A23EE003A24EE004A81ED101A81ED75
:10249000112A81ED123A81ED134A91ED141A91ED52
:1024A000152A91ED163A91ED174A21EE001A22EE07
:1024B000002A23EE003A24EE004A81ED141A81ED41
:1024C000152A81ED163A81ED174A91ED181A91ED12
:1024D000192A91ED1A3A91ED1B4A21EE001A22EECB
:1024E000002A23EE003A24EE004A81ED181A81ED0D
:1024F000192A81ED1A3A81ED1B4A91ED1C1A91EDD2
:102500001D2A91ED1E3A91ED1F4A403021EE001A2E
:1025100022EE002A23EE003A24EE004AB0F5307F86
:1025200081ED1C1A81ED1D2A81ED1E3A81ED1F4AB5
:102530009AD102B0BDEC088B01B0BDE8F08300BFBA
:102540006F12833AA8A19D3FF5CA83C0FBB3C04078
:10255000E09248C0C2A8C040CDCC4C3D0AD7A33BB6
:10256000000048C3ABAAAABB00000000ABAAAA3B6C
:102570002D152A3E2DE9F04F83B016460C9A984649
:102580000C46002A05467AD047F2E2794AF2F84032
:10259000C1F200090127C2F201004FF0000B310126
:1025A00040F2004389F8007080F802B0417080F872
:1025B00000B042F62710C4F202034FF4805AC1F271
:1025C000000000210122CDF800A001970DF04AFE85
:1025D00000285CD040F200494AF2F840C4F20209F7
:1025E000C2F20100002103224B46CDF800A0019762
:1025F0000DF038FE0020294622464B46CDF800A0BB
:10260000CDF804B00DF02EFEB8F1000F2FD04DF232
:1026100034380120C2F2010800904046214632467B
:1026200000230026FFF7A6FFC4F1000CA4F1010E61
:1026300018F80600A95D884242D1B64517D008EBCC
:102640000603AF1958787978884239D10CEB060126
:10265000881C0CD09878BA78904231D1C81C06D02A
:10266000D878F97888422BD10436B442E0D147F2C9
:10267000E2710020C1F200010127087029E04AF24E
:102680006D50C2F20100007880B1012721E04AF2CA
:102690006D50C2F20100077010A025F0A3FB16A038
:1026A00001210AF0CFFD89F800B012E047F2E27094
:1026B000C1F20000007800283FF466AF002708E070
:1026C00047F2E2740021C1F20004002725F0C2FCA9
:1026D0002770384603B0BDE8F08F00BF5B4552520B
:1026E0005D20454550524F4D206E6F7420666F75CA
:1026F0006E642E2E2E000000454550524F4D20692D
:102700006E6974206572726F720000002DE9F04FDF
:1027100083B04AF26D50C2F201000078002848D11F
:1027200040F200494AF2580A49F6EC65C4F202093F
:1027300000204FF48057C2F2010A0DF10B0BC1F2D9
:1027400000054FF000088DF80B0001E0C72E2DD2D8
:102750005046002101224B460124464608F101085B
:10276000009701940DF07EFD0020594601224B4652
:102770000024009701940DF075FD9DF80B00C00733
:1027800011D028682968091A0229DFD22968091A94
:102790000129DBD82968091A0129D7D82968091A1B
:1027A0000229EFD3D2E7B8F1C80F02D102A025F079
:1027B00019FB03B0BDE8F08F5B4552525D454550B3
:1027C000524F4D204C6F636B2077616974206572A6
:1027D000726F72002DE9F04F87B014464AF26D52C5
:1027E000C2F2010212780AB10125FBE047F2E2725F
:1027F000C1F200020B46014610780025002840F087
:10280000F180012010704DF6DC5040F20049C2F218
:1028100001001A46C4F202090693FFF7DFF8069991
:102820004AF2F84A080A059003942003C2F2010A0A
:102830004FF4805B002400274FF00108049000BF94
:102840000498A1EB042600EB0420020C000A8AF88D
:102850000100B0B2B0F5807F4AF2B4308AF80220AD
:10286000C2F201004FF000014FF001024B468AF81E
:10287000005028BF4FF48076CDF800B001950DF0E0
:10288000F1FC4AF24430C2F20100002101224B4621
:10289000CDF800B0CDF804800DF0E4FC50460021E6
:1028A00003224B46CDF800B0CDF804800DF0DAFCE1
:1028B0004DF6DC50C2F2010000EB0420B2B2002160
:1028C0004B46CDF800B001950DF0CCFCFFF71EFF94
:1028D000013705980699BCB2A042B1D249F6F1651C
:1028E000039CC1F200054FF0010B2846224600234D
:1028F000CDF800B000270E46FFF73CFE4DF6DC5E3B
:10290000C2F2010E28789EF8001047F2E278884261
:102910004FF00101C1F2000830D171420220B446EB
:102920000A18012A1DD02B180EEB000713F8016CB2
:1029300017F8014CA64216D19AB12E5C1EF8004041
:10294000A64213D1561C0CD05E787C78A6420CD1DE
:10295000023206D09A78BB7804309A42E0D002382E
:1029600004E0002639E0013800E001300021604534
:1029700038BF0121039C00274FF0010B200188F88C
:1029800000B08AF801004AF2B4304FF48054C2F229
:1029900001000E46002101224B468AF802708AF897
:1029A0000070009401970DF05DFC42F62810C1F212
:1029B0000000002101224B460094CDF804B00DF038
:1029C00051FC5046002103224B46009401970DF024
:1029D00049FCFFF79BFE88F80070002086F0010597
:1029E00088F80000284607B0BDE8F08F4AF228506A
:1029F000C2F20100017801291BD1002141F2040C2F
:102A00004AF224520170CEF2000CC2F2010242F6E8
:102A10007023DCF800101268C1F200031868891AEC
:102A200008441860DCF8000042F67421C1F200018D
:102A3000086043F61440C4F201000168C90708BFEA
:102A40007047012101601BF075B900004AF228505F
:102A5000C2F20100017801291BD1002141F2040CCE
:102A60004AF224520170CEF2000CC2F2010242F688
:102A70007023DCF800101268C1F200031868891A8C
:102A800008441860DCF8000042F67421C1F200012D
:102A900008604FF4806003F02FBF00004AF2285016
:102AA000C2F20100017801291BD1002141F2040C7E
:102AB0004AF224520170CEF2000CC2F2010242F638
:102AC0007023DCF800101268C1F200031868891A3C
:102AD00008441860DCF8000042F67421C1F20001DD
:102AE000086043F61440C4F201000168890758BF2A
:102AF0007047022101601BF01DB900004AF2285006
:102B0000C2F20100017801291BD1002141F2040C1D
:102B10004AF224520170CEF2000CC2F2010242F6D7
:102B20007023DCF800101268C1F200031868891ADB
:102B300008441860DCF8000042F67421C1F200017C
:102B40000860042003F0D8BE4AF22850C2F2010007
:102B5000017801291BD1002141F2040C4AF22452D0
:102B60000170CEF2000CC2F2010242F67023DCF8D2
:102B700000101268C1F200031868891A084418602E
:102B8000DCF8000042F67421C1F200010860082060
:102B900003F0B2BE4AF22850C2F2010001780129C6
:102BA0001BD1002141F2040C4AF224520170CEF2F2
:102BB000000CC2F2010242F67023DCF80010126829
:102BC000C1F200031868891A08441860DCF8000094
:102BD00042F67421C1F20001086043F61440C4F2C9
:102BE00001000168090658BF70478021016049F65D
:102BF000EC60C1F2000000684DF29C21C2F20101BC
:102C0000086070472DE9F04F83B04AF20800C2F225
:102C10000100D0F800909FEDE72A99F85E20B3EE0E
:102C2000091A1146002A18BFFF21009147F2F071DE
:102C3000C1F20001B2EE040A91F88A110192002A51
:102C400008BFB0EE410A32EE401AB7EE002A82EE1B
:102C5000011A82EE002A9FEDD83A9FEDD84A9FEDE7
:102C6000D85A9FEDD86A9FEDD87ADFEDD80A0023B5
:102C70004FF0320A43F2CE1C481E2B2445F20A05BF
:102C80000290A3E041EA022E4DF23621C2F2010188
:102C900021F813E0B9F85610B9F8502005EE90AAC3
:102CA000891AB9F85860B9F852B001EE901AF8EEE6
:102CB000655A04EE902AF8EEE11A65EE835AA6EB07
:102CC0000B01B9F85A60B9F85480F8EE644A65EE21
:102CD000A11A02EE901A71EEA41AA6EB0801F8EE02
:102CE000E22AFCEEE11A04EE90BA03EE901A11EE1D
:102CF000901AF8EE641A65EEA22A72EEA11AFCEEA2
:102D0000E11A11EE902A4FF478461FFA8EF706EA80
:102D1000012102F0FC0241EAC201FA0A02EE908AA5
:102D2000152A4FF01502C7F34516F8EEE31A38BF1F
:102D3000FA0A0EF01F072B2EF8EE622A65EEA11A92
:102D400028BF2646152F4FF0150028BF074647EA33
:102D5000C22271EEA21AFCEEE11A06F114072A440F
:102D600042EA471211EE907AC7F3C40749F6FC56BF
:102D70003944C1F2000626F813104DF2D016C2F203
:102D8000010626F81320CA0A152A4FF0150238BF8B
:102D9000CA0AC1F345112B2928BF2146152F28BF88
:102DA000074647EAC22214312A4449F6626042EAE1
:102DB0004111C1F2000020F8131001330298AAF16A
:102DC000010A332BACF1FF0C00F02B81062824D82C
:102DD000DFE800F01C2644637C990400CAEB0A215A
:102DE00048F21F5089B2C5F2EB10A1FB0012FF2080
:102DF000019FA0EB1211002F08BF110901F0FC0781
:102E0000FF0001F0F80247EAD1013BE7322B40F026
:102E10009580009F00223946E4E04FF6FF7E33E7BD
:102E200001EE90AAF8EE611AB4EE610AF1EE10FA22
:102E300040F3988001EE90CAF8EE611A62EE211A12
:102E40000199FCEEE11A002911EE907A00F0DC8085
:102E5000C7F1FF024FF47841FF27DAE001EE90AAB4
:102E6000F8EE611AB4EE610AF1EE10FA40F38E80CA
:102E700001EE90CAF8EE611A62EE211A0199FCEE99
:102E8000E11A002911EE907A00F0B580C7F1FF0138
:102E9000C1F3C401FF27FF22AFE0CAEB0A2148F2C9
:102EA0001F5089B2C5F2EB10A1FB001201994FF43B
:102EB00078470029009918BFA1EB121108BF07EA53
:102EC000021701F0FC0247EAC20217E0CAEB0A212E
:102ED00048F21F5089B2C5F2EB10A1FB0012019914
:102EE0004FF4FC660029009918BFA1EB121101F004
:102EF000F80708BF06EA520646EA0722C1F3C401F2
:102F000002EB010EC0E6CAEB0A2148F21F5089B25B
:102F1000C5F2EB10A1FB001201991F2600290099B0
:102F200018BFA1EB121101F0F80701F0FC0108BF76
:102F3000D60946EAC10141EA072EA5E601EE90AAAC
:102F40001B2BF8EE611A43D361EE841A71EE851AD9
:102F5000FCEEE11A11EE901AC1F1FF02C2F3C402B5
:102F60000F463FE070EE611A61EEA01A61EE811A21
:102F700071EEA01AFCEEE11A11EE907A01993A4630
:102F8000002908BF0A464FF4784142E070EE611A0A
:102F900061EEA01A61EE811A71EEA01AFCEEE11A40
:102FA000019911EE902A002917464FF0000108BF41
:102FB000FF2722E0000048420AD7A33C0429314100
:102FC000042931C157F619C1E890F04300007F434E
:102FD00061EE861A71EE871AFCEEE11A11EE901A74
:102FE000FF27002201F0FC0107F0F80742EAC101C7
:102FF00041EA072E48E600213A4607F0FC0702F0B6
:10300000F80241EAC7013DE64FF4784101EA0721A1
:103010000022C2F3C40207F0FC07114341EAC70EC5
:1030200032E647F2F076C1F2000696F887014FF4D7
:103030000074022859D34FF64471C0F6030151F8C9
:1030400020104AF25C00C2F2010042F60C158160C9
:10305000C1F200054068A9602821FEF790FB68686E
:103060002821FEF78CFB96F88761B4FBF6F07043DD
:10307000D0F5007035D142F21C7106EB4600C0F667
:10308000030101EB80004788456840F2FC7048F27C
:103090001C684AF2505900EB8704C1F20008C2F2E2
:1030A000010940462146A9F80270C9F80450FEF70C
:1030B00066FBC9F8088042F6D028C1F20008C8F8BB
:1030C000045048F62865C1F200052846214689F8D3
:1030D0000060A8F80270FEF752FBC8F8085088F8A4
:1030E00000604FF40070B0FBF6F44DF67070C2F261
:1030F0000100046041F60000C2F200004BF680318E
:10310000FEF7A1F94DF28030C2F2000046F22071C4
:103110003222FEF7B0FC43F64460C1F200004FF4E7
:103120008051FEF72CFB03B0BDE8F08F00000000DB
:103130002DE9F04F81B02DED108B8CB047F2F0707F
:10314000C1F2000090F889A1BAF1010F40F040816E
:103150009FEDBF0BCDF800A025F0E2FD9FEDBE1B5B
:1031600051EC100B53EC112B28F0DAFC41EC100B56
:1031700026F0E6F89FEDBA1B9FEDBB2B51EC110B2F
:103180009FEDBB1BCDE9031051EC120B9FEDBAABC9
:10319000CDE9011051EC110B9FEDB98BCDE90A106F
:1031A00057EC100B9FEDB8CA099051EC1A0B9FED2C
:1031B000B8DBB0EE4AEAB0EE4A0A0026C80F59EC76
:1031C000188BF0EE6AEAF0EE6A0A08903BE000BF66
:1031D000284631462A46334628F05AF99FED9C0B83
:1031E00053EC102B28F054F928F020F9079E4DF2EB
:1031F000DC5240F2FF11C2F20102891B42F82600A4
:1032000042F8210052F8260028F0DAFF82468B4669
:1032100054EC1E5B2846214652465B4629F01EF8B8
:1032200000281CBF5C465546DDE9050142464B4679
:1032300044EC1E5B28F02CF941EC100B013640F2F7
:10324000011086427AD0DDE9033251EC100B07966B
:10325000CDE9050128F064FCDDE9013228F018F918
:10326000B0EE48BAB0EE4AFA82468B460224F0EE3F
:1032700068BAF0EE6AFA30E025F052FD53EC1D2BEF
:1032800051EC100B28F04CFC41EC100B26F058F8D8
:10329000B0EE409AF0EE609A53EC1B2B5046594624
:1032A00028F03EFC27F05AFF02460B4651EC190B62
:1032B00028F036FC53EC1F2B28F0EAF8054641ECC9
:1032C0001F0B20460E4628F09FFB41EC1B0B0134E0
:1032D00040F2011084423FF47BAF601E00EE100A02
:1032E000B8EE400A20EE0C0A10EE100A28F068FF33
:1032F000DDE90A3228F014FC27F030FF099A3B463A
:1033000028F00EFC089A41EC190B62F3DF7142467B
:103310004B4628F08EFFB0EE490AF0EE690A00280D
:10332000AAD125F051FB53EC1D2B51EC100B28F0CA
:10333000F7FB27F013FF41EC190BADE79FED500BA6
:103340002A4651EC100B234628F056F981464DF2DF
:10335000DC50C2F20100DDF800A00D46A0F110061D
:103360004FF4007456F8100F28F02AFF02460B465F
:103370004846294628F0D4FB28F058F8306006F17A
:10338000040898E8810128F01BFF02460B464846D6
:10339000294628F0C5FB28F049F87060384628F027
:1033A0000FFF02460B464846294628F0B9FB28F095
:1033B0003DF8B060404628F003FF02460B46484601
:1033C000294628F0ADFB28F031F8043CF060C9D163
:1033D0004DF2DC579FED309A9FED30BA9FED30CA29
:1033E00040F288499FED2FDA9FED2FFADFED2FFA9B
:1033F000DFED2F8ADFED2F9ADFED2FAADFED2FBA59
:10340000DFED2FCADFED2FDA4FF00008C2F201071F
:10341000B7EE008AAAF10206B5EE00AAC0F60409CA
:103420000024B6EE00EA06E00134B4F5007F07F1AF
:10343000040700F08382052EF6D8B0EE480ADFE8D4
:1034400016F079001001BB014A024600430000BF9C
:1034500000000000006AF840800001020408603F9C
:1034600000000060FB21893F000050626A1509C01E
:10347000000000000000603F0000000000000000AD
:10348000000000000000F03FDB0F494000BF00BF1C
:103490000000000000F07F402040003B000000449E
:1034A000000000C42040803B3060C03BBDE00B3ECC
:1034B0007975FABE02582EBC6827BA3E0000003B60
:1034C0001F85EB3E713D0A3F87ED000AACE700EE39
:1034D000104AB8EE400A20EE090A30EE0A0ABDEEA4
:1034E000C01AB8EEC11A30EE410A20EE0B0ABDEE4A
:1034F000C01A11EE100AB8EB502F30EE0C1A1CBF98
:10350000B0EE410A002009EB800101EE100A91EDB6
:10351000002A91ED013AB8EE411A30EE410A32EE3E
:10352000431A21EE000A30EE420A20EE2C0A30EE59
:103530002D0AC9E700EE104AB8EE400A20EE091A3B
:1035400031EE0A1ABDEEC12AB8EEC22A31EE421A95
:1035500021EE0B1ABDEEC12A12EE100AB8EB502F65
:1035600031EE0C2A1CBFB0EE421A002009EB80019C
:1035700002EE100A91ED003A91ED014AB8EE422AAE
:1035800031EE421A34EE432A22EE011A20EE0D2AC1
:1035900032EE0A2A31EE031ABDEEC23AB8EEC33A51
:1035A00032EE432A22EE0B2ABDEEC23A13EE100A87
:1035B000B8EB502F32EE0C3A1CBFB0EE432A00207D
:1035C00009EB800103EE100A91ED004A91ED015ADA
:1035D000B8EE433A20EE0F0A32EE432A35EE443A73
:1035E00030EE0A0A23EE022ABDEEC03AB8EEC33A24
:1035F00030EE430A20EE0B0ABDEEC03A13EE100A7D
:10360000B8EB502F30EE0C3A1CBFB0EE430A00204E
:1036100009EB800132EE042A03EE100A91ED004A14
:1036200091ED015AB8EE433A30EE430A35EE443A92
:1036300023EE000A9FEDCF3A30EE040A22EE032A71
:103640009FEDCD3A21EE031A9FEDCD3A31EE031AEC
:1036500031EE021A9FEDC92A20EE020A31EE000A6D
:1036600032E700EE104AF8EE40EA2EEE890A30EE1C
:103670000A0ABDEEC01AB8EEC11A30EE410A20EEB9
:103680000B0ABDEEC01A11EE100AB8EB502F30EE47
:103690000C1A1CBFB0EE410A002009EB800101EEBC
:1036A000100A91ED002A91ED013AB8EE411A30EE80
:1036B000410A33EE421A21EE000A2EEE8D1A31EE47
:1036C0000A1A30EE020ABDEEC12AB8EEC22A31EE65
:1036D000421A21EE0B1ABDEEC12A12EE100AB8EB07
:1036E000502F31EE0C2A1CBFB0EE421A002009EB1D
:1036F000800102EE100A91ED003A91ED014AB8EE18
:10370000422A31EE421A34EE432A22EE011A9FED8C
:10371000962A31EE031A20EE020A9FED942A30EE2B
:10372000020A9FED932A21EE021A30EE010A10EEF2
:10373000100A28F045FD2EEE8F0A30EE0A0ABDEE83
:10374000C01AB8EEC11A30EE410A20EE0B0ABDEEE7
:10375000C01A824611EE100A0D46B8EB502F30EE1B
:103760000C1A1CBFB0EE410A002009EB800101EEEB
:10377000100A91ED002A91ED013AB8EE411A30EEAF
:10378000410A32EE431A21EE000A30EE420A10EEF0
:10379000100A28F015FD9FED720B53EC102B28F04A
:1037A000BFF902460B465046294627F071FE27F026
:1037B0003DFE00EE100A87E600EE104AB8EE400A21
:1037C00020EE091A31EE0A1ABDEEC12AB8EEC22A5D
:1037D00031EE421A21EE0B1ABDEEC12A12EE100A8A
:1037E000B8EB502F31EE0C2A1CBFB0EE421A00206D
:1037F00009EB800102EE100A91ED003A91ED014AC9
:10380000B8EE422A31EE421A34EE432A22EE011A71
:1038100020EE0D2A32EE0A2A31EE031ABDEEC23A2C
:10382000B8EEC33A32EE432A22EE0B2ABDEEC23A7C
:1038300013EE100AB8EB502F32EE0C3A1CBFB0EE6C
:10384000432A002009EB800103EE100A91ED004AA3
:1038500091ED015AB8EE433A20EE0F0A32EE432AB8
:1038600035EE443A30EE0A0A23EE022ABDEEC03AA3
:10387000B8EEC33A30EE430A20EE0B0ABDEEC03A72
:1038800013EE100AB8EB502F30EE0C3A1CBFB0EE1E
:10389000430A002009EB800132EE042A03EE100AED
:1038A00091ED004A91ED015AB8EE433A30EE430AE9
:1038B00035EE443A23EE000A21EE281A30EE040ACF
:1038C00022EE2F2A31EE2A1A31EE021A20EE290AB0
:1038D00031EE000AF8E500EE104AB8EE400A20EE9C
:1038E0002B0A30EE0A0ABDEEC01AB8EEC11A30EE4D
:1038F000410A20EE0B0ABDEEC01A11EE100AB8EB19
:10390000502F30EE0C1A1CBFB0EE410A002009EB1C
:10391000800101EE100A91ED002A91ED013AB8EE16
:10392000411A30EE410A32EE431A21EE000A30EE1F
:10393000420A20EE0E0A30EE0E0AC5E546F6CD50DC
:10394000C1F20000012101704BF25250C2F201009D
:1039500001700CB0BDEC108B01B0BDE8F08F00BF62
:10396000DEE8633E20D0893FF88BF9BE3927B63EAA
:103970008EB1133EB4AB103E2601FABE795D3FBC5A
:1039800014AEB73E2DE9F04F87B049F6C860C1F2DA
:1039900000000178012943D14CF6CC23C2F2010387
:1039A00093F83410012900F0FE81012183F83410CE
:1039B0009A6D93F83510012940F0F281022183F8C5
:1039C00035100021596519689F681E6CDB6D0D6804
:1039D000402F25F480250D6045F6C0554D6041F619
:1039E000000540F20007C2F20005C6F2080702BF58
:1039F0002F460025C6F208058D60CF603F2707FAE5
:103A000003F393600A6842F016020A601EB10A6866
:103A100042F008020A600A6842F001020A60C2E14C
:103A200047F60024C1F2000420464FF47071FDF700
:103A3000A6FE47F2F076C1F20006707806F120018A
:103A4000002808BF311D08680121069020F01EF8EB
:103A500000280146C8BF01390B28B8BF01304AB25F
:103A600091B240B28142009040F3AE8000204FF00E
:103A7000C0422A21C6F208001180002101230180E2
:103A800001800380DF2303802B231380B523018073
:103A90000380B623018003802C231380635A6218AD
:103AA00003805388403103809388B1F5707F038091
:103AB000D38803801389038053890380938903800B
:103AC000D3890380138A0380538A0380938A0380F7
:103AD000D38A0380138B0380538B0380938B0380E3
:103AE000D38B0380138C0380538C0380938C0380CF
:103AF000D38C0380138D0380538D0380938D0380BB
:103B0000D38D0380138E0380538E0380938E0380A6
:103B1000D38E0380138F0380538F0380938F038092
:103B2000D28F0280BAD10021635A62180380538871
:103B3000403103809388B1F5707F0380D388038080
:103B4000138903805389038093890380D389038079
:103B5000138A0380538A0380938A0380D38A038065
:103B6000138B0380538B0380938B0380D38B038051
:103B7000138C0380538C0380938C0380D38C03803D
:103B8000138D0380538D0380938D0380D38D038029
:103B9000138E0380538E0380938E0380D38E038015
:103BA000138F0380538F0380938F0380D28F028003
:103BB000BAD149F6CA60C1F200000021018007B005
:103BC000BDE8F04F00F0F8B84AF20800C2F2010078
:103BD00000689FED772A00F14203029300F144034D
:103BE00000F13E0A059300F140033C30049303903A
:103BF00006989FED703A00EE100A96F88701B8EE2D
:103C0000400A01EE100AB8EE411A06E0019A009847
:103C1000013291B281423FF729AF01EB410042F2FC
:103C20005C21C0F6030101EBC000D0E9043B002099
:103C30000026019204E000BF0136B0B28345E5D909
:103C400000EB400703EB87008268951E062D524665
:103C50000ED8DFE805F0040407070B090900039AF2
:103C600006E000BF059A03E0049A01E0029A00BF53
:103C700053F82770406804EE107AB8EE444A34EEE8
:103C8000404A24EE024A24EE014A34EE034ABDEED5
:103C9000C44A14EE105A04EE100AB8EE444A34EE48
:103CA000404A24EE024A24EE014A34EE034ABDEEB5
:103CB000C44A14EE101AB2F800806A090E2A4FEABC
:103CC000511288BF4FF0FF350E2A88BF4FF0FF31E9
:103CD0004A1C8E4608BF4FF4F07E6A1CA94608BFF6
:103CE0008E461EF1010118BF4FF00009002A18BFCF
:103CF000A94609EA0E0101310ED106998F429BD2E5
:103D000006994FF000094FF0FF3E884298BF4FF0F0
:103D1000FF3988BF4FF4F07E19F1010C18BF1EF176
:103D200001003FF489AFCE457FF786AFAEEB0900C7
:103D30006FEA090110F003020EEB010014D01FFA24
:103D400089F1012A24F811800FD01FFA8CF1022A80
:103D500009F1020C24F8118007D01FFA8CF124F825
:103D6000118009F1030C00E0CC460328FFF464AF96
:103D70001FFA8CF024F810800CF1010080B224F8B6
:103D800010800CF1020080B224F810800CF10300C6
:103D90000CF1040C80B2E64524F81080E8D14BE722
:103DA000002183F834100021017007B0BDE8F08FC6
:103DB0000AD7233C000070432DE9F04F81B02DED70
:103DC000028B84B049F6CA66C1F20006B6F80080DC
:103DD000B8F1000F00F0A480B8F1360F00F2BE80F9
:103DE00047F60860C1F2000090ED000A4AF2880030
:103DF000C1F2000000EB880090ED001A47F2F07964
:103E0000B8EE400AB8EE411AC1F2000930EE410A9C
:103E10009FEDBC1A99F8870120EE010A01EE100A05
:103E2000B8EE411A20EE018A18EE104A204627F01B
:103E3000B9F980F0004000EE100ABDEEC00AB5EE00
:103E4000408A10EE107AF1EE10FA4FF4F076204628
:103E50004FF00005A8BF2F464FF4F07AB7F5F07F7A
:103E6000B8BF3E4627F044F900EE100ABDEEC00A86
:103E700010EE101AB5EE408AF1EE10FAD8BF2946BE
:103E8000B1F5F07FA8BF51467018B0F5F07FC6F5C8
:103E9000F07543F6A02A4DF2362BC8BF00218D42A3
:103EA000C2F2010AC2F2010B6BDD51EA0600CDE954
:103EB000018179D0012FD646C0F2B8814AF20800BC
:103EC000C2F20100006843F6A0270278C2F201079F
:103ED000710038467446FDF7C6FDA646002D00F079
:103EE000A58147F6C2504CF23021C1F20000C2F267
:103EF000010140F2DF12B0F90000B1F90010921B8D
:103F00004DF280344DF2D01805F00303032AC2F2BB
:103F10000004C2F20108009380F0F680002543E11E
:103F20004FF0C0402A2101800021C6F20801002282
:103F30000123DF270A800A800B800F802B27078050
:103F40000A80EB220A8021220B800A802C2101802A
:103F5000B6F80080B8F1360F7FF642AF46F6C4508F
:103F6000C1F200000188013101804BF25150C2F2D0
:103F700001000021017047F2B470C1F2000001702D
:103F8000D3E24AF20800C2F2010000684FF47071F7
:103F9000027843F6A020C2F20100FDF764FD49F665
:103FA000CA68C1F200080FE247F6C2504CF2302155
:103FB000019AC1F20000C2F201014DF28033B0F962
:103FC0000000B1F90010C2EB0212C2F200034DF280
:103FD000D01903EB4212AAF1140C0026C2F2010917
:103FE000D6460392039B4D469A5D8E4288BF5D463E
:103FF000864238BF5D4635F812404D469A192CF876
:10400000144F741C8E4228BF5D46844238BF5D4603
:104010005778947835F817500EEB46077D80B51C1D
:10402000CE4692F8038092F804A08D4288BFDE4607
:10403000854238BFDE463EF814E0F41C4D468C4203
:1040400088BF5D46844238BF5D4635F81840351D4F
:10405000FC804C46A7F804E08D4288BF5C46854250
:1040600038BF5C4634F81AE0741D4B4655798C42D3
:1040700088BF5B46844238BF5B4633F815304D46F7
:10408000ACF80A30B31DACF808E08B4288BF5D463F
:10409000834238BF5D469379D47935F813304D4665
:1040A000BB81F31D92F808E0527A8B4288BF5D46CF
:1040B000834238BF5D4635F8143006F108044D469A
:1040C0008C4288BF5D46844238BF5D4635F81E503D
:1040D000FB813D8206F109034F468B4288BF5F4654
:1040E00043F6A02E834238BF5F4637F812200A36C7
:1040F000C2F2010EB6F5F07FACF812207FF472AF79
:1041000094E000BF0AD7233C25F003020392019AF2
:1041100007EB4609C2EB021504EB4515A9F1020CA9
:1041200005F1010E002500BF06EB050A0EEB0504A4
:10413000424614F8017C8A4588BF5A46824538BFFA
:104140005A4632F817201EF80570ACF802200AF122
:10415000010243468A4288BF5B46824238BF5B46C3
:1041600033F8172009EB45035A800AF102028A420C
:10417000474688BF5F468242627838BF5F4637F85D
:104180001220A4789A800AF1030243468A4288BF2B
:104190005B46824238BF5B4633F81420039B0435EC
:1041A000AB422CF8082FBFD1009F43F6A02E43F658
:1041B000A02CC2F2010EC2F2010CBFB3019A4DF263
:1041C0008034C2EB0212C2F2000404EB4219AB19B4
:1041D00019F8052044468B4288BF5C46834238BFAD
:1041E0005C4634F81220012F2CF813201ED06B1CD3
:1041F0009A1919F8033044468A4288BF5C468242C5
:1042000038BF5C4634F81330022F2CF812300DD032
:10421000AB1C9F1919F803208F4288BFD8468742EC
:1042200038BFD84638F812002CF81700029B49F620
:10423000CA6847F2F079012BC1F20008F246C1F2D8
:104240000009C0F2C1804AF20800C2F20100016810
:10425000C3F5F0740A780AEB44005900FDF703FC3B
:10426000DDF808E0002C00F0AF8047F6C2504CF2B9
:104270003021C1F20000C2F2010140F2DF12B0F9B8
:104280000000B1F90010A2EB0E02032A04F0030CA7
:1042900001D2002357E0019A4DF28033C2EB0212A3
:1042A000C2F20003754603EB42122A444DF2D019C4
:1042B00024F0030E02F10108AAF108050023C2F25E
:1042C000010900BF08EB03074A4617F8014C8B426F
:1042D00088BF5A46834238BF5A4632F8142018F82D
:1042E00003404E4625F8082F5A1C8B4228BF5E46D5
:1042F000824238BF5E4636F814209C1C8C424E46E3
:1043000088BF5E4684427C7838BF5E4636F81440EB
:104310006A80AC80DA1CBC784E468A4288BF5E4612
:10432000824238BF5E4636F8142004339E45EA8048
:10433000C8D149F6CA6847F2F079DDF808E0C1F261
:104340000008C1F20009BCF1000F3DD0019F4DF201
:104350008036C7EB0717C2F200064DF2D01403EB0C
:104360000E0206EB4717C2F20104BE5C22468B42E6
:1043700088BF5A46834238BF5A4632F81620BCF1ED
:10438000010F2AF813201FD05A1C02EB0E06BE5D47
:1043900025468B4228BF5D46824238BF5D4635F8D0
:1043A0001660BCF1020F2AF812600DD09A1C02EBC5
:1043B0000E03FB5C8A4288BF5C46824238BF5C4683
:1043C00034F813002AF8120099F98C01022846DB10
:1043D0004AF2B831C2F201010A68BBF84A00012A68
:1043E000A8BF2AF812004A68002AC8BF2AF812009B
:1043F0008A68012AA8BF2AF81200CA68012AA8BF41
:104400002AF812000A69012AA8BF2AF812004A698C
:10441000012AA8BF2AF812008A69012AA8BF2AF82F
:104420001200CA69012AA8BF2AF812000A6A012AE2
:10443000A8BF2AF812004A6A012AA8BF2AF8120067
:104440008A6A012AA8BF2AF81200CA6A012AA8BFEC
:104450002AF81200096B0129A8BF2AF8110099F85F
:104460008401B0B199F8010009F12401002808BFC6
:1044700009F10801086820F00100022809D147F677
:10448000C051C1F20001BBF83200B1F900102AF8A6
:1044900011004CF62C32C2F2010292F83400BBF843
:1044A00032100128AAF8E0113AD0012082F8340035
:1044B000916D92F8350001282FD1022082F8350045
:1044C0000020506510689368176CD26D0668402B09
:1044D00026F4802606604FF4F0764660534640F29C
:1044E000000604BF0023C6F20803C6F2080608BF90
:1044F000564683603F2303FA02F2C6608A60016871
:1045000041F0160101601FB1016841F0080101602E
:10451000016841F00101016002E0002082F83400EE
:10452000B8F800000130A8F8000004B0BDEC028B20
:1045300001B0BDE8F08F00002DE9F04147F2F074C2
:10454000C1F20004667804F13807394604F11C050D
:10455000002E08BF2946097804F120004FF03802E8
:1045600081F0010108BF1C22A154002E08BF201DAC
:10457000006801214FF001081FF088FA01280BDBC9
:10458000C1B28900002E08BF2F463A7851FA80F058
:1045900004EB800080F84F204BF69470C2F20100CB
:1045A00080F801804BF6CE70C2F2010080F80080E6
:1045B000BDE8F08147F2C171C1F20001087800281E
:1045C0004BF69470C2F2010028D04AF2144241F630
:1045D000BC13C2F20102C0F60403136042F66C126F
:1045E00041F64C23C1F20002C0F6040313604DF201
:1045F000D542C2F201024FF0000C82F800C049F629
:10460000DC62C1F20002127849F6DB63C1F20003FA
:104610001A7081F800C0012101701EE001220A70A9
:104620004AF2144141F2C063C2F20101C0F6040330
:104630000B6042F66C1141F64003C1F20001C0F676
:1046400004030B604DF2D541C2F201010A7049F634
:10465000DB61C1F2000115220A7001210170817134
:104660008172017281700171C172017081718172F8
:10467000017281700171C17242F61C10C1F200001A
:10468000002101604BF6B870C2F20100016042F6F1
:104690002410C1F20000FF2101704AF26A00C2F248
:1046A0000100017042F62510C1F20000017042F6CF
:1046B0002210C1F2000042F20F7101804AF268003C
:1046C000C2F20100018042F62010C1F20000018018
:1046D0007047000070B547F2F074C1F2000494F81E
:1046E0003501617880F0010504F1200084F835512E
:1046F000002908BF201D0068012101261FF0C6F90E
:1047000001280ADBC1B2890051FA80F0D4F83011D7
:1047100004EB800080F84C5081644BF69470C2F238
:10472000010046704BF6CE70C2F20100067070BDFB
:10473000B0B52DED028B47F2F074C1F2000494F88D
:10474000340194ED4C1A00EE100AB8EE400A31EE36
:10475000008AB3EE0F1AB4EE418AF1EE10FAC8BF28
:10476000B0EE408A607804F1200184ED4C8A002884
:1047700008BF211D0868012101251FF087F90128C4
:104780000BDBC1B2890094F8352151FA80F004EBBB
:10479000800080F84C2080ED128A4BF69470C2F2B3
:1047A000010045704BF6CE70C2F201000570BDEC01
:1047B000028BB0BDB0B547F2F070C1F20000417895
:1047C00059B100F1200E9EE80E50D0E90D45071DAD
:1047D00087E80E50C0E906450BE0051D00F1140EF8
:1047E0002ECD9EE8105000F1200730302EC780E813
:1047F000105049F6EC60C1F20000006847F6AC11B9
:10480000C1F20001086047F6B01044F2566144F668
:104810004372C1F20000C2F24F01C4F65012C0E967
:10482000001244F24951C0F24401C0F807104CF2A2
:104830001D00C2F20100002101704BF69470C2F21B
:104840000100817B00291CBF01218171012181733D
:10485000417041714BF6CE70C2F201000170B0BDE3
:10486000F0B581B04CF22920C2F20100012505709B
:1048700040F61800C4F202004FF40001016049F64E
:10488000EC60C1F20000006847F69811C1F2000127
:1048900047F2F0760860C1F20006707806F1200455
:1048A00080F0010171702146371D002818BF39467C
:1048B000086819F0DDFA707806F12401002808BFB5
:1048C00006F10801086808BF3C46214619F0D8FCEB
:1048D0004BF694704BF6CE71C2F20100C2F20101A8
:1048E00045704571C5710D704BF6CC71C2F2010176
:1048F0000D70057085718572057285700571C572C0
:1049000042F61C10C1F20000002101604BF6B870A5
:10491000C2F20100016042F62410C1F20000FF2142
:1049200001704AF26A00C2F20100017042F62510DD
:10493000C1F20000017042F62210C1F2000042F202
:104940000F7101804AF26800C2F20100018042F654
:104950002010C1F20000018001B0F0BD80B547F227
:10496000F070C1F2000090F8412182F0010180F85E
:10497000411116A018A1002A08BF014649F6EC60B3
:10498000C1F20000006847F6AC12C1F200021060EC
:1049900047F6B010C1F20000FBF779FF4CF21D00A2
:1049A000C2F20100002101704BF69470C2F20100C6
:1049B000817B00291CBF012181710121817341701C
:1049C0004BF6CE70C2F20100017080BD42414E44F0
:1049D0004D4150204F4E000042414E444D41502029
:1049E0004F4646002DE9F04147F2F075C1F200054F
:1049F00095F8018005F1200420462E1DB8F1000F26
:104A000008BF3046006801211FF040F8013841B26C
:104A1000002948BF0B20C1B2032901D041BB00BF10
:104A2000013841B2002948BF0B20C1B2002918BF8C
:104A300003291DD1013841B2002948BF0B20C1B262
:104A4000032918BF002913D1013841B2002948BFFA
:104A50000B20C1B2032918BF002909D1013841B286
:104A6000002948BF0B20C1B2002918BF0329D7D0A5
:104A700040B200EB800005EB8007386C2146B8F1AE
:104A8000000F08BF314619F0F3F9697897F8440030
:104A9000002908BF3446214619F0F2FB97F84C0074
:104AA000B96C85F83501C5F8301197F84D0097F8C5
:104AB0004E1085F88E0185F8781197F8500047F66A
:104AC0008C11C1F20001087097F84F006978382204
:104AD000002908BF1C22A85447F69C10C1F2000010
:104AE000002101704BF69470C2F201000121417067
:104AF0004171BDE8F08100002DE9F04147F2F07509
:104B0000C1F2000595F8018005F1200420462E1D14
:104B1000B8F1000F08BF3046006801211EF0B6FF53
:104B2000013041B20B29C8BF0020C1B2032901D016
:104B300041BB00BF013041B20B29C8BF0020C1B248
:104B4000002918BF03291DD1013041B20B29C8BF6C
:104B50000020C1B2032918BF002913D1013041B28E
:104B60000B29C8BF0020C1B2032918BF002909D1F1
:104B7000013041B20B29C8BF0020C1B2002918BFC3
:104B80000329D7D040B200EB800005EB8007386CDA
:104B90002146B8F1000F08BF314619F069F969786C
:104BA00097F84400002908BF3446214619F068FBF5
:104BB00097F84C00B96C85F83501C5F8301197F8B5
:104BC0004D0097F84E1085F88E0185F8781197F80A
:104BD000500047F68C11C1F20001087097F84F00A1
:104BE00069783822002908BF1C22A85447F69C1077
:104BF000C1F20000002101704BF69470C2F2010076
:104C0000012141704171BDE8F081000047F2C1719E
:104C1000C1F20001087800284BF69470C2F201003E
:104C200063D04AF2144241F6BC13C2F20102C0F64C
:104C30000403136042F66C1241F64C23C1F20002E9
:104C4000C0F6040313604DF2D542C2F201024FF0E8
:104C5000000C82F800C049F6DC62C1F20002127852
:104C600049F6DB63C1F200031A7081F800C001212C
:104C7000017042F61C120121C1F2000200230170F2
:104C800081718172017281700171C17213604BF682
:104C9000B872C2F20102136042F62412C1F200029D
:104CA000FF2313704AF26A02C2F20102137042F645
:104CB0002512C1F20002137042F62212C1F2000264
:104CC00042F20F7313804AF26802C2F201021380AB
:104CD00042F62012C1F200021380017081718172CC
:104CE000017281700171C17270474FF0010C81F83F
:104CF00000C047F2F071C1F200014B7801F12402CB
:104D0000002B08BF01F1080211688A1E022A21D374
:104D10000A1F022A3DD24AF2144141F2C062C2F295
:104D20000101C0F604020A6042F66C1141F640022D
:104D3000C1F20001C0F604020A604DF2D541C2F290
:104D4000010101220A7049F6DB61C1F200010C2267
:104D50000A708EE74AF2144141F2C062C2F20101C8
:104D6000C0F604020A6042F66C1141F64002C1F23C
:104D70000001C0F604020A604DF2D541C2F2010101
:104D800081F800C049F6DB61C1F200010A220A7015
:104D90006FE706294AF2144141F2C062C2F20101F2
:104DA000C0F604020A6042F66C1141F64002C1F2FC
:104DB0000001C0F604020A604DF2D541C2F20101C1
:104DC0004FF001020A7049F6DB61C1F2000114BF25
:104DD00008220B220A704CE747F2F070C1F2000083
:104DE00090F8471181F0010180F847114BF694705B
:104DF000C2F20100012141704BF6CE70C2F20100F7
:104E00000170704747F2F070C1F2000090F83C105A
:104E100081F0010180F83C104BF69470C2F2010061
:104E2000012141704BF6CE70C2F201000170704753
:104E300047F2C171C1F20001087800284BF6947066
:104E4000C2F2010028D04AF2144241F6BC13C2F269
:104E50000102C0F60403136042F66C1241F64C23C3
:104E6000C1F20002C0F6040313604DF2D542C2F253
:104E700001024FF0000C82F800C049F6DC62C1F27A
:104E80000002127849F6DB63C1F200031A7081F860
:104E900000C00121017038E04FF0010C81F800C022
:104EA00047F2F071C1F200014B7801F12402002BAE
:104EB00008BF01F1080211684AF2144241F2C063CE
:104EC000C2F20102C0F6040321F00101136042F6B0
:104ED0006C1241F64003C1F20002C0F6040302293D
:104EE000136006D149F6DB61C1F2000109220A70A4
:104EF0000BE04DF2D541C2F2010181F800C049F644
:104F0000DB61C1F2000107220A7042F61C12012186
:104F1000C1F20002002301708171817201728170FF
:104F20000171C17213604BF6B872C2F201021360D4
:104F300042F62412C1F20002FF2313704AF26A0201
:104F4000C2F20102137042F62512C1F20002137080
:104F500042F62212C1F2000242F20F7313804AF2AB
:104F60006802C2F20102138042F62012C1F200026E
:104F70001380017081718172017281700171C1723F
:104F80007047000080B547F2F070C1F2000090F861
:104F9000802182F0010180F8801113A015A1002A60
:104FA00008BF014649F6EC60C1F20000006847F610
:104FB000AC12C1F20002106047F6B010C1F200005E
:104FC000FBF765FC4CF21D00C2F2010000210170EC
:104FD0004BF69470C2F20100817B00291CBF0121B5
:104FE00081710121817380BD4B45594552204F4E3F
:104FF000000000004B45594552204F464600000036
:1050000047F2C170C1F20000007848B947F2F07071
:10501000C1F2000090F8461181F0010180F84611BC
:105020004BF69470C2F201000121417041724BF6BF
:10503000CE70C2F20100017070470000F0B581B07F
:1050400047F2F075C1F20005687805F124010028E7
:1050500008BF05F1080109780A2916D80224DFE8FB
:1050600001F0220C06060808140A0A140E0008248F
:1050700019E0062417E0042415E0032413E04BF69E
:105080009471C2F2010101220A7205F12001002887
:1050900008BF291D096849F27F62C0F29802002406
:1050A000914288BF012405F1200700283946204697
:1050B00005F1040608BF314619F0E2F868780121CD
:1050C000002808BF3746386801261EF0DFFC01289B
:1050D00007DBC1B2890051FA80F005EB800080F84F
:1050E000444047F69C10C1F20000067001B0F0BDCC
:1050F000F0B581B047F2C170C1F20000007800281D
:1051000043D049F6D761C1F20001012008704BF687
:10511000947142F61C12C2F20101C1F20002002396
:10512000087088718872087288700871C87213607C
:105130004BF6B872C2F20102136042F62412C1F2B9
:105140000002FF2313704AF26A02C2F201021370D6
:1051500042F62512C1F20002137042F62212C1F289
:10516000000242F20F7313804AF26802C2F2010297
:10517000138042F62012C1F2000213804870487278
:105180004BF6CE70C2F2010058E047F2F074C1F263
:105190000004617804F12400002908BF04F108002C
:1051A0000568E8B20A2827D80125DFE800F02506BF
:1051B000080A0C0E101214161E0000251CE0032510
:1051C0001AE0022518E0052516E0042514E009255B
:1051D00012E0082510E007250EE04BF69470C2F2AD
:1051E0000100012202720A2506E04BF69470C2F219
:1051F000010001220625027204F12007E8B200290D
:10520000394604F1040608BF314619F039F86078D0
:105210000121002808BF374638681EF037FC0128F6
:10522000A1BFC1B2890051FA80F004EB8000A8BF91
:1052300080F8445047F69C10C1F200000121017033
:1052400001B0F0BD4BF6FC70C2F20100017881F0B4
:10525000010101704BF69470C2F20100012141700E
:105260004BF6CE70C2F2010001707047F0B581B00C
:105270004CF22920C2F201000121017040F6180011
:10528000C4F202004FF40001016049F6EC60C1F283
:105290000000006847F69811C1F2000147F2F0756E
:1052A0000860C1F200056E7805F13400002E08BFD9
:1052B00005F11800016805F12C0008BF05F1100088
:1052C0000068814204D93421002E08BF182168509B
:1052D00005F13000002E08BF05F11400007800270A
:1052E000002846D149F6F814C1F200042046802176
:1052F000FCF745FA49F67820C1F200004FF400713E
:10530000FCF73DFA4DF2C840C2F20100076049F6D1
:10531000D060C1F2000007604DF2BC00C2F2010093
:10532000012101704DF2C000C2F20100046049F693
:105330007844C1F2000420464FF4BE71FCF71FFA16
:1053400049F6EC10C1F20000046049F6F01041F299
:105350006F21C1F20000C3F6032101604DF2C400C9
:10536000C2F20100076049F6F410C1F200000760C4
:1053700001273020002E08BF14202F544BF69470C4
:10538000C2F201000121C17141704BF6CE70C2F230
:105390000100017001B0F0BD70B547F2F074C1F2C8
:1053A000000494F88E01617880F0010504F120007A
:1053B00084F88E51002908BF201D006801210126B4
:1053C0001EF064FB012807DBC1B2890051FA80F0AE
:1053D00004EB800080F84D504BF69470C2F201004F
:1053E00046704BF6CE70C2F20100067070BD000030
:1053F00047F2C171C1F20001087800284BF69470A1
:10540000C2F2010028D04AF2144241F6BC13C2F2A3
:105410000102C0F60403136042F66C1241F64C23FD
:10542000C1F20002C0F6040313604DF2D542C2F28D
:1054300001024FF0000C82F800C049F6DC62C1F2B4
:105440000002127849F6DB63C1F200031A7081F89A
:1054500000C0012101701EE001220A704AF21441CD
:1054600041F60833C2F20101C0F604030B6042F6B4
:105470006C1141F60843C1F20001C0F604030B6051
:105480004DF2D541C2F201010A7049F6DB61C1F269
:10549000000100220A700121017081718172017284
:1054A00081700171C17201708171817201728170AC
:1054B0000171C17242F61C10C1F2000000210160AE
:1054C0004BF6B870C2F20100016042F62410C1F23E
:1054D0000000FF2101704AF26A00C2F2010001706F
:1054E00042F62510C1F20000017042F62210C1F20E
:1054F000000042F20F7101804AF26800C2F201001E
:10550000018042F62010C1F20000018070470000C7
:1055100047F69D10C1F20000017881F00101017091
:1055200000784CF21B01C2F2010108704BF6947036
:10553000C2F201000121C17141704BF6CE70C2F27E
:105540000100017017F032BF47F2C171C1F20001D2
:10555000087800284BF69470C2F2010028D04AF275
:10556000144241F6BC13C2F20102C0F604031360F8
:1055700042F66C1241F64C23C1F20002C0F604035D
:1055800013604DF2D542C2F201024FF0000C82F8D6
:1055900000C049F6DC62C1F20002127849F6DB6312
:1055A000C1F200031A7081F800C0012101701EE0F1
:1055B00001220A704AF2144141F2C063C2F20101B1
:1055C000C0F604030B6042F66C1141F64003C1F2D1
:1055D0000001C0F604030B604DF2D541C2F2010197
:1055E0000A7049F6DB61C1F2000100220A70012154
:1055F000017081718172017281700171C1720170DB
:1056000081718172017281700171C17242F61C1048
:10561000C1F20000002101604BF6B870C2F2010037
:10562000016042F62410C1F20000FF2101704AF22D
:105630006A00C2F20100017042F62510C1F20000BA
:10564000017042F62210C1F2000042F20F71018097
:105650004AF26800C2F20100018042F62010C1F255
:10566000000001807047000047F2C171C1F20001E3
:10567000087800284BF69470C2F2010028D04AF254
:10568000144241F6BC13C2F20102C0F604031360D7
:1056900042F66C1241F64C23C1F20002C0F604033C
:1056A00013604DF2D542C2F201024FF0000C82F8B5
:1056B00000C049F6DC62C1F20002127849F6DB63F1
:1056C000C1F200031A7081F800C0012101701EE0D0
:1056D00001220A704AF2144141F65813C2F2010144
:1056E000C0F604030B6042F66C1141F6B813C1F228
:1056F0000001C0F604030B604DF2D541C2F2010176
:105700000A7049F6DB61C1F2000104220A7001212E
:10571000017081718172017281700171C1720170B9
:1057200081718172017281700171C17242F61C1027
:10573000C1F20000002101604BF6B870C2F2010016
:10574000016042F62410C1F20000FF2101704AF20C
:105750006A00C2F20100017042F62510C1F2000099
:10576000017042F62210C1F2000042F20F71018076
:105770004AF26800C2F20100018042F62010C1F234
:105780000000018070470000B0B547F2F072C1F22E
:10579000000292F8460100B1B0BD47F2C170C1F2FB
:1057A0000000007818B34DF2D740C2F20100007833
:1057B000BDEEC00A012810EE100A69D149F6DA617F
:1057C000C1F200010978012802EB010595F8492191
:1057D00005F2491302EB000185F84911A1F1010519
:1057E00061DBECB21F2C5ED8212119706DE0B7EEA1
:1057F000002ABFEE001AB5EE400AB0EE423AF1EED2
:1058000010FAB8BFB0EE413A9FED4A1AB0EEC04A66
:10581000B4EE414AF1EE10FAC8BFB0EE403A50780B
:1058200092F83C3002F12001002802F59F7508BF74
:10583000111D0868002B08BF02F59E752A8800EE2E
:10584000102AB8EE400AB0FBF2F323EE000ABDEED8
:10585000C00A03FB120310EE105AB0EEC30A2A4628
:10586000002B18BF5A42B4EE420AF1EE10FAC8BF3C
:105870002A46104418F0FCFA4BF69470C2F201006C
:10588000012141714BF6CE70C2F201000170B0BD32
:105890004DF2D641C2F201010978012921D1BDE8BA
:1058A000B0400DF033BCEDB2202D4FF0000538BFF5
:1058B000012500284FF0000048BF012028424FF08A
:1058C00000002ED1CDB27E2D2BD8002A18BF5FEA62
:1058D000016027D04BF69470C2F201000121C17221
:1058E000B0BD4AF2144449F6DB65C2F20104C1F2CC
:1058F000000521682A7801EB02110A790D2A09D0E6
:10590000C96888472068297800EB011000790228CF
:1059100008BFB0BD4BF69470C2F201000121417383
:10592000B0BD18704BF69470C2F2010001210173F2
:10593000B0BD00BF9A99993F2DE9F04F85B047F26D
:10594000E271C1F20001087810B105B0BDE8F08F36
:105950000120087047F2F070C1F2000090F8460193
:10596000002840F0888140F60000C4F20200D0F820
:10597000101842F69000C1F20000037801F0100206
:10598000B3EB121F00F07781C1F30011002A017000
:1059900040F0718147F2C171C1F2000108784BF605
:1059A000947842F61C174BF6B87542F624144AF266
:1059B0006A0642F6251342F6221242F6201BC2F274
:1059C0000108C1F20007C2F20105C1F20004C2F2EF
:1059D0000106C1F20003C1F20002C1F2000BA8B13E
:1059E0004DF2D740C2F201000178012910D1002107
:1059F000017049F6DB60C1F20000017001209146A0
:105A00009A460EF09BF953464A4601E1084610E1DA
:105A10004DF2D640C2F201000178012914D10021D3
:105A2000017049F6DB60C1F2000001700120A2465E
:105A300014461E460EF082F933464AF26A062246A2
:105A40005446C2F20106E3E049F6D960C1F2000013
:105A50000178BA4601293CD1002707704BF6C07087
:105A600047F2F071C2F20100C1F2000100684A7809
:105A700099460B462031002A08BF191D18F0F8F985
:105A80004BF6BC70C2F2010000784BF6FC71C2F21A
:105A90000101087047F69D10C1F2000007704CF23A
:105AA0001B00C2F20100077047F6A610C1F2000009
:105AB000077017F07BFC49F6DB60C1F2000007704D
:105AC00001200EF03BF942F622124B46C1F20002D1
:105AD0006DE049F6D861C1F20001087899460128C5
:105AE0004DF2D540C2F2010039D14AF2144241F6DA
:105AF000BC13C2F20102C0F60403136042F66C123A
:105B000041F64C23C1F20002C0F6040313600022E8
:105B1000027049F6DC60C1F20000007849F6DB63F0
:105B2000C1F20003187047F2C170C1F200000A70A0
:105B30000270012088F8000088F8000088F806004C
:105B400088F80A0088F8080088F8020088F804003D
:105B500088F80B005746CAF800202A6044E0017814
:105B600039B34AF2144141F6BC12C2F20101C0F647
:105B700004020A6042F66C1141F64C22C1F20001A7
:105B8000C0F604020A600021017049F6DC60C1F22F
:105B90000000007849F6DB61C1F2000108700120C5
:105BA0000EF0CCF842F62212C1F200024B465746E4
:105BB0002EE047F2C1710020C1F2000108700121FE
:105BC000574688F8001088F8001088F8061088F802
:105BD0000A1088F8081088F8021088F8041088F86D
:105BE0000B10CAF800002860FF2042F622124AF289
:105BF00068012070307089F8000042F20F70C1F225
:105C00000002C2F201014B4610800880ABF8000090
:105C10004BF6CE70C2F201000121017049F6D76047
:105C2000C1F200000078012805D147F2D070C1F21E
:105C3000000001210170012088F8000088F80600AA
:105C400088F80A0088F8080088F8020088F804003C
:105C500088F80B00002038602860FF204AF26801B5
:105C600020703070187042F20F70C2F20101108083
:105C70000880ABF800004AF2B42449F6EC6BC2F29B
:105C80000104C1F2000B002000254FF0010900269D
:105C900006E000BF28B20135032828B280F20E8149
:105CA00000EBC00714F82700012831D14BF28450D3
:105CB000C2F2010000780028ECD104EB87004078A4
:105CC00040F6000340F018008DF811004FF480708A
:105CD000002600900DF111000DF10E010322C4F217
:105CE0000203ADF812608DF81060ADF80E600196F9
:105CF0000AF0B8FA4FF6FF7650B19DF80F009DF804
:105D0000101000F03F0001F00F0141EA001600BF43
:105D100004EB8707B2B20020B846642A38BF0120DE
:105D200008F8020FC2461AF8011F814206D0632A02
:105D300004D8DBF800307B6000233B7281420DD138
:105D4000632A0BD8DBF800107A68891AB1F5FA7F5C
:105D500003D9394611F8082F42B3014689B180B9F9
:105D6000DBF800007968401A80087C2808D847F2E0
:105D7000F071C1F20001387A91F84611084363D0FE
:105D80000020A9B2033918BF012161EA0901C9073E
:105D90008AF800007FF47EAF4AF2B020C2F2010020
:105DA00004684FF000094FF6FF7573E747F2F07291
:105DB000C1F2000292F84621002A4FF001020A7057
:105DC00006D0F96945F20102C0F600029142C4D141
:105DD00047F2C171C1F20001097811B1797A002945
:105DE000BBD03A6A0146002AB8D047F2F070C1F23F
:105DF000000090F8790108B347F6F8110120C1F2CC
:105E000000010870DBF80000DBF80010091A3329E4
:105E10000ED2DBF80010091A322909D8DBF800107D
:105E2000091A322904D8DBF80010091A3329EBD3F8
:105E300047F6F8110020C1F20001087090479AF867
:105E4000001098F8000089E747F2C170C1F2000025
:105E5000007810B1787A002892D0F86900283FF4D1
:105E60008FAF47F2F071C1F2000191F8791109B3D7
:105E700047F6F8120121C1F200021170DBF80010A0
:105E8000DBF80020521A332A0ED2DBF80020521A17
:105E9000322A09D8DBF80020521A322A04D8DBF85B
:105EA0000020521A332AEBD347F6F8120021C1F230
:105EB00000021170804798F8000062E747F2E27133
:105EC0000020C1F20001087005B0BDE8F08F0000AD
:105ED000F0B590F83C20012A08BFF0BDD1F800C011
:105EE0000122BCF10A0F80F83C200BD31FFA8CFE74
:105EF0004FEA4E02036812FA8CF2A2F11E0403F17B
:105F00000C0205E003680CEB4C0403F11002E646BA
:105F100007251668A54026EA050515608D681668F0
:105F200005FA04F4344314609A6B002622F44012FC
:105F30009A634D680A698C69CFF6F0769F6B06EB21
:105F40000256AA1A3E4303329E63D6B2B60056FAF0
:105F500082F21F269F6B964027EA06069E639E6B81
:105F60000EFA02F232439A639A68012722F47022F1
:105F70009A609A68C0F20F07BC4202D122F4401422
:105F800009E022439A609A6822F440129A60CA6932
:105F90009F6847EA02049C600A7D4F7D5E68002F7F
:105FA00026F4806618BF06F580665E605F68002A8A
:105FB00027F4805718BF07F58057032D5F6008D07E
:105FC000022D09D0012D14BF03F1200203F11402A8
:105FD00004E003F11C0201E003F11802176840F627
:105FE000FF76B7431760CF68166842F20431C4F2F7
:105FF00001013743A1F54176B34217600ED1BCF1E0
:10600000120F03D10A6842F4800206E02CF001026C
:10601000102A03D10A6842F400020A60002180F8C5
:106020003C10F0BD81B00021009190F83C10012996
:1060300055D00122016880F83C208A68D20726D119
:106040008A684DF6836342F001028A604AF2483260
:10605000C2F201021268C4F21B33A2FB03239A0CA2
:1060600002EB42020092009A8AB1009A013A009231
:10607000009A62B1009A013A0092009A3AB1009AED
:10608000013A0092009A12B1009A013AEAE78A684E
:10609000D20724D0026C43F201039A4302F58052E6
:1060A0000264026C0023D2055CBF0022426442F20B
:1060B000000C80F83C306FF00400C4F2010C086062
:1060C000DCF8043388684A68DB0600F4401002F408
:1060D000806306D0614508BF50EA030003D001B0D9
:1060E00070471843FBD1886840F48000886001B095
:1060F0007047000070B581B00022009290F83C20FB
:10610000012A00F08B80D1F800E00122BEF10A0FD5
:1061100080F83C200AD31FFA8EF25200066812FA69
:106120008EF2A2F11E0306F10C0204E006680EEBEB
:106130004E0306F110024FF0070C15680CFA03F439
:10614000A54315608D68146805FA03F323431360B3
:106150004968062905D801EB8101053906F13402A9
:1061600009E00C2901EB810187BF413906F12C02BE
:10617000233906F130021F2314688B4024EA0303FD
:1061800042F2043C1360C4F2010C1FFA8EF314684F
:1061900003FA01F1ACF5417321439E4211603AD1FB
:1061A000BEF1120F06D1DCF8001041F48001CCF8EA
:1061B000001030E02EF0010110292CD1DCF8001085
:1061C000BEF1100F41F40001CCF8001023D14AF2C7
:1061D0004831C2F2010109684DF68362C4F21B32F4
:1061E000A1FB0212910C01EB810149000091009981
:1061F00089B1009901390091009961B10099013983
:106200000091009939B1009901390091009911B1BB
:1062100000990139EAE7002180F83C1001B070BD17
:10622000002808BF704770B586B00446006C00288F
:106230006FD10020CDE90400CDE90200216842F2CF
:106240000012C4F201029142019039D042F20000E2
:10625000C4F20100814258D1002043F63001009081
:10626000C4F202014A6940F6000542F480724A61B4
:106270004A69032602F480720092009A00900A682C
:10628000C4F2020542F004020A600A6802F0040245
:106290000092009A00900A6842F002020A600968BF
:1062A00001F0020100910099CDE90166039001A976
:1062B000284601F031F9CDE90166A5F580601FE0BF
:1062C00043F630010090C4F202014A6942F40072C0
:1062D0004A614A6902F400720092009A00900868CC
:1062E00040F004000860086800F004000090009886
:1062F000302001900320029040F60000C4F202001A
:106300000021039101A901F007F90020606484F8DD
:106310003C00206CC00600F18B80206C41F2021121
:106320008843023042F204312064C4F2010108685B
:1063300020F4403008600A6894E849001A4325694F
:106340000A604168012321F4807141604168C0F610
:10635000007341EA05214160416821F040714160CC
:10636000416831434160816821F400618160E168E6
:10637000826811438160A16A8268994222F070624A
:106380008260826802D122F0405108E011438160AE
:10639000816821F040518160E16A82681143816027
:1063A000816821F0020181608168227E94F82030AA
:1063B00041EA42018160416883B141F4006141607A
:1063C00041684EF2000221F460414160616ACFF6FB
:1063D000FF72436802EB4131194301E021F400618F
:1063E0004160C16A002321F47001C162E269616900
:1063F000CFF6F073C66A03EB02523243C262826880
:1064000022F40072826094F83020836843EA4222CA
:106410008260826822F480628260826842EA81211E
:10642000816000206064206C012161F30100206420
:10643000002084F83C0006B0BDE8704070470000C2
:10644000F0B581B00446002000904AF24830C2F214
:1064500001000268D4E9166048F2B51337680821D4
:10646000C1F64E3381403942A2FB03250CD022688D
:1064700013685B0708D5136823F004031360B16049
:10648000616D41F00101616501218140394208D00F
:1064900022685269120604D5B160616D41F00201B3
:1064A000616504218140394208D022681268920750
:1064B00004D5B160616D41F0040161651021814036
:1064C000394215D020680268120711D5B160026800
:1064D0000168520306D4C90506D4016821F00801F9
:1064E000016001E0080342D4216C09B120468847CD
:1064F000E16D202000FA01F23A4244D0206803689E
:10650000DB0640D5B26094F835300268052B1ED109
:1065100022F016020260426922F080024261226C7F
:106520000AB9A26C1AB1026822F0080202603F2088
:106530008840B060002084F83400012084F83500E1
:10654000216D002957D02046884701B0F0BD016871
:10655000520310D4C90512D4016821F01001016062
:10656000002084F83400012084F8350007E0A16C95
:106570000029BBD1BCE7080301D4616C00E0E16BEA
:1065800009B120468847606DA8B3606DC0072ED062
:10659000052084F835002068A90A026822F001026B
:1065A0000260009A01328A4200921AD80268D20729
:1065B00017D0009A01328A42009212D80268D2079C
:1065C0000FD0009A01328A4200920AD80268D2079C
:1065D00007D0009A01328A42009202D80268D2079C
:1065E000DFD1002084F83400012084F83500E16C0C
:1065F00009B12046884701B0F0BD00002DE9F04107
:1066000049F6EC61C1F200010B68002861D000225C
:1066100080F83420022280F835200268156825F0C1
:10662000010515601568ED0736D1116848F23F0382
:10663000CFF21003D0E901540B4000F10C0E9EE89C
:10664000C2512B43234319433143394341EA0801E3
:10665000436A41EA0C01042B41EA0E043CD1D0E923
:106660000A5E016B4EEA0403194311605169BEF1E1
:10667000000F21F0030141EA050141F0040C31D083
:10668000B8F5005F53D0B8F1000F5FD1022D60D094
:10669000012D55D035BB5CE00D68ED1A052D42D8B3
:1066A0001568ED07C1D00F68FF1A052F3BD8176892
:1066B000FF07BAD00F68FF1A052F34D81768FF07F5
:1066C000B3D00F68FF1A052F2DD81768FF07E3D145
:1066D000ABE70120BDE8F0811460516921F00701AA
:1066E00041EA030C6FF00F014AF6AB2351FA82F135
:1066F000CAF6AA23A1FB03373B091CA7FB5C40F2A7
:10670000FF375F294FF03F01C2F814C022EA0702A9
:1067100001FA03F188BF0432C0E916239160002416
:10672000012300211CE003232024032118E0032D72
:10673000D8D8012340240121DFE805F0120B120212
:10674000AEF1C071B1FA81F1490904E0032D04D31F
:10675000C8D1CEF300610029C4D001234024012117
:10676000446580F835300846BDE8F0810006101613
:10677000000610162DE9F04349F6EC68C1F2000856
:10678000D8F8001090F83510022920D1D0F80090E8
:10679000D9F80010C90521D4D0E9161C20230F68B0
:1067A00003FA0CF31F421ED0426D002A1CBF426D3B
:1067B0005FEAC2723ED1302202FA0CF28A600021F6
:1067C00080F83410012180F83510BDE8F083802175
:1067D0004165002180F83410BDE8F0834FF48071EA
:1067E0004165BDE8F083082707FA0CF4012707FA92
:1067F0000CF5042707FA0CF602E000BF1F42D3D1C4
:10680000476DFF07D0D10F683C4204D0426D42F083
:10681000010242658C603D4204D0426D42F00202AA
:1068200042658D603E42E9D0426D42F0040242650D
:106830008E60E3E7D8F800E090F83520022A4AD1CC
:10684000D9F8002022F01602C9F80020D9F8142047
:1068500022F08002C9F81420026C0AB9826C2AB1B5
:10686000D9F8002022F00802C9F80020D9F8002049
:1068700022F00102C9F80020D9F80020D20730D058
:10688000D8F80020A2EB0E02052A1DD8D9F8002066
:10689000D20726D0D8F80020A2EB0E02052A13D882
:1068A000D9F80020D2071CD0D8F80020A2EB0E02A5
:1068B000052A09D8D9F80020D20712D0D8F800202C
:1068C000A2EB0E02052AD7D920224265002280F8C9
:1068D000342003220DE080224265002280F834201B
:1068E00069E73F2202FA0CF28A60002280F8342025
:1068F000012280F835205EE72DE9F04F81B043F6A4
:106900001441C4F201010A68024200F0D282086018
:106910004AF22851C2F201010A78012A19D1002253
:106920000A7041F204014AF22453CEF20001C2F28D
:10693000010342F670270A681B68C1F200073E682F
:10694000D21A32443A60096842F67422C1F2000257
:106950001160411E072910D80FF20400DFE811F082
:1069600008000800A9023901A902A902A9028D01A3
:1069700001B0BDE8F04F17F0DDB9802800F09C8130
:10698000B0F5806F40F0958247F6F910C1F2000033
:106990000078002846F60560C1F2000040F07482DD
:1069A0000178002940F0708247F2F075C1F20005CD
:1069B000697805F124070029394605F1080308BF65
:1069C000194609680A2900F05F824CF21B04C2F2E2
:1069D00001042178002940F20101C0F2FF0113D126
:1069E00047F6A612C1F2000212786AB947F69D1264
:1069F000C1F2000212783AB94BF6F872C2F2010203
:106A00001268002A00F0B1848E1C40F2180B45F287
:106A1000555240F61801C4F2020BCAF6A922C4F27C
:106A200002014BF8182C082200BF00BF00BFCBF8B2
:106A300000600A6004264FF440220E600A6000BF26
:106A400000BF00BF2278D2B947F6A612C1F20002F9
:106A50001278A2B947F69D12C1F20002127872B9FB
:106A60006A78002A08BF1F463A680A2A07D04BF600
:106A7000F872C2F201021268002A00F079844BF227
:106A8000705CC2F2010CDCF8002044F66027C2F210
:106A9000010707EB820797ED000A9FEDDC1ABEEEB7
:106AA000003A20EE010AB5EE400AB0EE434AB6EED7
:106AB000002AF1EE10FAC8BFB0EE424A34EE000AE6
:106AC000BDEEC00A10EE107A07F30F0545F260071D
:106AD000C2F2010707EB820292ED000A4FF47F43F6
:106AE00020EE010AB5EE400AF1EE10FAC8BFB0EE92
:106AF000423A33EE000ABDEEC00A10EE102A02F34D
:106B00000F044BF27852C2F2010217680137176086
:106B10004CF21002C2F2010212782F46002A08BF7E
:106B2000274608BF2C46A5B2BAB22D0A05F57F0547
:106B3000120ACBF800504FF4802563F31F2402F5AE
:106B40007F0263F31F270E6000BF00BF00BF0D6010
:106B500000BF00BF00BFCBF800400E6000BF00BF09
:106B600000BF0D6000BF00BF00BFCBF800200E606B
:106B700000BF00BF00BF0D6000BF00BF00BFCBF86B
:106B800000700E6000BF00BF00BF0D6000BF00BFFF
:106B900000BFDCF800104A1CBF29CCF8002000F030
:106BA000238140F27F12914240F06E814BF6D47106
:106BB000C2F201010A78002A00F0548146F6EC5135
:106BC000C1F2000101220A7040F27F11CCF80010DE
:106BD0005AE14BF6F470C2F201000078002800F090
:106BE000688147F2F070C1F20000417800F12402A0
:106BF000002908BF00F1080210680B2800F0598135
:106C000047F69D10C1F200000078002840F0518145
:106C10001820C4F202004CF21B01D0F8F823C2F293
:106C200001010B78012020EA920247F6A6164BF6E6
:106C300094744BF274559342C1F20006C2F20104FF
:106C4000C2F2010506D00A7000213170207228704E
:106C500016F0ACFB4CF21A00C2F201003178027857
:106C6000914200F026813178017001202072287055
:106C700001B0BDE8F04F16F099BB4BF6F470C2F2CC
:106C800001000078002800F0148140F61800C4F2DA
:106C90000200D0F8F817D0F8F82746F60660C1F2DF
:106CA00000000378C2F3C004012B10D14BF28050D6
:106CB000C2F20100027812E049F6EC60C1F2000075
:106CC00000684DF29C21C2F201010860F1E04BF234
:106CD0008052C2F20102147001220270224649F66B
:106CE000EC6542F6F458C1F20005C1F2000842F624
:106CF0002C202B68D8F80070C1F20000C678DB1B8E
:106D0000B342C0F0D680A24200F0D3801CB1827999
:106D1000002A40F09C804AF27057C2F20107C1F38A
:106D200040123968A2422FD1427901319142396033
:106D3000C0F28D804BF28251C2F201010A8846F600
:106D4000086C531C0B80C1F2000C2E68DCF800208C
:106D5000B21A322A60D91BB200EE103A9FED2C1AFB
:106D60002A68B8EEC00A20EE010A9FED2A1ACCF874
:106D700000204BF27C5230EE011AC2F2010282ED89
:106D8000001A00220A804DE04279013952429142B4
:106D900039605CDC4BF28251C2F201010A8846F68E
:106DA000086C531C0B80C1F2000C2E68DCF800202C
:106DB000B21A322A3AD91BB200EE103A9FED141AD9
:106DC0002A68B8EEC00A20EE010A9FED121ACCF82C
:106DD00000204BF27C5230EE010AC2F2010282ED39
:106DE000000A00220A8027E04BF6D471C2F20101AA
:106DF0000A78002A41D046F6EC51C1F20001012286
:106E00000A70BF21CCF800103EE000BF0000004730
:106E1000CDCCCC3D6766663F4BF27C51C2F201019E
:106E200091ED001A4078B1EE410A08E04BF27C5136
:106E3000C2F2010191ED000A4078B1EE401A00283B
:106E400008BFB0EE410AFEF79FFC002038602868BA
:106E5000C8F800004BF28050C2F20100047001B08B
:106E6000BDE8F08F4BF26C530022C2F20103CCF864
:106E700000201A7001220A7006E04BF26C52C2F236
:106E80000102012313700B704BF2745EC2F2010E0B
:106E90009EF8001059B946F60461C1F20001097864
:106EA00029B94AF23001C2F20101097809B100782A
:106EB00010B101B0BDE8F08F9EF8002040F2010C47
:106EC000C0F2FF0C45F255531821002A6246CAF65B
:106ED000A92340F61800C4F2020108BF0132C4F22F
:106EE000020041F8183C00BF00BF00BF0A60082242
:106EF0000260042202604FF44022026000BF00BF23
:106F000000BF9EF80020002A00F0E78047F2F074EE
:106F10004CF21B03C1F20004C2F20103627894ED4B
:106F20004C0A1B78E3B947F6A613C1F200031B789D
:106F3000B3B947F69D13C1F200031B7883B904F17E
:106F40002403002A08BF04F108031A680A2A07D09C
:106F50004BF6F872C2F201021268002A00F00382B6
:106F6000002294F88E3194F83551002B18BF02326C
:106F700045B1BDEEC00A10EE103A63F3C602DD065D
:106F800048BF803202F57F024CF214060A600423E7
:106F90004FF48022C2F20106036000BF00BF00BFB1
:106FA000026000BF00BF00BF77884FF47F4565F3E4
:106FB0001F270F60036000BF00BF00BF026000BF5B
:106FC00000BF00BF37683F0A65F31F270F600360EB
:106FD00000BF00BF00BF026000BF00BF00BF366837
:106FE00065F31F260E6042F62C26C1F200060360F0
:106FF00000BF00BF00BF026000BF00BF00BFF77945
:1070000007F57F070F60036000BF00BF00BF02608D
:1070100000BF00BF00BF377A07F57F070F6003602E
:1070200000BF00BF00BF026000BF00BF00BF777A93
:1070300007F57F070F60036000BF00BF00BF02605D
:1070400000BF00BF00BFB67A06F57F060E6047F6A8
:10705000A016C1F20006036000BF00BF00BF0260BF
:1070600000BF00BF00BF778865F31F270F60036074
:1070700000BF00BF00BF026000BF00BF00BF376895
:107080003F0A65F31F270F60036000BF00BF00BF0A
:10709000026000BF00BF00BF366865F31F260E60A8
:1070A000036000BF00BF00BF026000BF00BF00BFA1
:1070B000657804F12006002D08BF261D34684BF6C4
:1070C000A136A4F5B715A5F55875C0F20D06B54261
:1070D00080F0B0800CF1070436E146F60462C1F29C
:1070E00000021778002F00F0C0800023CAF6A92301
:1070F000042741F8183C00BF00BF00BF076000BF75
:1071000000BF00BF51F8083C47F6861503F00106A2
:10711000C1F200052E704BF6EE76C3F34003C2F2C7
:10712000010633704FF48023036000BF00BF00BF2F
:10713000076000BF00BF00BF51F8086C036000BFCC
:1071400000BF00BF076000BF00BF00BF51F8085C70
:10715000EDB245EA062647F68415C1F200052E80F9
:107160002E882C8806F400666FF3DF3444EA061696
:107170002E802E882C8806F4006624F4804444EA8D
:10718000C6062E802E882C8806F4006624F400544F
:1071900044EA86062E802E882C8806F4006624F4A5
:1071A000805444EA46062E80036000BF00BF00BF43
:1071B000076000BF00BF00BF51F8086C036000BF4C
:1071C00000BF00BF076000BF00BF00BF51F8081C30
:1071D0004BF6EC77C9B241EA0621C2F201073980C9
:1071E00039883E8801F400616FF3DF3646EA011109
:1071F000398039883E8801F4006126F4804646EAE9
:10720000C101398039883E8801F4006126F40056B6
:1072100046EA8101398039883E8801F4006126F40C
:10722000805646EA41013980036000BF00BF00BFBD
:10723000002068E0A4F5101540F62136A5F51F459D
:10724000C0F22006B54202D20CF118047CE045F2EF
:10725000E055CFF6BB754CF2C1662544C0F22D0651
:10726000B54220D20CF129046EE04AF23007C2F296
:1072700001073A78002A3FF41CAE4BF27552C2F275
:107280000102167856B30CF105030B60082101606A
:10729000042101604FF440210160002000BF00BFC5
:1072A00000BF38702CE048F62075CFF68D754AF691
:1072B00021262544C0F24406B54202D20CF13A041C
:1072C00042E0A4F537054BF68116A5F5D855C0F276
:1072D0002A06B5421BD20CF1430435E041F8183CB4
:1072E0000CF1040300BF00BF00BF0B600821016068
:1072F000042101604FF44021016000BF00BF00BFC6
:10730000107880F00100107001B0BDE8F08F42F6F7
:107310008035CFF61E754DF601562544C0F26D0638
:10732000B54202D20CF154040EE044F68065CFF66B
:10733000B06549F2816625440CF17604C0F29806E6
:10734000B54238BF0CF165040C60036000BF00BF9C
:1073500000BF0260002000BF00BF00BF8EF8000029
:1073600001B0BDE8F08F0122FBE5CE1CFFF74DBB5D
:107370004BF25052C2F20102127844F644634AF2D0
:10738000D056C1F20003C2F20106002A08BF1E4611
:107390004BF27853C2F201031F684FF4802E07F1BD
:1073A00001071F6040F20003CAF6A9234BF8183CFE
:1073B0004FF0040345F2446245F6446500BF00BF48
:1073C00000BF0B6000BF00BF00BF5BF8084CC1F8F6
:1073D00000E000BF00BF00BF0B6000BF00BF00BFE8
:1073E0005BF8087CC1F20002C1F2000508BF154637
:1073F000FAB242EA042247F6941912B2C1F2000925
:1074000000EE102A99F8002046F6C858C1F200088C
:10741000D8F80070002A32469FED3E1A08BF2A466F
:10742000B8EEC00A02EB870246F6E85720EE010AE2
:1074300044F2604CC1F20007C2F2010C82ED000A76
:107440003A6843F66064E246C2F2010408BFA2460D
:107450000AEB820282ED000AC1F800E000BF00BF23
:1074600000BF0B6000BF00BF00BF5BF8082CC1F875
:1074700000E000BF00BF00BF0B6000BF00BF00BF47
:107480005BF8083CDBB243EA022212B200EE102A9B
:1074900099F80020D8F80030B8EEC00A002A04BFDE
:1074A0003546644605EB83023B6820EE010A82ED17
:1074B000000A04EB830282ED000AC1F800E000BF7D
:1074C00000BF00BF3A680132B2F5C07318BF13465F
:1074D000D8F800203B600132B2F5007FC8F80020E8
:1074E00010D34BF250560022C2F20106C8F8002019
:1074F00046F6CC523778C1F200020123137087F0B0
:1075000001023270C1F800E000BF00BF00BFFFF70A
:10751000BBBC00BF000000382DE9F04F82B000F185
:107520003E4241F6004502F1FF77C4F2020508220F
:1075300043F6004E4FEAB726A84208BF0722C4F21E
:10754000010E072E38BF4FEAB7224FF0010A00267E
:1075500000274FF00008009209E000BF08F1010881
:107560000437B8F1100F06F1020600F0AA800C688B
:107570000AFA08F914EA090FF0D0D1F804C0BCF1F6
:10758000120F00F296800AFA0CF414F0061F00F0B5
:10759000908084680322CD68B2409443B5402C4368
:1075A000846044686FEA020A24EA09024FEA1C1464
:1075B00004FA08F42243B3464260C2688C6802EAC7
:1075C0000A0204FA0BF422434CF01004122CC2609D
:1075D00012D16FF0030202EA58020244D2F820C02E
:1075E00007F01C040F230D69A3402CEA0303A540F8
:1075F0002B431362D1F804C002680CF0030302EAC3
:107600000A0203FA0BF31A435FEACC034FF0010AB4
:107610000260A3D5002243F644030192C4F20203A0
:107620001A684FF6084C42F480421A601A68CFF686
:10763000FF7C02F480420192019A28F00302724416
:1076400052F80C3007F00C050F24AC40A343009C0B
:1076500004FA05F52B4342F80C30DEF800204B68A5
:1076600042EA0905DC0358BF22EA0905CEF80050BA
:10767000DEF804209C0342EA090558BF22EA090506
:10768000CEF80450DEF80820DC0242EA090543F691
:107690000C4458BF22EA0905CEF80850C4F2010490
:1076A00022689B0242EA090558BF22EA09052560C3
:1076B00054E7032202FA06F44FEA480B6FEA040A81
:1076C0007BE702B0BDE8F08FF0B585B0D0F800E000
:1076D00044F20C03DEF8081043F20C4CC4F2000331
:1076E000C4F2000C04910CF57D711A468E4504BF5E
:1076F00043F20C42C4F2000252F8044C0394DEF848
:107700000440029452F8084C0194446844F4007414
:10771000B4F5007F7DD1049CA40744BF029C5FEABE
:10772000046400F1E280039CE40750D0019C6406ED
:107730004DD58E4508BF63461968C36A23F8021BFE
:10774000C362418E01394186418E00293FD152F8F2
:10775000081C21F0600142F8081C418DB9BB43F6BA
:107760000043C4F2000301219E4580F841102ED150
:1077700047F2D171C1F200010B782BB147F6F91332
:10778000C1F2000301271F704CF22823C2F201034B
:1077900000271F7001230B7047F2F071C1F2000146
:1077A0004F7801F12406002F08BF01F10806316867
:1077B0000A2902BF4BF6D471C2F201010B7047F6E1
:1077C000FC11C1F200010B6803F5C0730B60039953
:1077D000490644BF01995FEA816100F1D7800499AD
:1077E000090744BF02995FEA81617CD5DEF8041085
:1077F00021F0A001CEF8041052F8081C21F060011D
:1078000042F8081C00210091DEF808100091009950
:107810004CE1039CA40744BF019C5FEA046400F1AF
:10782000D2800499C9074ED0029949064BD5DEF89B
:107830000C10C36A23F8021BC362418E01394186D2
:10784000418E00293FD1DEF8041021F06001CEF80E
:107850000410418DB9BB43F60043C4F2000301217B
:107860009E4580F841102ED147F2D171C1F200013E
:107870000B782BB147F6F913C1F2000301271F70F3
:107880004CF22823C2F2010300271F7001230B7062
:1078900047F2F071C1F200014F7801F12406002F88
:1078A00008BF01F1080631680A2902BF4BF6D471FE
:1078B000C2F201010B7047F6FC11C1F200010B6826
:1078C00003F5C0730B600499490644BF02995FEA4F
:1078D000816100F1CB800399090744BF01995FEAF8
:1078E000816100F1D78005B0F0BD446A34F8025BD5
:1078F0004462CEF80C50448D013C4485448D002CEC
:107900007FF411AFDEF8044024F0A004CEF8044068
:10791000448E002C7FF407AF43F60045C4F2000507
:107920000124AE4580F841407FF4FDAE47F2D174AA
:10793000C1F2000425782DB147F6F915C1F2000512
:1079400001262E704CF22825C2F2010500262E7069
:107950000125257047F2F074C1F20004667804F145
:107960002407002E08BF04F108073C680A2C02BF58
:107970004BF6D474C2F20104257047F6FC14C1F230
:107980000004256805F5C0752560CCE652F8081C92
:1079900021F0600142F8081CDEF8041021F0A0017B
:1079A000CEF8041000210091DEF80C100091DEF8F2
:1079B000081000910099012180F84110416C41F0BC
:1079C000020141640BE7446A8E4534F8025B44626D
:1079D00008BF63461D60418D01394185418D0029F5
:1079E0007FF41FAF52F8081C21F0A00142F8081CD8
:1079F000418E00297FF415AF43F60043C4F2000323
:107A000001219E4580F841107FF40BAF47F2D17100
:107A1000C1F200010B782BB147F6F913C1F2000354
:107A200001271F704CF22823C2F2010300271F70A8
:107A300001230B7047F2F071C1F200014F7801F1A0
:107A40002406002F08BF01F1080631680A2902BF89
:107A50004BF6D471C2F201010B7047F6FC11C1F272
:107A600000010B6803F5C0730B60DAE6DEF8041062
:107A700021F06001CEF8041052F8081C21F0A0019A
:107A800042F8081C012180F84110416C41F00201CC
:107A9000416420E752F8081C21F0A00142F8081CBC
:107AA000DEF8041021F06001CEF80410012180F806
:107AB0004110416C41F00401416405B0F0BD00008B
:107AC0002DE9F04F87B0002740F60005CDE9057796
:107AD000CDE903770446C4F202050068A5F5E63156
:107AE0008842029702D007B0BDE8F08F40F25C10E8
:107AF000C4F247204FF00109C0F8009043F630006F
:107B00000197C4F20200016902AE41F40041016133
:107B100001694FF0020B01F40041019101990197B5
:107B200001684FF0030841F00101016001684FF066
:107B3000060A01F00101019101990197016841F0E4
:107B4000040101600068314600F0040001900198D2
:107B50004FF400400290A5F50060CDE903B9CDF8DF
:107B60001480CDF818A0FFF7D7FC4FF4A050CDE952
:107B7000020B28463146CDE90498CDF818A0FFF74E
:107B8000CBFC4FF4006A0520CDE902ABCDE90498A7
:107B9000069028463146FFF7BFFC46F21000C4F2BB
:107BA000020049F624057830C1F200054021C5E9FC
:107BB000000705F108004FF480694FF400524FF4BC
:107BC000807380E882064FF4403B04262846C5E9CE
:107BD0000623C5E908B6C5E90A872F63FEF70EFD3F
:107BE000A563AC634CF6AC1546F21001C2F2010578
:107BF0004FF0C060C4F20201C5E900104FF400501C
:107C0000C5E90277C5E9049AA8614FF48070C5E917
:107C1000070B2846C5E90968C5E90B77FEF7EEFCB6
:107C20004EF60C50E563AC63CEF2000000684EF2F5
:107C30003340CEF2000007704EF20410CEF2000086
:107C40004FF40021016007B0BDE8F08F10B5014688
:107C50004CF6D430C2F20100D0F8044469B1D4F833
:107C600004038269002A08BF10BD94F8EC020328BF
:107C70002CD12046BDE810401047D4F8E422032A56
:107C800024D1D4E962239A4221D9C1EBC10100EB8E
:107C90008100D11AD0F80802C4F88811994238BF7F
:107CA0000B46D4F820239BB2C2F81032136900248B
:107CB000C2F80802C2F81442012BA2F8FC4108BF26
:107CC000C2F80C02106802F5FE711DE010BDD4F878
:107CD0000403016929B194F8EC02032801D120467C
:107CE00088470420C4F8E402D4F820034FF48072DB
:107CF0000146036921F83C2F002282640265012BB2
:107D0000426508BFC2640068DAB2BDE8104018F0EE
:107D100041B8000010B54CF6DC7CC2F2010C9CF8B6
:107D20001D1011B1DCF8001011E042F60002DCF881
:107D30000010C4F20002002391428CF81C3006D1DE
:107D400040F63C61C4F2472101230B601146022238
:107D50008CF81D20CA224A6253224A62CA6852061F
:107D600029D44FF0FF32CA6049F6EC62C1F200023A
:107D70001368C86840061ED41068C01AB0F57A7F30
:107D800071D8C868400616D41068C01AB0F57A7F5A
:107D90006BD8C86840060ED41068C01AB0F57A7F58
:107DA00065D8C868400606D41068C01AB0F57A7F56
:107DB000DFD9042252E088684FF6BF72CFF68F7287
:107DC00010408860DCE9010EDCE90332DCF8144085
:107DD00010438A682043104388600B61086940EAB9
:107DE0000E400861C86820F08000C860886880067E
:107DF0002AD4C86849F6EC6220F0A000C860C1F23D
:107E000000021368C86880061ED41068C01AB0F556
:107E10007A7F2ED8C868800616D41068C01AB0F5CC
:107E20007A7F28D8C86880060ED41068C01AB0F5CA
:107E30007A7F22D8C868800606D41068C01AB0F5C8
:107E40007A7FDFD9042209E0086C20F480200864DE
:107E5000DCF818000A6C104301220864FF20486215
:107E60008CF81D2010BD0422F8E70422F6E7042256
:107E7000F4E70422F2E70422F0E70422EEE7000030
:107E8000F0B582B049F68403C1F2000393F8506064
:107E9000012E02D14FF0020CC3E0012649F6EC6E30
:107EA00083F85060C1F2000EDEF8004093F85150A4
:107EB000012D66D100284FF0010C18BF002900F0F9
:107EC000AA80002A00F0A78093F85160042E1CBFFE
:107ED000052683F8516000265E659963DA879A87E4
:107EE0001863DA861D689A861E645E642E687606BC
:107EF00003D42E6846F040062E60D3F804C0013A41
:107F0000DE68BCFA8CF7B2FA82F27F095209B6F544
:107F1000006F42EA070244D132B130F8022BEA6026
:107F20001863DA8E013ADA861A68012506E000BF86
:107F3000DEF80060361BB6F5007F6AD2DE8E16B919
:107F4000DE8F002E72D09668B6070BD5DE8E012D1F
:107F500008D13EB130F8025BD5601863DD8E013D7B
:107F6000DD8600259668F607E2D0DE8F002EDFD092
:107F7000D56821F8025B9963DD8F013DDD8701251E
:107F8000D6E75E68B6F5827F08D1042D4FF0020C6B
:107F900041D19D68002D3FF48DAF3CE04FF0020CC5
:107FA00039E03AB100782873186B01301863D88E25
:107FB0000138D886012005E0DEF80010091BB1F574
:107FC000007F26D2D98E09B9D98F69B319688A681A
:107FD00092070DD5DA8E01280AD14AB1186B0078C4
:107FE0000873186B01301863D88E0138D8860020CA
:107FF0008A68D207E0D0DA8F002ADDD0C868996B92
:108000000870986B01309863D88F0138D8870120A9
:10801000D2E74FF0030C012083F85100002083F8D1
:108020005000604602B0F0BDD3F804C04AF24830B8
:10803000C2F20100006849F68171C1F25E61A0FBE5
:108040000101480D4FF47A71484301901868BCF55E
:10805000827F0FD18168090631D499684FF0000CF6
:108060000029D8D1CDF800C0C16800918068009087
:108070000098D0E701990029EFD0019901390191C9
:1080800081680906E9D501990029E6D001990139ED
:10809000019181680906E0D501990029DDD0019997
:1080A0000139019181680906D7D501990029D4D0F9
:1080B00001990139019181680906DBD4CDE70021DE
:1080C000DEF80020121BB2F5007F1ED28268120675
:1080D000C3D5DEF80020121BB1EB522F15D18268F8
:1080E0001206BAD5DEF80020121BB1EB522F0CD1CC
:1080F00082681206B1D5DEF80020121BB1EB522FB8
:1081000003D182681206DBD4A7E7416821F0E001C1
:1081100041609968B1F5004F02D0B1F5806F03D18D
:10812000016821F040010160996AB1F5005F07D153
:10813000016821F400510160016841F400510160BF
:108140004FF0010C002083F851C083F85000586DA7
:1081500040F020005865202058655CE72DE9F04785
:1081600086B049F6DC07C1F2000797F849100446CB
:1081700000293FD14BF28850C2F20100017800255E
:1081800087F848500595CDE903550295019589BBBF
:108190000121017043F638000095C4F20200016825
:1081A00040F6004841F0010101600068C4F2020895
:1081B00000F00100009000984FF6807001AE019031
:1081C0004FF002094FF00C0A08F580603146CDE906
:1081D00002950495CDF814A0FFF79EF94EF2B37006
:1081E000CDE9010940463146CDE90355CDF814A04B
:1081F000FFF792F93868D7E9021907F1100E9EE8E7
:108200004854D7F8248050F821208025CFF6F07507
:108210002A4042EA09021A43324342EA0A0242EA87
:108220000C0242EA0E02BE6A42EA0802FD6A3243CA
:108230003E6B2A437D6B32437E6C2A43BD6B3243D7
:108240002A43082B08BF42F0400240F82120B968B9
:10825000002500EB81014A6826692368CFF6F07596
:1082600002F0404205EB065665681A43A36842EAED
:108270000512E56842EA032242EA05423243D4E9A4
:1082800005631A4306F1FE0342EA03624A603A6B51
:108290007968B2F5804FBA6806BF51F822304FF0C6
:1082A000FF336FF0704341F82230B96850F8212055
:1082B00042F0010240F8212006B0BDE8F08700003E
:1082C000002808BF704710B581B090F83D1040F20B
:1082D000004C0029C4F2010C40F04981016840F6CD
:1082E000FF73C4F200030022994280F83C2040DC76
:1082F00040F20042C4F20002914277D040F6000200
:10830000C4F20002914200F0CB8040F60042C4F279
:108310000002914240F02B81002143F6400200917F
:10832000C4F20202136843F008031360126802F0FB
:1083300008020092009A4EF60C52CEF20002126829
:10834000C2F3022282F00703042B28BF0423033A5E
:1083500038BF0A464FF0FF319940052323EA010157
:1083600091404EF21D420901CEF2000251753221B8
:10837000EFE041F20002C4F20002914263D041F208
:108380000042C4F20002914200F0B780614540F023
:10839000EE80002143F640020091C4F202025368CD
:1083A00043F002035360526802F002020092009A06
:1083B0004EF60C52CEF200021268C2F3022282F094
:1083C0000703042B28BF0423033A38BF0A464FF0A3
:1083D000FF3199400A2323EA010191404EF21D42E8
:1083E0000901CEF20002D1732C21B2E0002143F644
:1083F00040020091C4F20202136843F002031360CA
:10840000126802F002020092009A4EF60C52CEF26E
:1084100000021268C2F3022282F00703042B28BF75
:108420000423033A38BF0A464FF0FF319940022334
:1084300023EA010191404EF21D420901CEF20002F1
:1084400011701D2185E0002143F640020091C4F225
:108450000202136843F010031360126802F0100266
:108460000092009A4EF60C52CEF200021268C2F34D
:10847000022282F00703042B28BF0423033A38BFEB
:108480000A464FF0FF319940082323EA0101914049
:108490004EF21D420901CEF200025176362158E01B
:1084A000002143F640020091C4F20202136843F037
:1084B00004031360126802F004020092009A4EF660
:1084C0000C52CEF200021268C2F3022282F00703BD
:1084D000042B28BF0423033A38BF0A464FF0FF316C
:1084E0009940092323EA010191404EF21D420901FE
:1084F000CEF2000251701E212BE0002143F6400213
:108500000091C4F20202136843F020031360126862
:1085100002F020020092009A4EF60C52CEF20002B7
:108520001268C2F3022282F00703042B28BF04233F
:10853000033A38BF0A464FF0FF3199400B2323EA34
:10854000010191404EF21D420901CEF200029176E6
:10855000372101F01F02012303FA02F24EF2001349
:10856000CEF2000343EAD10121F003010A600221A7
:1085700080F83D10026840F6FF3E1368C4F2000E1A
:1085800072450FDCB2F1804F19D040F20041C4F2C5
:1085900000018A4213D040F60001C4F200018A4271
:1085A0000DD010E040F60041C4F200018A4206D02E
:1085B000624504D00021C4F201018A4203D18168DE
:1085C00023F070030B4341F6FF71C4F200018A42AD
:1085D0000FDC724521DCB2F1804F41D040F2004106
:1085E000C4F200018A423BD040F60001C4F200010F
:1085F00034E043F6FF71C4F201018A421EDC42F20C
:108600000001C4F200018A422AD00021C4F2010113
:108610008A4225D0624523D026E040F60041C4F2CC
:1086200000018A421CD041F60001C4F200018A42D6
:1086300016D041F60041C4F200010FE044F20001FF
:10864000C4F201018A420BD044F60001C4F20101D8
:108650008A4205D044F20041C4F201018A4203D1AA
:10866000016923F440730B4323F080018369D0F840
:1086700004E0C46819431160D46242F48061C2F816
:1086800028E0614504BF416911630121516180F80F
:108690003D1001B0BDE810407047000080B590F873
:1086A0003C20012A08BF80BD012280F83C20022224
:1086B00080F83D20D0F800C04FF67772DCF8083023
:1086C00023EA0202CCF808200B683F2B1CDD5F2B4D
:1086D00020DD602B4FD0B3F5005F6CD0702B40F0E5
:1086E0009E80D1E901E3C968DCF8082043EA0E0363
:1086F00022F47F4243EA01211143CCF80810DCF850
:10870000081041F0770188E01F2B28DC5BB3102BA9
:1087100029D084E0402B61D0502B40F08080D1F8EC
:1087200004E0C968DCF82030DCF8202022F00102E7
:10873000CCF82020DCF8182022F0F00242EA0111E7
:1087400023F00A0242EA0E02CCF81810CCF82020DE
:10875000DCF8081041F0570121F020015DE0202BEA
:1087600001D0302B5BD1DCF8081021F070011943E7
:1087700041F0070151E0D1F804E0C968DCF820308D
:1087800023F01003CCF82030DCF81830DCF820207F
:1087900023F4704322F0A00243EA013142EA0E12B0
:1087A000CCF81810CCF82020DCF8081041F0670154
:1087B00021F0100131E0D1E901E3C968DCF80820BB
:1087C00043EA0E0322F47F4243EA01211143CCF82D
:1087D0000810DCF8081041F480411EE0D1F804E0F4
:1087E000C968DCF82030DCF8202022F00102CCF847
:1087F0002020DCF8182022F0F00242EA011123F0D8
:108800000A0242EA0E02CCF81810CCF82020DCF85C
:10881000081041F0470121F03001CCF80810012187
:1088200080F83D10002180F83C1080BD01680A6985
:10883000920744BFCA685FEA827239D40A69520754
:1088400044BFCA685FEA427239D40A69120744BF5A
:10885000CA685FEA027239D40A69D20644BFCA689C
:108860005FEAC26239D40869C0071FBFC8685FEAFF
:10887000C0706FF0010008610869000641BFC86858
:108880005FEA00606FF0800008610869400641BF40
:10889000C8685FEA40606FF04000086108698006C0
:1088A00041BFC8685FEA80606FF0200008617047D0
:1088B0006FF002020A618A6900220277BEE76FF058
:1088C00004020A618A6900220277BEE76FF008029B
:1088D0000A61CA6900220277BEE76FF010020A61DE
:1088E000CA6900220277BEE74AF22850C2F20100AC
:1088F0000178012919D10021017041F204004AF2E6
:108900002452CEF20000C2F2010242F67023016846
:108910001268C1F200031F68891A3944196000689F
:1089200042F67421C1F2000108604EF2FF054BF6D9
:108930008C5640F21847C0F2F5550FF22C08C2F2DF
:108940000106C4F202074FF4800400E03C60404698
:10895000002104F077FC00BF3068A842F6D2013055
:10896000306000BFF8E700BF48617264204661755F
:108970006C74000080B5C16901B180BD816BCA6BA8
:10898000824266D1D1F800E0DEF81C3003F4407377
:10899000B3F5007F07D0DEF81C3013F4407F02D01F
:1089A0000EF104030FE043F20443C4F2000303F5A5
:1089B0007F7C44F20403C4F20003E64504BF43F2A3
:1089C0000443C4F200031A6822F001021A60002274
:1089D0004A864A8DEABB43F60043C4F200030122F3
:1089E0009E4581F8412034D147F2D172C1F2000294
:1089F000137833B147F6F91CC1F2000C01238CF84F
:108A000000304CF2282CC2F2010C00238CF800300C
:108A10004FF0010C47F2F07E82F800C0C1F2000E68
:108A20009EF801300EF12402002B08BF0EF108025F
:108A300012680A2A02BF4BF6D472C2F2010282F80F
:108A400000C047F6FC12C1F20002136803F5C073C0
:108A500013608A6B824290D10868C26902F4407246
:108A6000B2F5007F14D0C26912F4407F10D043F2F7
:108A70000442C4F2000202F57F7344F20402C4F21D
:108A80000002984204BF43F20442C4F2000200E034
:108A9000021D136823F00203136000224A854A8EE8
:108AA000002A7FF46AAF43F60043C4F200030122B8
:108AB000984281F8412018BF80BD47F2D170C1F2C1
:108AC0000000017829B147F6F911C1F20001012235
:108AD0000A704CF22821C2F2010100220A70012121
:108AE000017047F2F070C1F20000427800F12403F7
:108AF000002A08BF00F1080318680A2802BF4BF6D5
:108B0000D470C2F20100017047F6FC10C1F20000FF
:108B1000016801F5C071016080BD0000806B0168D3
:108B20004A6822F003024A6043F20442C4F200029F
:108B300002F57F7302F54062994204BF43F204429A
:108B4000C4F20002116821F0030111600021418587
:108B50004186012180F84110416C41F008014164D7
:108B600070470000806B43F600410068C4F20001CA
:108B7000884218BF704747F2D171C1F200010878EE
:108B800028B147F6F910C1F20000012202704CF240
:108B90002822C2F2010201201070087047F2F07121
:108BA000C1F200014A7801F12403002A08BF01F153
:108BB000080319680A2902BF4BF6D471C2F20101F9
:108BC000087047F6FC10C1F20000016801F5C071A1
:108BD0000160704783B001688A68029290F8412072
:108BE000042A1DD1029AD20713D04A68520610D522
:108BF000CA68C36A23F8022BC362428E013A4286D6
:108C0000428E32B94A6822F060024A60012280F83E
:108C10004120029A520644BF4A685FEA826213D436
:108C200090F84120032A0DD1029A920744BF4A6866
:108C30005FEA02621BD4029A120744BF4A685FEAE5
:108C4000826227D403B070474A6822F060024A600B
:108C500000220192CA6801928A680192019A012257
:108C600080F84120426C42F002024264D8E7426A36
:108C700032F8023BCB604262428D013A4285428D1E
:108C8000002AD8D14A6822F0A0024A60012280F866
:108C90004120D0E74A6822F0A0024A6000220092F8
:108CA000896800910099012180F84110416C41F0E0
:108CB0000401416403B0704782B049F60000C1F678
:108CC000F070019047F2B470C1F200000121017010
:108CD0004BF6F470C2F2010000210170B1A0002136
:108CE00004F0B0FA04F074FD49F6EC62C1F200023F
:108CF000106800BF1168091AB1F57A7F0ED81168A3
:108D0000091AB1F57A7F09D81168091AB1F57A7F85
:108D100004D81168091AB1F57A7FEBD94EF6235CB5
:108D2000CEF2000CBFF35F8FDCF801004EF2100EA4
:108D300020F48030CCF801000020CEF2000ECCF8F8
:108D40007100DEF8001043F6000321F00201C4F2C6
:108D50000203CEF80010EFF3108172B6CEF80000D7
:108D6000CEF80800CEF804001068196841F001013F
:108D70001960196889071CD41168091A022900F2C0
:108D8000F1801968890714D41168091A022900F2C0
:108D9000E980196889070CD41168091A022900F2C0
:108DA000E1801968890704D41168091A0229E0D9F9
:108DB000D8E01868002140F080001860106841F287
:108DC000883499609D68116815F00C0F1ED0091A3F
:108DD000A14200F2C7809D68116815F00C0F15D0F4
:108DE000091AA14200F2BE809D68116815F00C0FAF
:108DF0000CD0091AA14200F2B5809D68116815F0E7
:108E00000C0F03D0091AA142DCD9ABE0186820F49A
:108E1000502018601C681068A4031BD5401A6428F1
:108E200000F2A0801C681068A40313D5401A6428BF
:108E300000F298801C681068A4030BD5401A6428BF
:108E400000F290801C681068A40303D5401A6428BF
:108E5000E0D987E0196821F0807119601C681168F9
:108E6000A40118D5091A02297CD81C681168A4012C
:108E700011D5091A022975D81C681168A4010AD5F0
:108E8000091A02296ED81C681168A40103D5091AB1
:108E90000229E3D966E0186820F08060186018683D
:108EA000000119D51068401A02285BD81868000123
:108EB00012D51068401A022854D8186800010BD542
:108EC0001068401A02284DD81868000104D51068AF
:108ED000401A0228E3D945E043F21000C0F20040F6
:108EE000586043F20000C2F20000C3F88400D86862
:108EF00042F2004120F4F850D860D868C0F2F40182
:108F000020F40050D860D86840F41F00D860D868BA
:108F100040F40010D860586F20F001005867586F77
:108F200040F0807058674AF24830C2F20100016098
:108F300049F6F060C1F20000027843F67F61CEF896
:108F40000410F0218CF8001000210723012ACEF82C
:108F50000810CEF8003005D15CF8172C8CF8001002
:108F6000012101704FF0FF30CEF87001CEF8700291
:108F7000CEF87401CEF87402CEF87801CEF87802FB
:108F8000CEF87C01CEF87C02CEF88001CEF88002CB
:108F900062B6019840680199096881F308888047A2
:108FA000FEE700BF466C61736820444655206D6F34
:108FB0006465000070B500254FF0C0422A21C6F25A
:108FC0000805118000230121DF262B802B802980BA
:108FD0002E802B2616802B802B803F2329802B80F0
:108FE0002C2349F204741380C1F2000494F8342055
:108FF00045F26066C2F20106012A308023D084F86F
:10900000341094F8350001281AD1022084F8350074
:10901000002060652068A1680268402922F480224F
:10902000026047F23052426031462A4604BF294668
:1090300032468160C260016841F00101016002E0D6
:10904000002084F834002046FDF794FB94F83400A7
:10905000012824D0012084F8340094F83500012838
:109060001AD1022084F83500002060652068A168CC
:109070000268402922F48022026047F230524260A6
:1090800031462A4604BF294632468160C2600168E3
:1090900041F00101016002E0002084F83400204624
:1090A000FDF768FB94F83400012824D0012084F8EF
:1090B000340094F8350001281AD1022084F83500D4
:1090C000002060652068A1680268402922F480229F
:1090D000026047F23052426031462A4604BF2946B8
:1090E00032468160C260016841F00101016002E026
:1090F000002084F834002046FDF73CFB94F834004F
:10910000012824D0012084F8340094F83500012887
:109110001AD1022084F83500002060652068A1681B
:109120000268402922F48022026047F230524260F5
:1091300031462A4604BF294632468160C260016832
:1091400041F00101016002E0002084F83400204673
:10915000FDF710FB94F83400012824D0012084F896
:10916000340094F8350001281AD1022084F8350023
:10917000002060652068A1680268402922F48022EE
:10918000026047F23052426031462A4604BF294607
:1091900032468160C260016841F00101016002E075
:1091A000002084F834002046FDF7E4FA94F83400F7
:1091B000012823D0012084F8340094F835000128D8
:1091C00019D1022084F83500002060652068A1686C
:1091D0000268402922F4802202604FF46162314625
:1091E000426004BF294635468160C560016841F090
:1091F0000101016002E0002084F8340049F20470AB
:10920000C1F20000BDE87040FDF7B4BA2DE9F04F9F
:1092100081B0B2F5EF7FDDF828E088BF40F2DF12C1
:10922000B3F59F7F88BF40F23F13571C5E1CBFB24F
:10923000B6B23F1A761A7E43002537464FF0C04C2F
:109240002A24C6F20805B6F5163F28BF4FF4163794
:10925000ACF80040040AC0B22C802880100A288094
:10926000D0B228802B20ACF80000080A2880C8B2B1
:109270002880180A2880D8B245F2606928802C20FE
:10928000C2F20109332FACF80000A9F800E043D383
:109290004BF27320C4F2E750A7FB0001480B47F2E2
:1092A000305600FB167049F20474C1F2000447F214
:1092B0002F5A4FF0010B4FF00008009007E000BF5D
:1092C00084F834802046FDF755FABF1B36D094F859
:1092D0003400574535D90128F4D084F834B094F8D7
:1092E00035000128ECD1022084F83500C4F8548000
:1092F0002068A1680268402922F480220260494661
:109300002A46466004BF29464A468160C260016819
:1093100041F001010160D5E786B100BF012EA5F83B
:1093200000E00BD0022EA5F800E007D0032EA5F830
:1093300000E003D0043EA5F800E0EFD101B0BDE8A5
:10934000F08F012822D0012084F8340094F83500F1
:10935000012818D1022084F83500002060652068BB
:10936000A1680268402922F480220260009A4946DE
:10937000426004BF29464D468160C560016841F0E6
:109380000101016002E0002084F8340049F2047019
:10939000C1F2000001B0BDE8F04FFDF7EBB90000ED
:1093A0002DE9F04F87B0994209D90D468346AB426B
:1093B0000BD82F46CDF818B01D46934607E01D4642
:1093C00093460B460246AB42F3D91F460692109BCA
:1093D000312D26D106990FFA8BF081425846C8BF2D
:1093E0000846BCBF58468B4602B2934202460FFA6B
:1093F0008BF1C8BF1A468B42BCBF02469B46501C2D
:1094000001B20029D8BF002081B2B1F5EF7F88BF3B
:1094100040F2DF1082B25A4514D2104631215A462A
:1094200012E03A4629B2312F18BF013A0FFA82F8FA
:10943000A3EB0B004145C5F1310403950CDD0FFA98
:1094400080FA4BE058463121119F31230097FFF7F6
:10945000DDFE07B0BDE8F08F069A791BA2EB0B0288
:1094600009B202970591A1B20FFA82F90FFA80FAB8
:1094700000270026019404910598049996FBF0F0CA
:1094800097FBF1F15844594402B20BB29A420B4691
:10949000C4BF0346084682B2581C01B200294FF0EF
:1094A0000001D8BF084681B2B1F5EF7F88BF40F216
:1094B000DF1083B2A9B2119C934226BF10461A4610
:1094C00018460B464E4457440094FFF79FFE681C15
:1094D00005B24545D0DD109BDDE9014728B23128B2
:1094E0003DDC0699C7F13102591A0BB203991FFAF4
:1094F00082F8411AC01B01FB0AF600FB03F71FFAB2
:1095000084F9059397FBF8F00699059C084496FBAF
:10951000F9F102B259440BB29A420B46C4BF03465A
:10952000084682B2581C01B20029D8BF002081B27F
:109530002744B1F5EF7F88BF40F2DF1083B2A9B2B4
:10954000119C934226BF10461A4618460B465644B5
:109550000094FFF75BFE28B201353128D2DB07B05B
:10956000BDE8F08F4FF0C0400121018049F6EC606A
:10957000C1F20000016800BF0268521A152A0BD21E
:109580000268521A142A07D80268521A142A03D8F9
:109590000268521A152AEFD34FF0C04111220A80F7
:1095A000016800BF0268521A152A0BD20268521ACB
:1095B000142A07D80268521A142A03D80268521AC9
:1095C000152AEFD34FF0C042132300211380D0237C
:1095D000C6F2080113804FF0070C4223A1F800C027
:1095E0000B8018230B80D123138000230B801023C2
:1095F000A1F800C00B80D223138001220A8002222E
:109600000A80026803689B1A152B0BD203689B1A09
:10961000142B07D803689B1A142B03D803689B1AD2
:10962000152BEFD34FF0C042C023138010220A80C5
:109630003B220A8000220A8002220A8011220A802C
:10964000026800BF03689B1A152B0BD203689B1A94
:10965000142B07D803689B1A142B03D803689B1A92
:10966000152BEFD34FF0C042C523138003220A808D
:10967000026800BF03689B1A152B0BD203689B1A64
:10968000142B07D803689B1A142B03D803689B1A62
:10969000152BEFD34FF0C042C82313800022322392
:1096A0000A800B8036230B8045230B8006230B801A
:1096B00016230B8037230B8075230B8077230B80B9
:1096C00054230B800C230B800A80026803689B1ACA
:1096D000152B0BD203689B1A142B07D803689B1A0F
:1096E000142B03D803689B1A152BEFD34FF0C042FD
:1096F0003623138008220A80026800BF03689B1A81
:10970000152B0BD203689B1A142B07D803689B1ADE
:10971000142B03D803689B1A152BEFD34FF0C042CC
:109720003A23138055220A80026800BF03689B1AFF
:10973000152B0BD203689B1A142B07D803689B1AAE
:10974000142B03D803689B1A152BEFD34FF0C0429C
:109750002A23138000220A800A8001220A803F22E5
:109760000A80026803689B1A152B0BD203689B1AA8
:10977000142B07D803689B1A142B03D803689B1A71
:10978000152BEFD34FF0C0422B23138000220A8009
:109790000A8001220A80DF220A8001680268521AC8
:1097A000152A0BD20268521A142A07D80268521AD4
:1097B000142A03D80268521A152AEFD34FF0C04179
:1097C00021220A80016800BF0268521A152A0BD2B2
:1097D0000268521A142A07D80268521A142A03D8A7
:1097E0000268521A152AEFD34FF0C04138220A807E
:1097F000016800BF0268521A152A0BD20268521A79
:10980000142A07D80268521A142A03D80268521A76
:10981000152AEFD34FF0C04129220A80016808E0E1
:109820000268521A142A88BF70470268521A152A11
:1098300007D20268521A152A03D20268521A142A51
:10984000EED970472DE9F04F85B0202AC0F0AB81EA
:1098500047090E2F00F2A7818F09042F00F2A38180
:10986000DDF83CC00CEB4C0700EB4705002D00F089
:109870009A8101EBCC06002E00F095810024013D79
:109880004FF0C0492A27C6F20804AF2A88BF013228
:109890001FFA85FAA9F80070070AC0B22780208055
:1098A0004FEA1A202080E8B220802B20013EA9F840
:1098B0000000080A1FFA86F82080C8B220804FEA0C
:1098C00018202080F0B220802C20A9F80000D0B20F
:1098D00080004FF6887150FA82F0C0F603010A1832
:1098E000085CDDF838E00490507800270390907809
:1098F0000290D07801901079009003E00137082F92
:1099000000F051810120019E00FA07F504980399A7
:10991000029A05EA0608009E284029402A4005EAE6
:1099200006094FF0000A05E00AF1010A4FFA8AF52C
:109930006545E3DAE0B14FF0000B00BF4BF00105E5
:109940006DB26545238031DA4BF002056DB2654595
:1099500023802BDA4BF003056DB26545238025DAB1
:109960000BF1040B4FFA8BF565452380E6DB1DE018
:10997000002500BF45F0010676B26645A4F800E078
:1099800014DA45F0020676B26645A4F800E00DDA76
:1099900045F0030676B26645A4F800E006DA043521
:1099A0006EB26645A4F800E0E4DB00BF0025B9B163
:1099B00045F0010676B2664523802DDA45F00206B1
:1099C00076B26645238027DA45F0030676B266450F
:1099D000238021DA04356EB266452380E8DB1BE084
:1099E00045F0010676B26645A4F800E014DA45F0C9
:1099F000020676B26645A4F800E00DDA45F00306EB
:109A000076B26645A4F800E006DA04356EB2664523
:109A1000A4F800E0E4DB00BF0025BAB145F0010680
:109A200076B2664523802DDA45F0020676B26645A9
:109A3000238027DA45F0030676B26645238021DAD3
:109A400004356EB266452380E8DB1BE045F0010675
:109A500076B26645A4F800E014DA45F0020676B264
:109A60006645A4F800E00DDA45F0030676B26645D7
:109A7000A4F800E006DA04356EB26645A4F800E00A
:109A8000E4DB00BF0025B8F1000F17D045F0010658
:109A900076B2664523802DDA45F0020676B2664539
:109AA000238027DA45F0030676B26645238021DA63
:109AB00004356EB266452380E8DB1BE045F0010605
:109AC00076B26645A4F800E014DA45F0020676B2F4
:109AD0006645A4F800E00DDA45F0030676B2664567
:109AE000A4F800E006DA04356EB26645A4F800E09A
:109AF000E4DB00BF0025B9F1000F17D045F00106E7
:109B000076B2664523802DDA45F0020676B26645C8
:109B1000238027DA45F0030676B26645238021DAF2
:109B200004356EB266452380E8DB1BE045F0010694
:109B300076B26645A4F800E014DA45F0020676B283
:109B40006645A4F800E00DDA45F0030676B26645F6
:109B5000A4F800E006DA04356EB26645A4F800E029
:109B6000E4DB00BF002500BF45F0010676B2664584
:109B7000A4F800E0BFF6D8AE45F0020676B266451E
:109B8000A4F800E0BFF6D0AE45F0030676B2664515
:109B9000A4F800E0BFF6C8AE04356EB26645A4F87E
:109BA00000E0E1DBC0E605B0BDE8F08F2DE9F04F45
:109BB000B3EB010848BFC8F10008171A48BF7F423D
:109BC000B84508DD9446024699420AD860469E464A
:109BD00094460B4607E09C4613460A4601469942C6
:109BE000F4D910468E464FF0FF31604588BF012101
:109BF0009E4538BFBDE8F08FAEEB03020FFA82F945
:109C0000B0EB0C0609EBD9704FEA600440F200009B
:109C100048BF7642DDF824B0C6F20800B84536B237
:109C20004FF0C0474FF02C0A26DD00BF2A223A80B1
:109C3000CCF307255FFA8CF82B220580A0F8008072
:109C40000580A0F800803A80C3F30725DAB20580CA
:109C500002800580028022B2941B220403F10103DA
:109C60009AB2A7F800A044BF8C4409FA84F4724564
:109C7000A0F800B0DAD925E02A223A80C3F30725FC
:109C80005FFA83F82B220580A0F800800580A0F8F9
:109C900000803A80CCF307255FFA8CF205800280C1
:109CA0000580028022B2941B220403F101039AB2C0
:109CB000A7F800A044BF8C4409FA84F47245A0F8C8
:109CC00000B0D9D9BDE8F08F2DE9F04381B0064648
:109CD00010B200281446DDF82090D8BF0024B4F557
:109CE000EF7F1F46904688BF40F2DF14B4420D4616
:109CF0000BD22046294632462B46CDF80090FFF77E
:109D000085FA2046394632460AE030462946224640
:109D10002B46CDF80090FFF779FA304639462246B7
:109D20003B46CDF80090FFF771FA781E01B200298A
:109D3000D8BF002081B2B1F59F7F88BF40F23F10AD
:109D400084B23046AC420BD2214632462B46CDF887
:109D50000090FFF75BFA4046214642462B460AE058
:109D6000294632462346CDF80090FFF74FFA404689
:109D7000294642462346CDF80090FFF747FA01B046
:109D8000BDE8F0832DE9F04F83B0DDE90E68DDE931
:109D90000C750093198000244FF4F07E4FF4A073EB
:109DA0004FF000094FF0000A3A8034802C80029373
:109DB00008E000BF98F80A100A4400210234282C59
:109DC00000F0A480055D002D00F0A0800D2D53D083
:109DD0000A2D05D198F80A100A4400214CE000BF72
:109DE00098F808C0AC4547D898F80970AF4243D3FB
:109DF000D8F80470A5EB0C0507EBC50595F90570BF
:109E00000FFA8EF30F440FFA87FC95F90660D346DC
:109E1000CDF804909C45AB7895F803A0B8BFBE463A
:109E20008C464146F046DDF808E016443B440FFA04
:109E300086F9013B0FFA8EF7B9450FFA83F90FFA4D
:109E40008BF7B8BFB646B945DDF8049006EB0A07B4
:109E5000A7F10107CDF808E03EB2C8BF9B460FFA54
:109E600089F39E422B79C64688466146DA460CEB5A
:109E70000301C8BFB94600BF03195D78002D45D066
:109E80000D2D9BD00A2D95D098F80870AF4295D82B
:109E900098F80930AB4291D3D8F80430EF1B03EBAC
:109EA000C70595F90530CDF804900B440FFA83F9F6
:109EB0000FFA8EF6B145AE7895F906701E4495F806
:109EC0000390C346A6F10108B8BF9E46029E174400
:109ED0000FFA87FC33B29C450FFA88FC0FFA8AF31D
:109EE000B8BF3E469C4507EB0903DDF80490A3F19B
:109EF000010302961FB20FFA89F6C8BFC246B742E5
:109F00002F79D8463944C8BF994657E70FFA8EF0E3
:109F10000FFA8AF1814207DB00980D99A0F800E062
:109F2000AAEB0E0001300880029A0FFA89F110B2F4
:109F3000814206DB0C980E990280A9EB02000130E9
:109F4000088003B0BDE8F08F2DE9F04F85B00F9C7D
:109F5000074604EB44004500D01E984693460E4643
:109F6000002180B24FF000094FF0000A02900392E6
:109F70001FE000BF002A43D0A9EB0A0000FB0560E8
:109F80000E9980B20091594643460194FFF75AFC5E
:109F900009F10100A0EB0A0101FB056149F6DE624F
:109FA000C1F2000211801FFA89F281B27F2A814634
:109FB00026D27A5C5E2ADDD1C81940786F28DBD1C1
:109FC000C34609F101086FEA0A000AF1010A049088
:109FD0001FFA88F0A8EB0A0101FB05613A5C0E98B4
:109FE0005B46009088B202990194FFF72BFC04991C
:109FF00009F10200C146D846DDF80CB00144CBE7B8
:10A0000005B0BDE8F08F00002DE9F04F89B0DDE923
:10A0100012EC49F6DE690026C1F20009C6F2080614
:10A020004FF00008A9F800100CE000BF9CF80A707F
:10A0300000213A44A9F8001008F10108B8F5807F22
:10A0400000F09A8110F808500A2DEFD00D2DF3D0B2
:10A05000002D00F091819CF80870BD42ECD39CF873
:10A060000940A542E8D8DCF80440A5EB070A04EB58
:10A07000CA05AF78002F00F07C81EF78002F00F048
:10A0800078815FFA8AF7CDE9005004EBC70595F9AE
:10A09000060095F803A0029210FA82F234F837B065
:10A0A00002EB0A071404A7F101074FF0000495F82A
:10A0B00004C038B248BF22468CB200284FF0C049D5
:10A0C0004FF02A004FEA1424A9F80000348001EB75
:10A0D0000C04A4F10104C9B2CDF81CC03180A1B2B6
:10A0E0004FEA11213180E1B2318091B24FF02B0063
:10A0F0004FEA1121A9F800003180D1B24FF00000E1
:10A10000D8BF07463180B9B2090A3180F9B2BAF135
:10A11000000F4FF02C003180CDF818A0A9F80000F6
:10A1200000F01C81681D05900798AF1C01460128AE
:10A1300098BF01214A1ECDE9032101F0FC01002551
:10A140004FF0000C002408E0A6F800E00798089DF6
:10A15000069A0135954280F001810028089500F0AB
:10A16000B18005984FF0000A90F9009003980328F9
:10A17000049800F00300054627D200280798E6D08F
:10A18000CA45C0F2A18038784844504540F39C80CD
:10A190005FEA4C700CF1010C06D113981FFA8BF496
:10A1A00000680BF1010B045D60B2B0F1FF3F18468F
:10A1B000C8BF70463080640088E000BFA6F800E0A9
:10A1C0000AF1040A28465145D7D0CA451ADB387827
:10A1D0004844504516DD5FEA4C700CF1010C06D185
:10A1E00013981FFA8BF400680BF1010B045D60B249
:10A1F000B0F1FF3F18464FEA4404C8BF70463080B4
:10A2000002E000BFA6F800E00AF10100484519DBB2
:10A210003A784A44824215DD5FEA4C700CF1010C39
:10A2200006D113981FFA8BF200680BF1010B845CC6
:10A2300060B2B0F1FF3F1846C8BF7046308064007E
:10A2400002E000BFA6F800E00AF10200484519DB71
:10A250003A784A44824215DD5FEA4C700CF1010CF9
:10A2600006D113981FFA8BF200680BF1010B845C86
:10A2700060B2B0F1FF3F1846C8BF7046308064003E
:10A2800002E000BFA6F800E00AF10300484595DBB4
:10A290003A784A44824291DD5FEA4C700CF1010C3D
:10A2A00006D113981FFA8BF200680BF1010B845C46
:10A2B00060B2B0F1FF3F1846C8BF704630806400FE
:10A2C0007EE700BF002042E7A6F800E0012D284607
:10A2D0003FF43CAF0AF1010048451BDB3A784A44A1
:10A2E000824217DD5FEA4C700CF1010C06D1139825
:10A2F0001FFA8BF200680BF1010B845C60B2B0F1C5
:10A30000FF3F1846C8BF704630806400022D3FF4FE
:10A310001DAF04E0A6F800E0022D3FF417AF0AF1EC
:10A3200002004845FFF610AF3A784A4482427FF770
:10A330000BAF5FEA4C700CF1010C06D113981FFAB9
:10A340008BF200680BF1010B845C60B2B0F1FF3F4F
:10A350001846C8BF704630806400F7E649F6DE69EB
:10A36000C1F20009B9F80010029ADDF84CC0DDE92D
:10A3700000502F7939445DE609B0BDE8F08F000048
:10A380002DE9F04F8FB047F2C171C1F20001097899
:10A3900011B10FB0BDE8F08F044678B147F2B47048
:10A3A000C1F20000007850B34BF69470C2F2010085
:10A3B0000121417181710FB0BDE8F08F4BF6B8708B
:10A3C00047F2F073C2F20100C1F20003026858784C
:10A3D0001D6A596800282B4608BF0B469A42D8D000
:10A3E00047F2B472C1F2000212787AB14BF694705F
:10A3F000C2F20100012141710FB0BDE8F08F47F2B8
:10A40000F072C1F2000250785168156A47F2B473D5
:10A41000002847F2F070C1F200034FF00102C1F2D0
:10A4200000001A7008BF0D4690F85911B0F85A0193
:10A4300043F609525043002918BF05EB80154CF62E
:10A44000FF10C3F69A30854228BF05464BF6B87018
:10A45000C2F20100056049F27F60C0F298004EF23E
:10A46000FF0671278542C0F2F55688BF4927B542DD
:10A4700088BF25277CB14AF20800C2F201000068BB
:10A480003221B0F800C0252040F297127C23CDF88D
:10A4900000C0FEF7BBFEB5420CD84AF20800C2F27B
:10A4A000010000684121068825203A467423009661
:10A4B000FEF7ACFE44F6D350C1F26200A5FB0012D9
:10A4C0009109A1FB00034DF68360C4F21B30A5FB8C
:10A4D00000064FF61840CFF6FF7001FB00589809B0
:10A4E0004FF47A714843B50C41F29C06C0EB9219C7
:10A4F00047F2B570C0F60406C1F20000314642468C
:10A50000F5F762FF4BF6AE70C2F2010031464A46E3
:10A51000F5F75AFF47F2BB70C1F2000031462A46F8
:10A52000F5F752FF4AF2680A43F2A02642F6221BD0
:10A53000C2F2010AC0F60306C1F2000B6CB9BBF807
:10A540000000854209D102AF38463221F7F717F9EA
:10A5500047F2B47BC1F2000B1CE04AF20800C2F2E1
:10A56000010000683946438900887422009047F250
:10A57000BB70C1F200000196FFF746FD02AF3846FE
:10A580003221ABF80050F7F7FAF847F2B47BC1F28A
:10A59000000B1CB9BAF8000081451ED04BF6AE7115
:10A5A00040F6BF530025C2F20101C0F6040338464D
:10A5B0000322009516F0CCFC4AF20800C2F201001A
:10A5C0000068AA2183890088742200903846019689
:10A5D000FFF71AFDAAF8009094B942F62010C1F2D4
:10A5E0000000008880450BD14BF6CE70C2F201000E
:10A5F000012101704BF69470C2F20100053033E086
:10A6000047F2B57140F6BF530025C1F20001C0F614
:10A61000040338460322009516F09AFC4AF208001B
:10A62000C2F20100006849F22016C3890088C0F612
:10A6300003060090384640F2331172220196FFF76C
:10A64000E3FC42F62010C1F20000A0F800804BF6B7
:10A65000CE70C2F20100012101704BF69470C2F27B
:10A660000100457114B106300021017000208BF803
:10A6700000000FB0BDE8F08F2DE9F04F81B02DED57
:10A68000048BAAB047F2C171C1F200010978002918
:10A6900041F0638047F2B471C1F200010A783AB127
:10A6A0004BF69470C2F201000121417201F055B8DD
:10A6B0004FF0010881F800804CF21B01C2F2010149
:10A6C000097847F2F073C1F200030790E9B947F641
:10A6D000A611C1F200010978B9B947F69D11C1F27E
:10A6E0000001097889B95A7803F12401002A08BFCA
:10A6F00003F1080109680A2907D04BF6F871C2F284
:10A7000001010968002901F034804AF20804C2F20C
:10A71000010420687D210088712200905820852343
:10A720004FF05809FEF772FD4CF20800C2F201002A
:10A73000006821F045FD0B4641F202210DF1400A6F
:10A740000246C0F604015046F5F73EFE206800219F
:10A75000B0F800B00025002621E000BF002A40D05C
:10A76000A81B00EB400009EB400080B27D214FF4B4
:10A770007843CDF800B0CDF80480FFF763F8681C8B
:10A78000811B01EB410149F6DE6209EB4101C1F297
:10A7900000021180AAB281B27F2A054621D21AF89E
:10A7A00001205E2ADAD101EB0A0040786F28D7D168
:10A7B0006F1CF4430136B91BB8B201EB41011AF822
:10A7C000002009EB410080B27A214FF47843CDF8A4
:10A7D00000B0CDF80480FFF735F8A81C01193D46FC
:10A7E000CFE74AF20804C2F2010420687D21008804
:10A7F000A82200908F2085234FF08F0BFEF706FDD7
:10A800004CF20000C2F20100006821F0D9FC0B46B6
:10A8100041F282010246C0F604015046F5F7D4FD2C
:10A820002068002106884FF00109002500241FE060
:10A83000002A40D0281B00EB40000BEB400080B208
:10A840007D214FF478430096CDF80490FEF7FAFF8F
:10A85000681C011B01EB410149F6DE620BEB410173
:10A86000C1F200021180AAB281B27F2A054622D22B
:10A870001AF801205E2ADBD101EB0A0040786F282C
:10A88000D8D16F1C6FEA04080134391BB8B201EB50
:10A8900041011AF800200BEB410080B27A214FF4FD
:10A8A00078430096CDF80490FEF7CCFFA81C00EB8F
:10A8B00008013D46CEE74AF20804C2F201042068CE
:10A8C0007D210088DF220090C6208523C626FEF762
:10A8D0009DFC47F69010C1F20000006821F070FC6A
:10A8E0000B4641F282010246C0F604015046F5F7DC
:10A8F0006BFD2068002107884FF0010800254FF00C
:10A90000000B21E0002A44D0A5EB0B0000EB400037
:10A9100006EB400080B27D214FF478430097CDF8DC
:10A920000480FEF78FFF681CA0EB0B0101EB4101D7
:10A9300049F6DE6206EB4101C1F200021180AAB2C3
:10A9400081B27F2A054624D21AF801205E2AD9D185
:10A9500001EB0A0040786F28D6D16C1C6FEA0B0916
:10A960000BF1010BA4EB0B01A0B201EB41011AF8B2
:10A97000002006EB410080B27A214FF47843009723
:10A98000CDF80480FEF75EFFA81C00EB0901254608
:10A99000CCE74CF20000C2F2010090ED000A47F64D
:10A9A0009010C1F20000B1EE0C1A90ED002A9FED5C
:10A9B0003B3AB4EE410AF1EE10FAC8BFB0EE410ADC
:10A9C00022EE031ABDEEC11A20EE030A11EE100AA0
:10A9D000BDEEC01A11EE105A01464AF2080985422E
:10A9E00088BF2946C2F201099FED2D2A081AD9F81D
:10A9F00000103D3032EE400A4F8E86B2BDEEC00AE6
:10AA00003D208F213246962310EE108A0097FEF7E4
:10AA1000FDFBD9F800003D35C48AAFB230468F2126
:10AA20003A4696230094FEF7F1FBD9F800008F21F7
:10AA3000068805EB080082B2384696230096FEF79A
:10AA4000E5FBD9F800007D21008840F2A9120090B2
:10AA50004FF4C87085234FF4C87BFEF7D7FB47F649
:10AA60008810C1F2000090ED000A9FED0E1A0FF25F
:10AA7000F85120EE010ABDEEC00A10EE102A504631
:10AA80000692F5F7A1FCD9F800000021B0F818A053
:10AA9000048801270026002524E000BF25492A421A
:10AAA000000095430000C842002A40D0701B00EB14
:10AAB00040000BEB400080B27D215346009401978B
:10AAC000FEF7C0FE701C411B01EB410149F6DE623E
:10AAD0000BEB4101C1F200021180B2B281B27F2AB8
:10AAE000064624D210A8425C5E2ADDD10844407894
:10AAF0006F28DBD106F101086FEA05090135A8EBE3
:10AB000005011FFA88F001EB410110AA125C0BEB62
:10AB10004100012780B27A21534600940197FEF745
:10AB200091FEB01C00EB090146460127CCE7069CCC
:10AB30005A2048F21F516043C5F2EB11A0FB0112ED
:10AB40004AF20801C2F20101096896234F8E4FF4C0
:10AB5000B97101EB521542F28B31884288BF4FF434
:10AB6000E6754FF4B9708F212A460097FEF74EFB29
:10AB700047F2F076632CC1F200060DD84AF20800C5
:10AB8000C2F2010000688F21078EA8B24FF4E6726E
:10AB900096230097FEF73AFB0020CDE90E00CDE9A1
:10ABA0000C00CDE90A00CDE90800707806F1240216
:10ABB00006F10801002810460592069108BF0846D4
:10ABC000006808281DD8DFE800F005050A0A1616F7
:10ABD00027191900B6F87221B6F8703103E0B6F8FB
:10ABE0006E21B6F86C3141F29001C0F6040108A85C
:10ABF000F5F7EAFB19E0B6F876210FE0B6F8702118
:10AC00000CE044F65540C0F24C00099045F2427009
:10AC1000C4F23A60089008E0B6F8742141F2990154
:10AC2000C0F6040108A8F5F7CFFB1DAE304632216F
:10AC3000F6F7A5FD08AF30463946F5F728FEF5F7DB
:10AC40004AFE0B2809D820243046F5F744FE34523A
:10AC50003046F5F740FE0C28F6D31DA93846F5F727
:10AC600016FE4AF20800C2F2010000680021C48CFE
:10AC7000B0F800A04FF03C0B4FF001080026002573
:10AC800020E000BF002A44D0701B00EB40000BEB1B
:10AC9000400080B2A1212346CDF800A0CDF8048069
:10ACA000FEF7D0FD701C411B01EB410149F6DE624D
:10ACB0000BEB4101C1F200021180B2B281B27F2AD6
:10ACC000064626D27A5C5E2ADCD1C81940786F2805
:10ACD000DAD106F101086FEA05090135A8EB050193
:10ACE0001FFA88F001EB41013A5C0BEB41004FF099
:10ACF000010C80B29E212346CDF800A0CDF804C0FF
:10AD0000FEF7A0FDB01C00EB090146464FF001081C
:10AD1000CAE747F2F071C1F2000191F8470168B14A
:10AD200000208DF8280044F64340C5F241200990E8
:10AD300044F65210C3F6542008900DE091F8370104
:10AD4000002800F010854CF20400C2F201000268F5
:10AD5000C7A108A8F5F738FB1DAE30463221F6F73B
:10AD60000EFD0DF1200A30465146F5F790FDF5F73E
:10AD7000B2FD0B2809D820243046F5F7ACFD34523B
:10AD80003046F5F7A8FD0C28F6D31DA95046F5F777
:10AD90007EFD4AF20800C2F2010000680021B0F80E
:10ADA00028B0B0F800808C240127002600251EE082
:10ADB000002A42D0701B00EB400004EB400080B240
:10ADC000A1215B46CDF800800197FEF73BFD701C8A
:10ADD000411B01EB410149F6DE6204EB4101C1F286
:10ADE00000021180B2B281B27F2A064625D21AF83B
:10ADF00001205E2ADCD101EB0A0040786F28D9D10E
:10AE0000771C6FEA05090135791BB8B201EB4101E6
:10AE10001AF8002004EB41004FF0010C80B29E2193
:10AE20005B46CDF80080CDF804C0FEF70BFDB01CEA
:10AE300000EB09013E460127CBE74AF24C30C2F253
:10AE40000100006821F0BCF902460B468BA1504678
:10AE5000F5F7BAFA4AF20800C2F2010000680021D0
:10AE6000B0F82AB0B0F80080C824012700260025D9
:10AE70001FE000BF002A42D0701B00EB400004EB33
:10AE8000400080B2A1215B46CDF800800197FEF71B
:10AE9000D9FC701C411B01EB410149F6DE6204EB59
:10AEA0004101C1F200021180B2B281B27F2A06468E
:10AEB00025D21AF801205E2ADCD101EB0A00407885
:10AEC0006F28D9D1771C6FEA05090135791BB8B213
:10AED00001EB41011AF8002004EB41004FF0010C96
:10AEE00080B29E215B46CDF80080CDF804C0FEF70D
:10AEF000A9FCB01C00EB09013E460127CBE74AF252
:10AF00002C50C2F20100006821F05AF902460B46AB
:10AF10005DA15046F5F758FA4AF20800C2F2010066
:10AF200000680021B0F82CB0B0F800804FF48C74A9
:10AF30000127002600251EE0002A42D0701B00EBEE
:10AF4000400004EB400080B2A1215B46CDF80080B8
:10AF50000197FEF777FC701C411B01EB410149F69C
:10AF6000DE6204EB4101C1F200021180B2B281B293
:10AF70007F2A064625D21AF801205E2ADCD101EB91
:10AF80000A0040786F28D9D1771C6FEA050901358E
:10AF9000791BB8B201EB41011AF8002004EB410023
:10AFA0004FF0010C80B29E215B46CDF80080CDF8B9
:10AFB00004C0FEF747FCB01C00EB09013E46012728
:10AFC000CBE747F2F072C1F20002507802F1300193
:10AFD000002808BF02F11401087850B145F255402D
:10AFE000C0F24F00CDF8270043F64820C5F241508B
:10AFF00006E04620ADF8280043F64820C4F24F6032
:10B00000099044F64E70C4F254301DAE089030469C
:10B010003221F6F7B4FB0DF1200A30465146F5F720
:10B0200036FCF5F758FC0B2809D820243046F5F7F4
:10B0300052FC34523046F5F74EFC0C28F6D31DA9CD
:10B040005046F5F724FC4AF20800C2F201000068FD
:10B050000021B0F830B0B0F8008040F24F14012762
:10B060000026002535E000BF2564252500000000EE
:10B0700053484946543A256400000000564C543A5F
:10B08000252E3166200000004350553A252E3166AA
:10B0900020000000002A42D0701B00EB400004EBAF
:10B0A000400080B2A1215B46CDF800800197FEF7F9
:10B0B000C9FB701C411B01EB410149F6DE6204EB48
:10B0C0004101C1F200021180B2B281B27F2A06466C
:10B0D00025D21AF801205E2ADCD101EB0A00407863
:10B0E0006F28D9D1771C6FEA05090135791BB8B2F1
:10B0F00001EB41011AF8002004EB41004FF0010C74
:10B1000080B29E215B46CDF80080CDF804C0FEF7EA
:10B1100099FBB01C00EB09013E460127CBE747F243
:10B12000F070C1F2000090F8870101380F2834D880
:10B13000DFE800F008103318333333203333333370
:10B14000333333267A20ADF8280043F63400C4F6B2
:10B150006B001CE07A20ADF8280043F23240C4F6C0
:10B160006B0014E07A20ADF8280043F23120C4F6D9
:10B170006B000CE02020ADF8280046F6363004E0E5
:10B180002020ADF8280046F63330C7F64820099055
:10B1900044F24660C3F6542008904AF20800C2F216
:10B1A000010000680021B0F81EB0B0F800804FF434
:10B1B000D2740127002600251FE000BF002A42D0DC
:10B1C000701B00EB400004EB400080B2A1215B4605
:10B1D000CDF800800197FEF735FB701C411B01EB99
:10B1E000410149F6DE6204EB4101C1F20002118027
:10B1F000B2B281B27F2A064625D21AF801205E2A11
:10B20000DCD101EB0A0040786F28D9D1771C6FEAB6
:10B2100005090135791BB8B201EB41011AF800208C
:10B2200004EB41004FF0010C80B29E215B46CDF84B
:10B230000080CDF804C0FEF705FBB01C00EB09014F
:10B240003E460127CBE74AF20800C2F2010000683F
:10B250004121078840F2B31040F2C71249230097FA
:10B26000FDF7D4FF47F68610C1F2000000780028F1
:10B2700053D04CF21B00C2F20100007800284CD1E0
:10B2800047F6A610C1F200000078002845D147F625
:10B290009D10C1F20000007800283ED147F2F07006
:10B2A000C1F2000040780028DDE9050108BF08462A
:10B2B00000680A2831D04BF6F870C2F2010000682D
:10B2C00058BB4AF20800C2F20100006841F21E09B0
:10B2D000458F04880026C0F6040940F2B31A4FF0E7
:10B2E000010B40F2B918032E17D006EB460719F8E8
:10B2F00006200AEB470080B241212B460094CDF88E
:10B3000004B0FEF79FFA013649F6DE6108EB47000C
:10B31000802EC1F200010880E5D14BF6EE70C2F23A
:10B320000100007860B34AF20800C2F20100006830
:10B3300041F21E09458F04880026C0F6040940F238
:10B34000B31A4FF0010B40F2B91800BF032E17D00B
:10B3500006EB460719F806200AEB470080B24121A8
:10B360002B460094CDF804B0FEF76CFA013649F68E
:10B37000DE6108EB4700802EC1F200010880E5D1B4
:10B3800047F6F910C1F200000078012850D14CF2C4
:10B390001B00C2F201000078002849D147F6A61030
:10B3A000C1F200000078002842D147F69D10C1F29A
:10B3B00000000078E0BB47F2F070C1F20000407876
:10B3C0000028DDE9050108BF084600680A282FD0DB
:10B3D0004BF6F870C2F20100006848BB4AF2080060
:10B3E000C2F2010000680026458F04880FF630691C
:10B3F00040F2B31A4FF0010B40F2B918032E17D0E8
:10B4000006EB460719F806200AEB470080B24121F7
:10B410002B460094CDF804B0FEF714FA013649F635
:10B42000DE6108EB4700802EC1F200010880E5D103
:10B4300046F6EC50C1F20000007800284ED04CF2E5
:10B440001B00C2F201000078F0B947F6A610C1F265
:10B4500000000078C0B947F69D10C1F200000078E6
:10B4600090B947F2F070C1F2000040780028DDE9A1
:10B47000051008BF014608680A2805D04BF6F87089
:10B48000C2F20100006848B34AF20800C2F20100AB
:10B4900000680026458F04880FF6885840F2B319DB
:10B4A0004FF0010A40F2B91B032E17D006EB4607F6
:10B4B00018F8062009EB470080B241212B46009482
:10B4C000CDF804A0FEF7BEF9013649F6DE610BEBBC
:10B4D0004700802EC1F200010880E5D147F2E070FC
:10B4E000C1F20000007848B34AF20800C2F201003D
:10B4F00000680026458F04880FF62C5840F2B319D7
:10B500004FF0010A40F2B91B032E17D006EB460795
:10B5100018F8062009EB470080B241212B46009421
:10B52000CDF804A0FEF78EF9013649F6DE610BEB8B
:10B530004700802EC1F200010880E5D142F60000EC
:10B54000C4F20000006842F62416C0F3015141EA3B
:10B550008101C0F3034202EB4103C0F3023101EB6E
:10B560008101C0F3032202EB4102C0F3021101EB9F
:10B57000810100F00F00C1F2000600EB41003178BC
:10B5800047F20C644BF6C47A47F2E57B47F6E06875
:10B590004AF26A09C1F20004C2F2010AC1F2000BC8
:10B5A0009942C0F60308C2F2010923708AF800200C
:10B5B0008BF8000001D10798E8B341F29C0110AD6F
:10B5C000C0F6040128461A46F4F7FEFE40F6BF53C3
:10B5D0000027C0F60403284629460222009715F0EA
:10B5E000B7FC4AF20807C2F20107386840F2951129
:10B5F000B0F84E300088112200902846CDF8048023
:10B60000FEF702FD386849F6DE61B0F84E3000887A
:10B61000C1F200010988009040F64560C0F60400C0
:10B620001122CDF80480FEF7EFFC079920789AF8F4
:10B630000020307019B999F80000824243D041F2DD
:10B640009C0110ADC0F604012846F4F7BDFE40F69B
:10B65000BF530027C0F6040328462946022200975C
:10B6600015F076FC4AF20804C2F2010420684FF497
:10B67000D771B0F84E300088112200902846CDF8DE
:10B680000480FEF7C1FC206849F6DE61B0F84E3058
:10B690000088C1F200010988009040F64560C0F6BC
:10B6A00004001122CDF80480FEF7AEFC07999AF849
:10B6B000000089F8000031B19BF8002042F6251601
:10B6C000C1F2000612E042F62516C1F200069BF810
:10B6D00000203078824209D14BF69470C2F201000A
:10B6E00047F2B4720930C1F2000232E041F29C012B
:10B6F00010ADC0F604012846F4F766FE40F6BF53CD
:10B700000024C0F60403284629460222009415F0BE
:10B710001FFC4AF20800C2F20100006840F2C711A3
:10B72000B0F84E300088112200902846CDF80480F1
:10B73000FEF76AFC9BF80000079930704BF6947096
:10B7400047F2B472C2F20100C1F20002447211B1B8
:10B750000A3000210170002010702AB0BDEC048B6B
:10B7600001B0BDE8F08F44F24F60C0F24600FFF731
:10B77000DEBA42F63016C1F200061F1D03F12001A9
:10B7800096ED000A002ACDE9051708BF3946096879
:10B7900044F2FF32C0F69502914204D996ED000AB8
:10B7A0009FED671A01E09FED671AB8EEC00A9FEDA2
:10B7B000662A30EE010A9FED651A9FED653A9FED0E
:10B7C000654A20EE022A20EE011A32EE032AB4EE78
:10B7D000440AF1EE10FAB8BFB0EE412AB7EE000A03
:10B7E0009FED5D1A32EE002AB4EE412A42F61C1497
:10B7F000F1EE10FAC8BFB0EE412AB4EE402AC1F211
:10B800000004F1EE10FAB8BFB0EE402A94ED001A31
:10B81000B6EE083AB5EE004A21EE033A22EE042ACB
:10B8200032EE038AB4EE481AF1EE10FA08BF00288F
:10B8300000F0A58231EE482ABDEEC83A13EE105A48
:10B84000B5EE402AF1EE10FA05F13C0615DD4AF29C
:10B85000080032EE000AC2F20100BDEEC00A006824
:10B8600010EE101A0788701882B2B0B28F2196239A
:10B870000097FDF7CBFC94ED001A4AF20804C2F2DF
:10B880000104BDEEC10A216810EE100A00F13C026D
:10B890000F8800F13E0190B28AB28221A023009766
:10B8A000FDF7B4FC2068B2B2478E3C208F2196236E
:10B8B00003920097FDF7AAFC4BF6AC74C2F20104A8
:10B8C000208800EE100AB8EE400AB4EE408AF1EE8D
:10B8D00010FA11DA4AF20801C2F20101096800F116
:10B8E0003C020F8800F13E0190B28AB28F2196236C
:10B8F0000097FDF78BFC208849F6EC614BF6A872A7
:10B90000C1F20001C2F2010240B10B681768DB1BF3
:10B91000B3F57A7F84BF0138208000E0002083B235
:10B9200000EE103AB8EE400AB4EE408AF1EE10FA9A
:10B93000049515DD258008681060284612E000BFD8
:10B94000000013430000FE4237D02940D8828D40CA
:10B950003C0ABF423D0A58420000C7435555D541F5
:10B9600000F13C064AF20804C2F201042168962361
:10B97000CF8E00F13E01B0B28AB28F210097FDF761
:10B9800045FC20680027068B04880FF610094FF04D
:10B990003A0A4FF0010B4025012F17D007EB47085B
:10B9A00019F807200AEB480080B27D213346009445
:10B9B000CDF804B0FDF746FF013749F6DE6105EB2F
:10B9C0004800802FC1F200010880E5D14AF208004A
:10B9D000C2F20100006840F6FD59068B048800277A
:10B9E000C0F604094FF0540A4FF0010B4FF05A080B
:10B9F000012F17D007EB470519F807200AEB450080
:10BA000080B27D2133460094CDF804B0FDF71AFFD3
:10BA1000013749F6DE6108EB4500802FC1F20001D5
:10BA20000880E5D14AF20800C2F201000068002750
:10BA3000068B04880FF268794FF08A0A4FF0010BE9
:10BA40004FF09008012F17D007EB470519F8072092
:10BA50000AEB450080B27D2133460094CDF804B056
:10BA6000FDF7F0FE013749F6DE6108EB4500802F57
:10BA7000C1F200010880E5D14AF20800C2F20100DB
:10BA800000680027068B04880FF218794FF0BF0A70
:10BA90004FF0010B4FF0C508012F17D007EB4705FA
:10BAA00019F807200AEB450080B27D213346009447
:10BAB000CDF804B0FDF7C6FE013749F6DE6108EBAC
:10BAC0004500802FC1F200010880E5D14AF208004C
:10BAD000C2F2010000680027068B04880FF2C869D3
:10BAE0004FF0F40A4FF0010B4FF0FA08012F17D076
:10BAF00007EB470519F807200AEB450080B27D21C6
:10BB000033460094CDF804B0FDF79CFE013749F6AA
:10BB1000DE6108EB4500802FC1F200010880E5D10D
:10BB20004AF20800C2F2010000680027068B048870
:10BB30000FF278694FF4957A4FF0010B4FF4987833
:10BB4000012F17D007EB470519F807200AEB45002E
:10BB500080B27D2133460094CDF804B0FDF772FE2B
:10BB6000013749F6DE6108EB4500802FC1F2000184
:10BB70000880E5D14AF20800C2F2010000680027FF
:10BB8000068B04880FF2286940F2571A4FF0010B18
:10BB900040F25D18032F17D007EB470519F807206F
:10BBA0000AEB450080B27D2133460094CDF804B005
:10BBB000FDF748FE013749F6DE6108EB4500802FAE
:10BBC000C1F200010880E5D14AF20800C2F201008A
:10BBD00000680027068B04880FF2D8594FF4C67A04
:10BBE0004FF0010B4FF4C978032F17D007EB47052F
:10BBF00019F807200AEB450080B27D2133460094F6
:10BC0000CDF804B0FDF71EFE013749F6DE6108EB02
:10BC10004500802FC1F200010880E5D14AF20800FA
:10BC2000C2F2010000680027068B04880FF28859D1
:10BC30004FF4E17A4FF0010B4FF4E478032F17D063
:10BC400007EB470519F807200AEB450080B27D2174
:10BC500033460094CDF804B0FDF7F4FD013749F602
:10BC6000DE6108EB4500802FC1F200010880E5D1BC
:10BC70001FEDC69A00241FE005F13B0080B2882129
:10BC800002468D23CDF80090FDF7C0FAB8B28621A8
:10BC900002468D23CDF80090FDF7B8FA05F13D007E
:10BCA00080B2882102468D23CDF80090FDF7AEFAD0
:10BCB0000F2E04F101041FD2E6B24AF2080000EE92
:10BCC000106AC2F20100B8EE400A006820EE090ACC
:10BCD0001421BDEEC00A082E88BF162130F801904D
:10BCE00010EE105A002E05F13C07C5D014F00100EB
:10BCF000C2D1B8B28921D5E74AF20804C2F20104E0
:10BD000020688D21878A3C204FF495728E230097FE
:10BD1000FDF7DAFF20688D21C78A40F22B104FF41F
:10BD2000E6728E230097FDF7CFFF20689721878A60
:10BD30003C204FF4957298230097FDF7C5FF2068CB
:10BD40009721C78A40F22B104FF4E6729823009790
:10BD5000FDF7BAFF20688221878E0498A0233E3029
:10BD600082B203980097FDF751FA42F61C1042F692
:10BD70003016C1F20000C1F2000680ED008A326880
:10BD80000DF1400A0FF234415046F4F71DFB1DAE91
:10BD900030463221F5F7F3FC30465146F4F777FD93
:10BDA000F4F799FD062809D820243046F4F793FDCE
:10BDB00034523046F4F78FFD0728F6D31DA95046BC
:10BDC000F4F765FD4AF20800C2F2010000680021A4
:10BDD000B0F824B007880524012600254FF000099B
:10BDE0001FE0002A44D0A5EB090000EB400004EB63
:10BDF000400080B2A1215B4600970196FDF722FD2D
:10BE0000681CA0EB090101EB410149F6DE6204EB7D
:10BE10004101C1F200021180AAB281B27F2A054617
:10BE200026D21AF801205E2ADBD101EB0A00407805
:10BE30006F28D8D16E1C6FEA090809F10109A6EB39
:10BE40000901B0B201EB41011AF8002004EB4100F6
:10BE50004FF0010C80B29E215B460097CDF804C0E4
:10BE6000FDF7F0FCA81C00EB080135460126CAE7E7
:10BE700042F61810C1F2000090ED000A9FEDD11AB1
:10BE800042F63011C1F2000120EE010A91ED001AD4
:10BE90009FEDCD2AB8EEC11A21EE021A31EE000A4A
:10BEA00080ED000A91ED001AB8EEC11AB4EE410A15
:10BEB000F1EE10FA05DA91ED000AB8EEC00A80ED55
:10BEC000000A47F2F076C1F2000670780028DDE93A
:10BED000051008BF0146086844F2FF31C0F695011D
:10BEE0000131884262D29FEDC61AB4EE410AF1EEEA
:10BEF00010FA40F3C0809FEDC31AB4EE410AF1EE90
:10BF000010FA40F3C0809FEDC01AB4EE410AF1EE82
:10BF100010FA40F3C0809FEDBD1AB4EE410AF1EE75
:10BF200010FA40F3C0809FEDBA1AB4EE410AF1EE68
:10BF300010FA40F3C0809FEDAD1AB4EE410AF1EE65
:10BF400010FA40F3C0809FEDB31AB4EE410AF1EE4F
:10BF500010FA40F3C0809FEDB01AB4EE410AF1EE42
:10BF600010FA40F3C0809FEDA31AB4EE410AF1EE3F
:10BF700010FA40F3C0809FEDA01AB4EE410AF1EE32
:10BF800010FA40F3C0809FED9D1AB4EE410AF1EE25
:10BF900010FA40F3C0809FEDA11AB4EE410AF1EE11
:10BFA00010FA40F3C080BBEE0C1A55E09FED871AE3
:10BFB000B4EE410AF1EE10FA5DDD9FED851AB4EEA4
:10BFC000410AF1EE10FA5EDD9FED821AB4EE410AED
:10BFD000F1EE10FA5FDD9FED801AB4EE410AF1EE4A
:10BFE00010FA60DD9FED7D1AB4EE410AF1EE10FA11
:10BFF00061DD9FED7B1AB4EE410AF1EE10FA62DDCD
:10C000009FED781AB4EE410AF1EE10FA63DD9FED70
:10C01000761AB4EE410AF1EE10FA64DD9FED731A60
:10C02000B4EE410AF1EE10FA65DD9FED711AB4EE3F
:10C03000410AF1EE10FA66DD9FED6E1AB4EE410A88
:10C04000F1EE10FA67DD9FED6C1AB4EE410AF1EEE5
:10C0500010FA68DD9FED691A3020B4EE410AADF8A0
:10C06000440043F65310F1EE10FACCBFC3F22B603C
:10C07000C3F22B405EE000208DF8420043F25310E3
:10C08000ADF840005BE000208DF8420043F2532001
:10C09000ADF8400053E000208DF8420043F25330E9
:10C0A000ADF840004BE000208DF8420043F25340D1
:10C0B000ADF8400043E000208DF8420043F25350B9
:10C0C000ADF8400037E000208DF8420043F25360A5
:10C0D000ADF840002FE000208DF8420043F253708D
:10C0E000ADF8400027E000208DF8420043F65300F1
:10C0F000ADF840001FE000208DF8420043F65310D9
:10C10000ADF8400017E03020ADF8440043F653107E
:10C11000C3F22B100EE03020ADF8440043F653106C
:10C12000C3F22B2006E03020ADF8440043F6531054
:10C13000C3F22B30109047F2F076C1F200061DAD2D
:10C1400028463221F5F71BFB10A92846F4F79FFB80
:10C15000F4F7C1FB052809D820242846F4F7BBFBD7
:10C160002C522846F4F7B7FB0628F6D310A81DA9D1
:10C17000F4F78DFB4AF20801C2F20101096847F6A3
:10C180002C174B8C0988C0F6030700910C219622CE
:10C190000197FDF739FFFEF7FFBC00BF5300000019
:10C1A00033000000350000003700000039000000B7
:10C1B0002B3230002B3430002B36300025646442A3
:10C1C0006D000000EC51783F8FC2F53C00000AC3BF
:10C1D000000004C30000FCC20000F0C20000E4C282
:10C1E0000000D8C20000CCC20000C0C20000B0C233
:10C1F00000009CC2000088C2000068C2000040C26B
:10C200000000ECC20000E0C20000D4C20000C8C2BE
:10C210000000BCC20000A4C2000098C2000018C206
:10C220005742460046424600554246002DE9F04F2F
:10C2300081B02DED048B88B047F2C171C1F20001CD
:10C240000978002940F0718347F2B471C1F200010E
:10C250000446087848B14BF69470C2F201000121FF
:10C26000002C0CBFC17101725FE34AF20806012085
:10C27000C2F2010608704CB130687D2107880020A9
:10C280004FF4F072A9230097FCF7C0FF4CF21B009B
:10C29000C2F20100007847F6E067002847F69D10DB
:10C2A00047F2F073C0F60307C1F20000C1F20003C9
:10C2B000059419D147F6A611C1F20001097899B980
:10C2C000017889B9597803F12402002908BF03F1E4
:10C2D000080211680A2907D04BF6F871C2F2010171
:10C2E0000968002900F0278301783068838B008873
:10C2F00021B100900FF2A060032105E0009041F20F
:10C300008A00C0F6040004214B220197FDF77CFE51
:10C3100030688D21878A3C20E4228E230097FDF728
:10C32000D3FC30688D21C78AE4204FF4B4728E2389
:10C330000097FDF7C9FC30689721878A3C20E422EA
:10C3400098230097FDF7C0FC30689721C78AE42046
:10C350004FF4B47298230097FDF7B6FC9FEDE58A81
:10C36000002400BFE5B200EE105AB8EE400A20EEFD
:10C37000080A3068BDEEC00A10EE101A1422092D0A
:10C3800088BF1622875A01F13C00E10780B24FF0C6
:10C39000870102464FF08D0308BF82210097FCF70A
:10C3A00035FF102D04F10104DCD3306849F6DE6658
:10C3B000058C048800274FF041094FF0010B4FF026
:10C3C000470AC1F2000600BF042F14D00FF2CC5070
:10C3D00007EB4708C25D09EB480080B27D212B4680
:10C3E0000094CDF804B0FDF72DFA01370AEB4800B0
:10C3F000802F3080E8D14AF20800C2F201000068C4
:10C400000027058C04884FF078094FF0010B4FF09E
:10C410007E0A00BF042F14D00FF2885007EB4708A4
:10C42000C25D09EB480080B27D212B460094CDF817
:10C4300004B0FDF707FA01370AEB4800802F30807F
:10C44000E8D14AF20800C2F2010000680027058C1A
:10C4500004884FF0AF094FF0010B4FF0B50A00BF51
:10C46000042F14D00FF2445007EB4708C25D09EBCC
:10C47000480080B27D212B460094CDF804B0FDF732
:10C48000E1F901370AEB4800802F3080E8D14AF209
:10C490000804C2F2010420688D21878A4FF4B97024
:10C4A0004FF4E6728E230097FDF70EFC206897216B
:10C4B000878A4FF4B9704FF4E67298230097FDF71E
:10C4C00003FC20680027058C048840F277194FF0A0
:10C4D000010B40F27D1A00BF042F14D00FF2D4409C
:10C4E00007EB4708C25D09EB480080B27D212B466F
:10C4F0000094CDF804B0FDF7A5F901370AEB480028
:10C50000802F3080E8D14AF20807C2F2010747F2D3
:10C51000F07B3868C1F2000B9BF80110448A058A51
:10C52000002089B15221252268230094FCF76EFE79
:10C5300040F61E7606A80DF11A0107AAC0F60406F9
:10C54000CDE90021029010E05221252268230094B9
:10C55000FCF75CFE06A80DF11A0107AA40F6F76683
:10C56000CDE900210290C0F6040647F6E06A0DF11D
:10C570001E03304600215222C0F6030ACDF80CA05B
:10C58000FDF700FCBDF81A00BDF81810C0F1250039
:10C5900000EBD0705C2202EB5102C0F34F01304639
:10C5A0002B460094CDF804A0FDF72EFD9BF801006A
:10C5B0000BF12408002840460BF1080408BF204670
:10C5C0003A6800680FF2F431B2F8009051F8206038
:10C5D000158F40F2A110532140F2D1126923CDF8FA
:10C5E000009040F2A117FCF711FE06A80DF11A0108
:10C5F00007AACDE9002102900DF11E03304640F25A
:10C60000A1115322CDF80CA0FDF7BCFBBDF81A0018
:10C61000BDF81810C0F1300000EBD07007EB5000EF
:10C620005D2202EB5102CDF800904AF2080981B276
:10C6300030462B46C2F20109CDF804A0FDF7E4FC18
:10C64000D9F800001921078840F2811040F2DB126E
:10C6500032230097FCF7DAFDD9F800001921B0F871
:10C6600060704FF4C87040F2CD1219230097FCF7A8
:10C67000CDFDD9F800003221B0F8607040F2811091
:10C6800040F2DB1232230097FCF7C0FDD9F800001E
:10C690003221B0F860704FF4C3704FF4C8721923A0
:10C6A0000097FDF783FAD9F800003221B0F86070E6
:10C6B0004FF4EB704FF4E67219230097FDF776FA0A
:10C6C0009BF801009FEDC91A002808BFA046D8F8C2
:10C6D0000000B7EE008A082800F27980B0EE410A27
:10C6E000B0EE482ADFE800F0081F364D6477691283
:10C6F000290000BF00009641BBF872019FEDC02ADF
:10C7000000EE100AB8EE400A20EE020ABBF87001F3
:10C710009FEDBB3A02EE100AB8EE422A22EE032A3F
:10C72000B0EE418A57E0BBF872019FEDB52A00EEEA
:10C73000100AB8EE400A20EE020ABBF870019FED25
:10C74000B03A02EE100AB8EE422A22EE038AB0EEA8
:10C75000412A40E0BBF86E019FEDA81A00EE100AD6
:10C76000BBF86C01B8EE400A20EE010A01EE100A97
:10C770009FEDA12AB8EE411A9FED9C8A21EE022A74
:10C7800029E0BBF86C019FED9C1A00EE100ABBF883
:10C790006E01B8EE400A20EE018A00EE100A9FED0D
:10C7A000971AB8EE400A9FED912A20EE010A12E096
:10C7B000BBF876019FED8F2A03E0BBF874019FED73
:10C7C0008C2A00EE100AB8EE400A20EE028AB0EE83
:10C7D000410AB0EE482AB3EE0E9A22EE091ABDEED7
:10C7E000C11A20EE090A11EE107ABDEEC00A10EE51
:10C7F000108A87B3D9F80000C7F5D771B0F8644044
:10C80000C8F5D7708EB285B230461A212A46312338
:10C810000094FCF7FBFCD9F8000040F2A511B0F839
:10C820006440C81B80B2312132461A23009601941D
:10C83000FCF7B6FDB8F1000F0DD0D9F800001A21B1
:10C84000B0F864704FF4D770009028462A46312320
:10C850000197FCF7A5FDB5EE408AF1EE10FA35DD43
:10C8600028EE090ABDEEC00AD9F8000010EE104A01
:10C8700008F5D771B0F8647004F5D7708DB286B240
:10C8800028461A21324631230097FCF7BFFCD9F81D
:10C8900000003121B0F8647004F2B71080B2324663
:10C8A0001A2300960197FCF77BFDB8F1000F0DD01D
:10C8B000D9F800001A21B0F864704FF4D7700090D6
:10C8C00028462A4631230197FCF76AFD4BF6A471EE
:10C8D000C2F201010A789BF83731002A104618BFCE
:10C8E0004FF4D770002B11BF002A012008704FF4BD
:10C8F000D770D9F80010431EB1F86270821C98B24C
:10C90000252131230097FCF781FC059A4BF69471A1
:10C91000002A47F2B472C2F201014FF00000C1F2E6
:10C920000002C87118BF0872107008B0BDEC048B0B
:10C9300001B0BDE8F08F4BF69470C2F20100012106
:10C94000417230680321438B00884B22009011A074
:10C950000197FDF759FB306840F6BC558389008884
:10C9600043F2A024C0F60405C0F603040090284654
:10C97000972174220194FDF747FB306840F21D11A6
:10C98000C38900887422009028460194FDF73CFB7F
:10C99000B9E500BF52580000545500005357523AB1
:10C9A000000000004657443A000000005245463A55
:10C9B00000000000414C433A00000000FF0E040854
:10C9C000030F04088C0F0408691004089C0F040866
:10C9D000A00F0408990F0408910F04086E100408B2
:10C9E00004100408FF0F0408881004080000000069
:10C9F00017B7D13817B751386F12833ACD339A3AF7
:10CA0000CD339A392DE9F04F97B047F2C171C1F299
:10CA10000001097811B117B0BDE8F08F47F2B47189
:10CA2000C1F200010A7842B14BF69470C2F20100E3
:10CA30000121417017B0BDE8F08F4AF208040122CD
:10CA4000C2F201040A70049048B1206801210788ED
:10CA5000002040F2DF1233230097FCF7D7FB47F2A8
:10CA6000F0772068C1F2000797F88E11021D048943
:10CA7000002908BF821D1588022001214022292398
:10CA800000944FF00209FCF7C1FB40F63D7647F6F3
:10CA9000E0680DF1560116AA0DF15A00C0F6040621
:10CAA000C0F60308CDE90002029105AB3046022131
:10CAB0000122CDF80C80FDF765F9BDF85800BDF8EE
:10CAC0005610C0F13E0000EBD07009EB500014226C
:10CAD00002EB510281B230462B460094CDF804801F
:10CAE000FDF792FA05AD28464021F4F748FE97ED90
:10CAF0004C0A0FF2CC41BDEEC00A10EE102A2846B7
:10CB0000F3F762FCD7F830012923400002BF45F259
:10CB10004140C0F2540005904AF20800C2F2010000
:10CB2000006897F83511021D0489002908BF821D8D
:10CB3000158842200121802200944FF0420AFCF720
:10CB400065FB16A805AE0DF1540900900DF1560BCA
:10CB50000DF15A03304642210122CDE901B9CDF849
:10CB60000C80FDF70FF9BDF85600BDF85410C0F168
:10CB70003E0000EBD0700AEB5000142202EB510291
:10CB800081B230462B460094CDF80480FDF73CFA84
:10CB90004AF20800C2F20100006897F83C10021D3A
:10CBA0000489002908BF821D1588C22001214FF485
:10CBB000807229230094C227FCF728FB41F2640607
:10CBC000C0F604060DF1580A0DF15A033046C22191
:10CBD0000122CDE900ABCDF80890CDF80C80FDF72F
:10CBE000D1F8BDF85600BDF85410C0F13E0000EB7E
:10CBF000D07007EB5000142202EB510281B2304694
:10CC00002B460094CDF80480FDF7FEF94AF20800A7
:10CC100047F2F073C2F20100C1F2000300685978D4
:10CC200003F138020489002908BF03F11C021178BE
:10CC3000021D002908BF821D158882200121C02203
:10CC4000292300948227FCF7E1FA40F62076C0F60B
:10CC500004060DF15A03304682210122CDE900ABD2
:10CC6000CDF80890CDF80C80FDF78CF8BDF8560093
:10CC7000BDF85410C0F13E0000EBD07007EB50003F
:10CC8000142202EB510281B230462B460094CDF8BB
:10CC90000480FDF7B9F94AF20807C2F201073868C3
:10CCA0004BF6FC71C2F2010104890978021D0029CA
:10CCB00008BF821D15884FF4817001214FF4A072C6
:10CCC000292300944FF4817AFCF7A0FA40F65076BD
:10CCD0000DF1580B0DF15600C0F60406CDF800B06A
:10CCE000CDE901090DF15A0330464FF4817101225B
:10CCF000CDF80C80FDF746F8BDF85600BDF854108D
:10CD0000C0F13E0000EBD0700AEB5000142202EBA1
:10CD1000510281B230462B460094CDF80480FDF7D5
:10CD200073F9386801210489C68847F2F070C1F2AE
:10CD3000000090F846714FF4A1704FF4C07229239F
:10CD400000944FF4A179FCF761FA40F6877515A8B5
:10CD5000C0F604050DF1560A02900DF15A0328465B
:10CD60004FF4A1710122CDF800B0CDF804A0CDF8A8
:10CD70000C80FDF707F8BDF85600BDF854101422DA
:10CD8000C0F13E0002EB51024FF6000100EBD07003
:10CD9000CFF6FF7109EB5000002F08BF31468BB270
:10CDA00081B228460094CDF80480FDF72DF94AF2AF
:10CDB00008074AF2B029C2F20107C2F20109386835
:10CDC000D9F800100489B0F85C5001F10A0600207F
:10CDD00040F22311762240F241130094FCF716FA38
:10CDE000CDF800B0D346CDF804A00DF1540A0DF1F2
:10CDF0005A033046002140F22312CDF808A0CDF8A6
:10CE00000C80FCF7BFFFBDF85600BDF85410C0F110
:10CE1000760000EBD07040F2311202EB5102C0F309
:10CE20004F0130462B460094CDF80480FDF7ECF816
:10CE30003868D9F800100489B0F85C5001F12E066A
:10CE4000782040F22311EE2240F24113009478271B
:10CE5000FCF7DCF916A8CDE9000B0DF15A033046BA
:10CE6000782140F22312CDF808A0CDF80C80FCF711
:10CE700089FFBDF85600BDF85410C0F1760000EBF4
:10CE8000D07007EB500040F2311202EB510281B238
:10CE900030462B460094CDF80480FDF7B5F84AF2F1
:10CEA0000800C2F201000068D9F800100489B0F847
:10CEB0005C5001F15206F02040F223114FF4B3729E
:10CEC00040F241130094F027FCF7A0F916A8CDE931
:10CED000000B0DF15A033046F02140F22312CDF839
:10CEE00008A0CDF80C80FCF74DFFBDF85600BDF84A
:10CEF0005410C0F1760000EBD07007EB500040F208
:10CF0000311B0BEB510281B230462B460094CDF819
:10CF10000480FDF779F84AF20800C2F201004AF2F3
:10CF2000B0210068C2F2010109680489B0F85C50C0
:10CF300001F176064FF4B47040F223114FF4EF7212
:10CF400040F2411300944FF4B477FCF75FF916A850
:10CF500000900DF15600CDE9010A0DF15A0330465B
:10CF60004FF4B47140F22312CDF80C80FCF70AFFA5
:10CF7000BDF85600BDF85410C0F1760000EBD0703B
:10CF800007EB50000BEB510281B230462B46009468
:10CF9000CDF80480FDF738F804994BF69470C2F28E
:10CFA000010000294FF00001417018BF817047F265
:10CFB000B470C1F20000017017B0BDE8F08F00BF7F
:10CFC00041545425640000002DE9F04F87B047F22A
:10CFD000B475C1F20005287810B107B0BDE8F08F34
:10CFE0004BF69477C2F20107387860B101202870BF
:10CFF0004AF20800C2F2010000680088FBF7DAFF7D
:10D00000002038702870787810B10020FFF7FAFC03
:10D01000B87810B10120FFF7F5FCF87847F2C17439
:10D02000C1F2000458B1207848B9287810B1012025
:10D03000F87004E0012028700020F870287038791A
:10D0400060B1207850B9287810B10120F87005E05F
:10D05000012028700020F87038712870787910B19C
:10D060000020FDF78DF9B87910B10120FDF788F99E
:10D07000F87910B10020FFF7D9F8387A10B1012003
:10D08000FFF7D4F8787A10B10020FDF7F5FAB87AF6
:10D0900010B10120FDF7F0FAF87A10B1002006F087
:10D0A0004DFE387B10B1012006F048FE787B78B346
:10D0B00049F6DB60C1F2000001784FF2F100CFF2D7
:10D0C000F000A1FB0002100900EB00100A1AC0B228
:10D0D0004DF2D443C2F20103081A1A7000EBC000EB
:10D0E000052202EB40034AF21440C2F2010002683A
:10D0F000080110584AF2184602EB0112C2F201066A
:10D10000117992683380012316F08CF9002078732E
:10D11000B87B00283FF461AF0120B873287800285D
:10D120007FF45BAF207820B10020B87307B0BDE872
:10D13000F08F012042F2E8762870C0F6030605A8B9
:10D140000DF1160106AACDE90021CDE9020647F648
:10D15000B010C1F200000DF11A03F0214622F024B4
:10D16000FCF710FE4CF21D0AC2F2010A9AF80010F8
:10D17000BDF81600012904D1BDF814904FEA500BF8
:10D1800032E04AF20802C2F20102A4EB5001126836
:10D19000BDF814904FEA500B0844B2F84AC00A3068
:10D1A00009F150028CB21FFA80F896B2204646214F
:10D1B00042463346CDF800C0FCF728F84AF2080092
:10D1C000C2F2010000684621B0F84CC02046424639
:10D1D000334642F2E876C0F60306CDF800C0FCF70D
:10D1E00073FD01208AF800004AF20800C2F2010033
:10D1F0000068CBF1F501B0F84830B0F84A0009F109
:10D200004B02009047F6B01089B292B2C1F2000012
:10D210000196FCF7F9FE002049F6EC6147F6AC12E6
:10D220002870C1F20001C1F2000209681268891A6F
:10D23000B1F57A7F82BFB8730120B87107B0BDE83D
:10D24000F08F00002DE9F04387B04BF6B476C2F2C0
:10D25000010632780C460546C2BB47F2F070C1F2B7
:10D26000000090F8850142F27C31C0F6030166228D
:10D270004AF2080710FB0210C2F201073860FCF7FF
:10D2800071F94FF0C040362101800020C6F208003D
:10D290002821018049F6EC60C1F20000016800BF5E
:10D2A0000268521A792A0BD20268521A782A07D8D1
:10D2B0000268521A782A03D80268521A792AEFD3E0
:10D2C00038680088FBF776FE0120307047F2B478AA
:10D2D000C1F20008012088F800004FF478404FF4B4
:10D2E0007846FBF767FE42F2E877C0F6030705A829
:10D2F0000DF1160106AACDE90021CDE902070DF1D5
:10D300001A032846002100224FF00009FCF73AFDDD
:10D31000BDF81600F021A1EB5000BDF81410A022BA
:10D32000A2EB510281B292B228464FF6FF730096EB
:10D330000197FCF769FE002C57D049F6EC60C1F26A
:10D34000000001680268521AB2F5FA6F0ED802683E
:10D35000521AB2F5FA6F09D80268521AB2F5FA6F8A
:10D3600004D80268521AB2F5FA6FEBD94BF69471F1
:10D370000020C2F20101012288F800000A708A71BF
:10D380008A720A728A700A71CA7242F61C11C1F25C
:10D39000000108604BF6B871C2F20101086042F664
:10D3A0002410C1F20000FF2101704AF26A00C2F2AB
:10D3B0000100017042F62510C1F20000017042F632
:10D3C0002210C1F2000042F20F7101804AF268009F
:10D3D000C2F20100018042F62010C1F2000001807B
:10D3E000FFF7F2FD07B0BDE8F08388F8009007B0C2
:10D3F000BDE8F0832DE9F04F83B04AF26D55C2F2DB
:10D400000105297840F200430646C4F2020371B9CF
:10D410004FF48050009042F626100027C1F2000021
:10D4200000210122019702F01DFFF5F76FF942F686
:10D430002C2BC1F2000B002458462021002201238E
:10D440000094F5F797F880BB42F62C20C1F200005B
:10D450002021002201230094F5F78CF828BB42F626
:10D460002C200024C1F2000020210022012300947E
:10D47000F5F780F8C8B942F62C20C1F2000020214F
:10D48000002201230094F5F775F870B942F62C20BC
:10D490000027C1F200002021002201230097F5F7A8
:10D4A00069F810B9AEA01AF09DFC9BF81D00642825
:10D4B00062D19BF8000064285ED1002E5CD19BF8FD
:10D4C00001009BF802109BF8032008449BF804100D
:10D4D00010449BF8052008449BF8061010449BF864
:10D4E000072008449BF8081010449BF809200844C2
:10D4F0009BF80A1010449BF80B2008449BF80C1072
:10D5000010449BF80D2008449BF80E1010449BF823
:10D510000F2008449BF8101010449BF81120084479
:10D520009BF8121010449BF8132008449BF8141029
:10D5300010449BF8152008449BF8161010449BF8E3
:10D54000172008449BF8181010449BF81920084431
:10D550009BF81A1010449BF81B2008449BF81E10DF
:10D5600010449BF81F20084410449BF81C103838C6
:10D57000C0B2814200F0DE8048F21864C1F20004BB
:10D58000208848F218554CF27828029600277FA68A
:10D59000C1F20005C2F201084FF000090BE000BF24
:10D5A00081B2B1F5807F09F1010924BF00202080FC
:10D5B000B9F11B0F1BD016F8091082B2A954013023
:10D5C000B8F8001082B28A422080E9D14FF0000AF8
:10D5D000F4F720FCB7EB5A2F03D101280AF1010A16
:10D5E000F6D0F4F717FC012801D02088D8E79BF883
:10D5F0001D0000211AF02EFD9BF8000000211AF0FA
:10D6000029FD6420002164241AF024FD02980021E1
:10D610001AF020FD9BF81C0000211AF01BFD9BF85E
:10D6200000009BF801109BF802209BF8033008448F
:10D6300010449BF80410184408449BF805109BF80C
:10D64000062008449BF8071010449BF80820084463
:10D650009BF8091010449BF80A2008449BF80B1013
:10D6600010449BF80C2008449BF80D1010449BF8C4
:10D670000E2008449BF80F1010449BF8102008441B
:10D680009BF8111010449BF8122008449BF81310CB
:10D6900010449BF8142008449BF8151010449BF884
:10D6A000162008449BF8171010449BF818200844D3
:10D6B0009BF8191010449BF81A2008449BF81B1083
:10D6C00010449BF81D2008449BF81E1010449BF842
:10D6D0001F2008441044C0B200211AF0BBFC642093
:10D6E000C0F2010041F6321141F61A32C4F600616F
:10D6F000C2F61A028BE8070041F62D20ABF80C00A9
:10D7000050208BF80E004FF6F370ABF8100000209D
:10D710000021C4F23010C4F22011CBE9050122A08F
:10D720008BF81D401AF05EFB06F082FD4AF26D5543
:10D73000C2F20105287880B94FF4805000904AF277
:10D74000453040F200430027C2F2010000210122CF
:10D75000C4F20203019702F085FD03B0BDE8F08F2B
:10D760005B4552525D205265616420454550524FE1
:10D770004D2043414C494252415445206D756C74D3
:10D7800069706C65206572726F7273005B455252EE
:10D790005D2043414C49425241544520466C6173DF
:10D7A0006820636865636B005B4F4B5D204C6F6165
:10D7B0006465642064656661756C742063616C697E
:10D7C00062726174652073657474696E67730000BA
:10D7D0002DE9F04F81B04CF22026C2F201063078DC
:10D7E000012840F08E814CF24064C2F20104D4F86A
:10D7F000040301254168204684F8EC528847D4F898
:10D80000207397F8BC03012800F07B81396887F802
:10D81000BC53886840F6445220F001008860D1F87B
:10D82000000EC0F2030220F00300C1F8000ED1F890
:10D83000040840F00200C1F804084FF48460086155
:10D84000104604380CD00B699B0609D50B699B0662
:10D8500044BF0B695FEA836302D50B699B06F0D472
:10D86000B86A012806D1B869012803D0886B20F472
:10D87000803088630020032387F8BC0387F8BD331A
:10D880004FF67F33C1F80839C1F8083BC1F8283991
:10D89000C1F8283BC1F84839C1F8483BC1F868399C
:10D8A000C1F8683BC1F88839C1F8883BC1F8A8398C
:10D8B000C1F8A83BC1F8C839C1F8C83BC1F8E8397C
:10D8C000C1F8E83BC1F8083AC1F8083CC1F8283A69
:10D8D000C1F8283CC1F8483AC1F8483CC1F8683A58
:10D8E000C1F8683CC1F8883AC1F8883CC1F8A83A48
:10D8F000C1F8A83CC1F8C83AC1F8C83CC1F8100842
:10D90000C1F81408C1F81C0810200861104600BFB7
:10D91000043800F0F4800B69DB0641BF0B695FEA55
:10D92000C3630B695FEAC36302D50B69DB06EFD4FF
:10D930004FF484600861043A00F0E18008698006D1
:10D9400009D50869800644BF08695FEA806002D58E
:10D9500008698006EFD43868B0F1A04F40F0088124
:10D9600043F634000097C4F20200026843F6004117
:10D9700040F20009C4F2010122F08002C4F202095F
:10D98000026000244FF0010CA1F57E7B4FF00F0EDA
:10D99000002200204FF00F0A31E000BF911CD9F89F
:10D9A0000030032707FA01F16FF003078B4307EA02
:10D9B0005000C9F8003048440CF01C03076A0AFA0A
:10D9C00003F327EA03030362D9F80C004FF0010CBC
:10D9D0008843C9F80C00D9F804004FF00F0E00EA94
:10D9E0000800C9F80400D9F808008843C9F80800FD
:10D9F000681C0432102804F1080400F0AA800CFA14
:10DA000000F515F4C05F47D087085BF8276004F085
:10DA100008030EFA03F31E426FEA050519D143F617
:10DA20000041C4F201010E682E400E604E682E4087
:10DA30004E608E682E408E6043F60C41C4F20101A8
:10DA40000E682E400E605BF8276026EA03034BF851
:10DA50002730D9F80030032101FA02F76FF00301F3
:10DA6000BB4301EA5006C9F800304E4404F01803E5
:10DA7000316A0EFA03F399433162D9F80C10B943B5
:10DA8000C9F80C10D9F804102940C9F80410D9F8C5
:10DA90000810B943C9F80810451C0CFA05F717F42B
:10DAA000C05FA5D04FEA900E04F1040C5BF82E1075
:10DAB0000CF00C030AFA03F319426FEA07087FF42B
:10DAC0006DAF43F60046C4F20106316801EA080171
:10DAD0003160716801EA08017160B16801EA08010A
:10DAE000B16043F60C46C4F20106316801EA080150
:10DAF00031605BF82E1099434BF82E104EE7002052
:10DB000030704CF6D430C2F2010090F8BC130129F9
:10DB10001CD00168012280F8BC23D1F8002E22F02D
:10DB20000302C1F8002ED1F8042842F00202C1F825
:10DB30000428826A012A06D18269012A03D08A6BED
:10DB400022F480328A63002180F8BC1301B0BDE862
:10DB5000F08F4EF28810CEF2000008210160BFF372
:10DB60004F8FBFF36F8F4CF22026009FC2F2010649
:10DB7000002087F8BD03307001B0BDE8F08F0000D1
:10DB80004AF22850C2F201000178012919D100217E
:10DB9000017041F204004AF22452CEF20000C2F2B7
:10DBA000010242F6702301681268C1F200031F6887
:10DBB000891A39441960006842F67421C1F20001E3
:10DBC00008604EF2FF0547F2C47640F21847C0F2F3
:10DBD000F5550FF22C08C1F20006C4F202074FF40B
:10DBE000800400E03C6040460021FFF72BFB00BFB3
:10DBF0003068A842F6D20130306000BFF8E700BFBD
:10DC00004D656D6F7279204661756C74000000007F
:10DC10002DE9F0412DED108B47F2F070C1F20000BC
:10DC2000417800F12C02002908BF00F110021168B0
:10DC30004AF26C00B1F5FA5FC2F2010012DB42F267
:10DC40000F7291421ADD42F2107291422BD043F6CC
:10DC5000982291422AD044F62062914238D19FED19
:10DC6000AC0A33E041F26F72914211DC09B341F228
:10DC7000883291422CD19FEDA40A27E0B1F5FA5FDA
:10DC80001FD042F22832914222D19FEDA40A1DE01A
:10DC900041F27072914217D041F65832914217D139
:10DCA0009FEDA00A12E09FED9C0A0FE09FED990AFC
:10DCB0000CE04CF600019FED950AC4F22F71016053
:10DCC00008E09FED970A01E09FED970A80ED000ABA
:10DCD00090ED000A47F2D87047F2CC7C4BF6C87E34
:10DCE00047F2C878C1F20000C1F2000CC2F2010E86
:10DCF000C1F2000890ED001A9CED00BA9EED002ADA
:10DD000098ED00CA41F200509FED883A9FED884A95
:10DD10009FED885A9FED886A9FED887ADFED880A2B
:10DD2000DFED881ADFED882ADFED883ADFED884ADB
:10DD300040F2884141F20024DFED865ADFED866A29
:10DD4000DFED867A9FED868A9FED869A0023C2F2E8
:10DD50000000C0F60401C2F200040025B5EE00AADE
:10DD600077E000BF2CEE26DA2DEE00DA2DEE27DA72
:10DD7000BDEECDEA1EEE107AB5EE40DAF1EE10FA05
:10DD8000B8BF013F0EEE107AB8EECEEA3DEE4EEA95
:10DD90002EEE08EABDEECEFA1FEE107AB3EB572F47
:10DDA0003EEE09FA1CBFB0EE4FEA002701EB8702F6
:10DDB0000FEE107AD2ED008AD2ED019AB8EE4FFA4A
:10DDC0003EEE4FEA39EEE8FA2FEE0EEA3EEE28EA92
:10DDD0002EEE01EA3DEE0ADA86ED00EABDEECDEA6E
:10DDE0001EEE102AB5EE40DAF1EE10FAB8BF013A95
:10DDF0000EEE102AB8EECEEA3DEE4EDA2DEE08DA3F
:10DE0000BDEECDEA1EEE102AB3EB522F3DEE09EA2D
:10DE10001CBFB0EE4EDA002201EB82060EEE102A95
:10DE200096ED00FAD6ED018AB8EE4EEA3DEE4EDAF6
:10DE300038EECFEA2EEE0DDA3DEE0FDA04EB850276
:10DE400001352DEE01DAC02D2BEE03BA82ED00DA9A
:10DE500050D000EB8506B0EE42DA96ED002A2CEEAB
:10DE600004CA32EE0BBA3BEE4DBA2BEE05DA3CEEAD
:10DE70000DDAB4EE46DAF1EE10FAB0EE4DCA19DD65
:10DE80003CEE07DAB4EE46DAF1EE10FA12DD3CEEC3
:10DE900020DAB4EE46DAF1EE10FA0BDD3CEE21DAD0
:10DEA000B4EE46DAF1EE10FA04DD3CEE22DAE0E7F9
:10DEB0003DEE25DAB4EE47DAF1EE10FAB0EE4DCAD7
:10DEC000BFF650AF3DEE06CAB4EE47CAF1EE10FA07
:10DED000BFF648AF3DEE23CAB4EE47CAF1EE10FAE2
:10DEE000BFF640AF3DEE24CAB4EE47CAF1EE10FAD9
:10DEF000DEDB37E78CED00BA8EED002A88ED00CA34
:10DF0000BDEC108BBDE8F08100007A4500C82F47BA
:10DF100000401C470060EA4600606A4600204B460D
:10DF200000E02B460000FA450080BB453333733FC9
:10DF30000012833AF1F4723F00803B4700803BC7F8
:10DF40000080BBC700A00CC800803BC80080BB4756
:10DF500000A00C4800803B481F42893883F9223ECC
:10DF600000000044000000C44AF22850C2F2010040
:10DF70000178012918BF7047002141F2040C4AF2D0
:10DF800024520170CEF2000CC2F2010242F670235C
:10DF9000DCF800101268C1F200031868891A0844FE
:10DFA0001860DCF8000042F67421C1F2000108603C
:10DFB000704700002DE9F04F89B04AF22850C2F2B4
:10DFC00001000178012919D10021017041F20400FA
:10DFD0004AF22452CEF20000C2F2010242F670234D
:10DFE00001681268C1F200031F68891A3944196078
:10DFF000006842F67421C1F2000108604CF6D43684
:10E00000C2F20106D6F80080D8F81400C00741F02B
:10E010002E83D8F81400D8F81810014201F0278395
:10E02000D8F81400D8F818100840800705D5D8F89B
:10E03000140000F00200C8F81400D8F81400D8F852
:10E0400018100840C0067DD5D8F8180020F0100040
:10E05000C8F81800D8F82000C0F34342062A00F0A0
:10E060000F0154D0022A67D147F6F072024063D004
:10E07000C1EBC10006EB80000323D0F8086203EB7C
:10E080001215002300F5027CB3EB950F4FEA121333
:10E0900030D0AA08541E02F00307032C324617D3CF
:10E0A0006FF0030202EA950255424FF48054324663
:10E0B00058F804100435116058F80410516058F8ED
:10E0C0000410916058F80410D16002F11002EFD1F1
:10E0D00087B14FF4805558F80510012F116009D011
:10E0E00058F80510022F516004D04FF4805158F8B1
:10E0F00001109160D0F81422F118CCF80010D1185A
:10E100004CF6D436C0F81412C2F2010614E04FF4F3
:10E11000805258F80230C1EBC101C6F8C43358F838
:10E12000022006EB8101C6F8C823D1F81422C0F3FF
:10E130000A101044C1F81402D8F8180040F010007A
:10E14000C8F81800D8F81400D8F81810CDF81880BE
:10E1500008400003404640F17986D8F81808D8F8FE
:10E160001C184FF0000E0840BEEB104F00F06D86FB
:10E1700043F20A0B070C06F505754FF43069C4F637
:10E18000547B4FF0000A3CE0C0F810EBD0F8101BB5
:10E1900041F40021C0F8101BD0F8101B41F0180109
:10E1A000C0F8101BD0F8101B41F0C041C0F8101B84
:10E1B00006F57171C0F8141BD0F8001B41F08021E6
:10E1C000C0F8001BE00642BF08EB09001021816087
:10E1D000A00642BF08EB090020218160A00442BFD5
:10E1E00008EB09004FF4005181600AF1010ABEEB0F
:10E1F000570F4FEA570709F1200905F11C0500F0F8
:10E200002286F807F1D0306809EB00018A68D0F85F
:10E21000143803EA0204E20762D12007D2D540464F
:10E220004844082102970594039581603068D046E0
:10E23000D0F840E048448168090404D5DE4584BF35
:10E240004FF400418160D6F804A496F8C4530AF54F
:10E250003E748AF8F85296F8C53301948AF8F93278
:10E2600096F8C67396F8C70305F01F0447EA002C1A
:10E27000AAF8FAC296F8C81396F8C923022C41EA04
:10E280000220AAF8FC02B6F8CA234FF00106AAF849
:10E29000FE22CAF8E462CDF81CA0CAF8E822CDF844
:10E2A00010E05AD0012C6BD0002CC24640F0B08058
:10E2B00015F0600100F014814CF6D436DDE90684D7
:10E2C000029F4029C2F2010602D0202940F040817D
:10E2D000D4F80403019982682046904740E100BFCA
:10E2E00008EB090201239360036C8A683669012EEA
:10E2F00019D1160700F19C80960600F1D5804CF6E6
:10E30000D43612F0280FC2F201067FF486AF0BF16B
:10E310000106B342C0F0528112F4004200F04E8177
:10E320004FF40040C1E00BF58076B34240F091809D
:10E330004CF6D4361004C2F2010600F18680900635
:10E3400044BF202088605FFA8AF0F9F77FFC4FF025
:10E35000000E20077FF536AF61E715F0600600F08C
:10E360000381069C029F402EC24602D0202E40F020
:10E3700013810798D0F804138A680199904714E133
:10E380004CF6D436029F15F06000C2F20106C24678
:10E3900018BF402840F09280079C94F8EC020138A6
:10E3A000022800F28F80039DDDF81880082900F212
:10E3B0007681079C0199D4F804038268204690472F
:10E3C0004CF6D43600284FF0000EC2F2010640F0A1
:10E3D0007581B4F8FE02002840F07081D4F8200363
:10E3E0000421C4F8E41201464FF4807221F83C2F56
:10E3F0000269C0F848E0C0F850E0012AC0F854E0D3
:10E4000008BFC0F84CE00068D2B211F0C3FC4FE185
:10E41000079805F0800110F0B1FB4CF6D436DDF81A
:10E420001880C2F201064FF0000E039D029F45E1E5
:10E430000BF101004CF6D4368342C2F20106FFF420
:10E44000ECAE12F400403FF4E8AE4FF400408860B8
:10E45000E3E64CF6D436C2F20106D6F8101251EAC1
:10E460000A011AD1016C594503D9D0F8001B0029C3
:10E4700013D4C0F810EBD0F8101B41F40021C0F801
:10E48000101BD0F8101B41F01801C0F8101BD0F879
:10E49000101B41F0C041C0F8101B5FFA8AF0F9F779
:10E4A000D5FB4FF0000E01E0202088604CF6D436FA
:10E4B000C2F2010620077FF585AEB0E620283FF4C2
:10E4C0006BAF079C2046802110F058FB20460021AE
:10E4D00010F054FB039DDDF818804FF0000EEDE0C6
:10E4E000092B4FF0000E00F21B81DFE813F00A0049
:10E4F000FB0019012B01190150016C0119018C015C
:10E50000B501079C039D94F8EC020138022800F243
:10E51000AD814CF6D436DDF81880029F022AC2F293
:10E52000010640F0A982079C0223D4F8F4024FF4BC
:10E53000807200284FF0030008BF012044F80C0F40
:10E54000D4F81403C4F8D83201462361636178E13A
:10E550002046802110F012FB2046002110F00EFB17
:10E56000039D4FF0000EA9E0069C029F002B4FF088
:10E57000000EC2465DD0039D012B00F08280032B6C
:10E58000A04640F08C80079890F8EC32032B00F006
:10E590007E81022B7ED082E0079D8021284610F0EC
:10E5A000EDFA2846002110F0E9FA4CF6D436039D26
:10E5B000C2F201064FF0000EA0467FE0096955E95E
:10E5C00004236FF3DF41511A296099184CF6D436B1
:10E5D00045F80C1CC2F20106D6F8101251EA0A01E5
:10E5E0007FF4B1AE016C594504D9D0F8001B002965
:10E5F0003FF5A9AEC0F810EBD0F8101B41F4002194
:10E60000C0F8101BD0F8101B41F01801C0F8101B07
:10E61000D0F8101B41F0C041C0F8101B06F5717115
:10E62000C0F8141BD0F8001B41F08021C0F8001B7B
:10E6300089E607984CF6D43690F8EC02039D03283F
:10E64000C2F2010600F04C810228A04640F014827C
:10E6500041F08000802840F00F8201F07F00079B8E
:10E6600000EB400003EBC00202F114004FF0020C7B
:10E67000090658BF02F5BE70C0F800E0C3F8E4C256
:10E68000E4E10798A04690F8EC22032A00F05181BB
:10E69000022A04D141F08000802840F08B81079C41
:10E6A0002046802110F06AFA2046002110F066FA18
:10E6B0004CF6D4364FF0000EC2F201060498059CC9
:10E6C00058457FF67FAD306901287FF47BAD306817
:10E6D000016C59457FF658ADD0F8001B00297FF535
:10E6E00053AD6FE5079C039D94F8EC1201390229A4
:10E6F00000F2BC801FFA8CF04CF6D436DDF818809E
:10E70000029F0128C2F20106D8D1D4F820030421C7
:10E71000C4F8E41201464FF48072C4F8F4E228E031
:10E72000079C8021204610F029FA2046002110F095
:10E7300025FA4CF6D436DDF818804FF0000EC2F200
:10E74000010672E61FFA8CF04CF6D436DDE906823B
:10E75000DDE902750128C2F20106AFD10120C2F83D
:10E76000F402D2F820030421C2F8E41201464FF467
:10E77000807221F83C2F0269C0F848E0C0F850E0F0
:10E78000012AC0F854E008BFC0F84CE053E340EA67
:10E790000201039D090468D11FFA8CF07F2864D818
:10E7A000079C4CF6D43694F8EC02C2F2010603281A
:10E7B00040F007812046802110F0E0F9204600213A
:10E7C00010F0DCF9C3E10798ADF822E0B0F8FA02E6
:10E7D0004FF0FF3101EB1021039D062945D8DFE8FA
:10E7E00011F0070057016901440044007F018901CD
:10E7F0000798D0F8000301680DF122008847DDF882
:10E800001880029FA6E2039D012A2ED1079C4CF698
:10E81000D43694F8EC02DDF81880411E029F0229DC
:10E82000C2F2010680F0098144F808EF0220C4F822
:10E83000DC02D4F81803012301464FF480726361AF
:10E84000A36121F83C2F026984640365012AC0F8A2
:10E8500054E008BFC464EEE247F6F010039D022FB7
:10E86000C1F200000770C0F08480079C2046802120
:10E8700010F084F92046002110F080F94CF6D436CF
:10E88000DDF818804FF0000EC2F20106CEE55FEA17
:10E890000C4007D141F08000802803D012B90798BE
:10E8A00010F06CF9079A0421D2F82003C2F8E412A0
:10E8B00001464FF4807221F83C2F026900238364E3
:10E8C0000365012A436508BFC3640068D2B211F032
:10E8D00061FA0798D0F804138A6801999047E7E62F
:10E8E00001F00F00A046079C00EB400011F08003F0
:10E8F00004EBC00014BF8069D0F8800100283FF409
:10E90000CFAE01F07F0606EB460004EBC00202F139
:10E910001400002B41F0800108BF02F5BE70802971
:10E9200040F01A81D4F820C34CF6D436C0F800E089
:10E9300028E15FEA0C4007984CF6D436C2F2010693
:10E940007FF4BCAED0F820034A0600F0C8814368CB
:10E9500001F00F029A4200F2C281090600F18A8199
:10E96000C2EBC20100EB810303F5FE7183F8FDE108
:10E970008DE107984CF6D43690F8EC02C2F201060D
:10E98000032800F0C780022840F0D380002F00F059
:10E990001381079C0321D4F804036760002884F8DE
:10E9A000EC123FF407AF01682046884700287FF447
:10E9B00001AF1DE1079C204610F0E0F820468021C1
:10E9C00074E6D4F8200384F8EE7290F8BC130129A1
:10E9D00012D080F83870016807F07F03D1F8002862
:10E9E00022F4FE62C1F80028D1F8002842EA03129E
:10E9F000C1F8002880F8BCE3079A0421C2F8E412A9
:10EA000001464FF4807221F83C2F51F82C2CC1F8AC
:10EA10000CE0C1F814E0012AC1F818E008BFC0F802
:10EA20004CE00068D2B211F0B5F9002F14BF0220FB
:10EA30000120079981F8EC0289E003281CD1079B8B
:10EA40000221181D4FF0010CC3F8E412C3F81CC0DA
:10EA5000D3F82023C3F820C011464FF4807321F867
:10EA60003C3F90641369C2F850C0012BC2F854E0D7
:10EA700008BFD06410689DE0079C2046802110F0FC
:10EA80007DF82046002110F079F84FF0000E15E6D1
:10EA90000798DDF81880017CD0F804030029029F54
:10EAA0000CBF816AC16A0DF1220088470646022028
:10EAB000707050E1C0B207283FF6D7AEDDF818807D
:10EAC000029FDFE810F00800220127012C0131012C
:10EAD00036013B0140010798D0F80003416836E158
:10EAE000079CDDF81880207C029F50B9D4F80403FD
:10EAF000416B2CE1079CDDF81880207C029F0028E8
:10EB000061D02046802110F039F82046002110F015
:10EB100035F870E1002F60D0079CDDF81880606840
:10EB2000029F01287AD1D4F820030421C4F8E4120A
:10EB30001CE6079C8021204610F020F8204600218A
:10EB400010F01CF8D4F80403416820468847DDF82B
:10EB500018804FF0000E69E4D4F820C3C6EBC6015C
:10EB60000CEB810101F13E06002B08BF01F5FF7699
:10EB700031784CF6D43600290EBFC0F800E00121F0
:10EB80000160079CC2F20106022261464FF48073C5
:10EB9000C4F8E422C4E9072221F83C3F51F82C3C98
:10EBA000C8604A61012BC1F818E008BFCCF84C00DE
:10EBB000DCF80000DAB240E1079A0421D2F8200321
:10EBC000C2F8E41219E0D4F80403016B0DF122003D
:10EBD0008847064607207070BDE0079C0221D4F8E4
:10EBE000040384F8EC1241682046C4F804E0884726
:10EBF000D4F820030421C4F8E41201464FF48072D3
:10EC000021F83C2F02690023DDF81880029F8364FD
:10EC10000365012A436508BFC3640CE1D4F804030B
:10EC200041682046884747F6F011D4F80403C1F242
:10EC300000010978002861603FF41FAF0168204699
:10EC4000884700287FF419AFD4F820030421C4F8C2
:10EC5000E41201464FF4807221F83C2F0269002330
:10EC600083640365012A4FF0000C436508BFC0F8B8
:10EC70004CC0E0E0C2EBC20100EB810C01234CF67A
:10EC8000D4360CF13C018CF83D30C2F2010690F80C
:10EC9000BC3381F802E0012B0A7020D04E78036863
:10ECA000012E4FF001064FEA421280F8BC6314BFF8
:10ECB00003F5306303F510639E5826F400169E504A
:10ECC000C97801F0FE01022903D1D15841F08051E9
:10ECD000D1504CF6D436C2F2010680F8BCE3079A54
:10ECE0000421C2F8E41201464FF4807221F83C2F4F
:10ECF00051F82C2CC1F80CE0C1F814E0012AC1F83D
:10ED000018E008BFC0F84CE095E00798D0F8000381
:10ED100081681CE00798D0F80003C16817E00798E5
:10ED2000D0F80003016912E00798D0F800034169A8
:10ED30000DE00798D0F80003816908E00798D0F843
:10ED40000003C16903E00798D0F80003016A0DF1E0
:10ED5000220088470646BDF8221019B3079B4FF0E2
:10ED6000000CB3F8FE0200284CD0814238BF0846A0
:10ED7000D3F820230221C3F8E412D86118621146A7
:10ED80004FF4807321F83C3F1369ADF82200106501
:10ED90009664012BC2F854C008BFD6641068DAB27A
:10EDA00010F0F8FF079B4FF0000CB3F8FE0248B3D9
:10EDB000BDF8221000293FF472AC814238BF0846EA
:10EDC000079B0221D3F82023C3F8E412D86118620C
:10EDD00011464FF4807321F83C3F1369ADF82200CF
:10EDE00010659664012BC2F854C008BFD664106841
:10EDF000DAB210F0CFFF4CF6D436C2F201064FF073
:10EE0000000E5BE4D3F820030421C3F8E4120146AA
:10EE10004FF4807221F83C2F02694CF6D436012A57
:10EE2000C2F20106C0F848C0C0F850C0C0F854C0D3
:10EE300001D1C0F84CC00068D2B210F0ABFF4FF067
:10EE4000000EFFF73BBC306800E040464169826934
:10EE50001140490340F1D081D0F81818D0F81C288F
:10EE600011401FFA81F8B8F1000F00F0C581069833
:10EE7000002300F510604FF0000A059008E000BF85
:10EE80000AF1010AB3EB580F4FEA580800F0AF81BE
:10EE90005FEAC870F4D04CF6D436C2F2010630688E
:10EEA0000AF00F05D0F81018D0F8342800EB4A13F8
:10EEB000EA40D201D2B2D3F80839114301EA030B78
:10EEC000059F5FEACB714FEA4A19049500F0D6809E
:10EED000069B0124D3F8341804FA05F29143C3F8D1
:10EEE000341807EB09018C60316901290AD1CAEB9A
:10EEF000CA0106EB8101D1E91123BAF1000F1A44CE
:10EF00008A641BD0D6F804445FEA0A6010D0D4F8B3
:10EF100004034269002A00F0B18094F8EC0203284F
:10EF200040F0AC805FFA8AF120469047059FA5E04B
:10EF3000CAEBCA0006EB800048302FE0316D49BBB8
:10EF4000016C43F20A02C4F65472914203D9D0F81C
:10EF5000001B00291ED40021C0F8101BD0F8101B84
:10EF600041F40021C0F8101BD0F8101B41F018012B
:10EF7000C0F8101BD0F8101B41F0C041C0F8101BA6
:10EF800006F57171C0F8141BD0F8001B41F0802108
:10EF9000C0F8001BD6F8044406F14800D4F8E41287
:10EFA000022964D1D4E90812914219D9891AD4F8F6
:10EFB00020238BB2006813651369216211464FF458
:10EFC0008076002521F83C6F9064012B556508BFC1
:10EFD000D0641068DAB210F0DDFED4F8200332E01D
:10EFE0001ED1E06988421BD3D4F8E812884217D2B8
:10EFF000D4F820034FF48072014621F83C2F0269B7
:10F00000002585640565012A456508BFC56400685B
:10F01000D2B210F0BFFED4F82003C4F8E85212E0D8
:10F02000D4F804030025C06820B194F8EC12032939
:10F0300008BF8047204680210FF0A0FDD4F82003B0
:10F040000521C4F8E412C0F80852C0F81052026951
:10F05000C0F81452012AA0F8FC5108BFC0F80C52A5
:10F0600000F5FE710068D2B210F094FE059F94F88E
:10F07000F002012804BF002084F8F0025FEA0B7060
:10F0800042BF07EB0900082181605FEACB6042BF05
:10F0900007EB0900102181605FEA4B6042BF07EB7C
:10F0A0000900402181605FEA8B704FF0000342BF8E
:10F0B00007EB0900022181605FEA0B607FF5E0AE9B
:10F0C0004CF6D431CAEBCA00C2F2010101EB800058
:10F0D000014651F850EF0A4652F804CFE645FFF4D6
:10F0E000CFAE4CF6D433C2F201031D6883465BF801
:10F0F000443FAEEB0C0609EB05049E4288BF1E465A
:10F10000D4F818790336BFB2B7EB960F28BFE6459F
:10F110000DD8E6454FF000033FF6B2AED5F83408FF
:10F12000049A012191408843C5F83408A8E6483084
:10F13000D0F8009004F51064029005F580504FEA75
:10F140000A36079403954CF6D435C2F20105AEEBAE
:10F150000C072C7C9F4288BF1F469CB11368FD1C86
:10F1600003EB070C079BC2F800C09B69D1F800E0D5
:10F170009BB2B3EB950FB94428BFE64532D9DBF813
:10F180000030E0E7032313FA87F30025B5EB930F74
:10F19000E4D09C08651E04F0030C032D4C4611D3EB
:10F1A0006FF0030505EA93035B424C462568043380
:10F1B000355065683550A5683550E56804F1100490
:10F1C0003550F3D1BCF1000FC8D02368BCF1010F5A
:10F1D0003350C3D06368BCF1020F33501CBFA36827
:10F1E0003350BBE70298039DC0F8009091E74CF6BE
:10F1F000D436C2F20106306841698269DDF818E050
:10F200001140B1F1FF3F1BDCDEF8041821F00101D1
:10F21000CEF8041896F8F413012903D1002186F8DA
:10F22000F41309E0D6F8041491F8EC22042A04BF80
:10F2300091F8ED2281F8EC22416901F00041416131
:10F24000416982691140090520D5DEF80818C9070F
:10F2500018D0D6F8041491F8EC2281F8ED2204229B
:10F2600081F8EC22D0F8001E41F00101C0F8001E28
:10F27000316A39B14EF61051CEF200010A6842F0FF
:10F2800006020A60416901F40061416141698269D5
:10F290001140C90440F14D81DEF804280EF50061EB
:10F2A00022F00102CEF804284FF48462026140F695
:10F2B0004452C0F20302043A0CD003699B0609D5FC
:10F2C00003699B0644BF03695FEA836302D5036950
:10F2D0009B06F0D47368002B00F0D7805A1E032AD7
:10F2E00003F0030C01D200237CE023F003035F4210
:10F2F00000234FF67F3600BF0EEB0305C5F8086903
:10F30000D5F80049043724F40014C5F80049D5F8AD
:10F31000004903F1800344F00064C5F80049C5F8D2
:10F32000086BD5F8004B24F40014C5F8004BD5F851
:10F33000004B44F00064C5F8004BC5F82869D5F8C7
:10F34000204924F40014C5F82049D5F8204944F098
:10F350000064C5F82049C5F8286BD5F8204B24F483
:10F360000014C5F8204BD5F8204B44F00064C5F8D4
:10F37000204BC5F84869D5F8404924F40014C5F875
:10F380004049D5F8404944F00064C5F84049C5F803
:10F39000486BD5F8404B24F40014C5F8404BD5F821
:10F3A000404B44F00064C5F8404BC5F86869D5F897
:10F3B000604924F40014C5F86049D5F8604944F068
:10F3C0000064C5F86049C5F8686BD5F8604B24F453
:10F3D0000014C5F8604BD5F8604B44F00064C5F8E4
:10F3E000604B89D1BCF1000F4FD00EF51067FE18AD
:10F3F0004FF67F35B560FE58BCF1010F26F40016BC
:10F40000FE50FC580EF5306644F00064FC5006EBEC
:10F410000304A560F45824F40014F450F45844F0A4
:10F420000064F45031D003F120043A1995603A5940
:10F43000BCF1020F22F400123A513A5942F0006234
:10F440003A5106EB04029560325922F4001232510F
:10F45000325942F00062325117D003F14002BB181A
:10F460004FF67F359D60BB5823F40013BB50BB584B
:10F4700043F00063BB50B3189D60B35823F40013EE
:10F48000B350B35843F00063B350CA694CF6D43656
:10F4900042F00112CA61C2F20106326B42B1D1F8E8
:10F4A000842042F00B02C1F8842001F1440206E0FE
:10F4B0004A6942F22B031A434A6101F110021368B0
:10F4C00043F00B0313600A6843F20A0322F4FE625E
:10F4D0000A603169026CC4F654739A4203D9D0F8B9
:10F4E000002B002A21D40022C0F8102BD0F8102BBA
:10F4F000C9B242F40022C0F8102BD0F8102B012919
:10F5000042F01802C0F8102BD0F8102B42F0C04285
:10F51000C0F8102B09D106F57171C0F8141BD0F892
:10F52000001B41F08021C0F8001B416901F48051AB
:10F53000416141698269114089044FD5D0F80019B1
:10F5400040F2FF729143C0F80019D0F8041841F45A
:10F550008071C0F80418D0F8081811F0060F04D014
:10F56000890700F187800F2100E00021F1604FF44E
:10F570001051C268012522F47052C260C268114362
:10F58000C160D6F804440020C4F8E4026060C4F806
:10F59000F402D4F80403257484F8EC5210B14168E5
:10F5A00020468847204600210022102310260FF015
:10F5B00079FA2046802100221023C4F88051C4F833
:10F5C0008C610FF06FFA4CF6D430C2F20100006883
:10F5D000A5616662416901F4005141614169826936
:10F5E0004CF6D4351140C2F2010509070FD5D5F804
:10F5F000041491F8EC22032A05D1D1F80413C96947
:10F6000009B188472868416901F0080141614169F1
:10F6100082691140C90203D5416901F48011416139
:10F62000416982691140890203D5416901F40011E1
:10F630004161416982691140490003D5416901F086
:10F640008041416141698269114049070FD5446891
:10F65000610709D5D5F804040122D0F8041380F815
:10F66000EC2249688847286841682143416009B015
:10F67000BDE8F08F4AF24831C2F20101096845F253
:10F680004032CFF6277243F200530A44C0F20C0313
:10F690009A424FF00202F26002D24FF4705168E7D2
:10F6A00041F64062CFF61B7244F240230A44C0F296
:10F6B0000F039A4202D24FF460515AE7A1F5740247
:10F6C00044F68073A2F51052C0F212039A4202D29D
:10F6D0004FF450514DE7A1F183724DF22063A2F532
:10F6E000E742C0F213039A4202D24FF4405140E77E
:10F6F0004BF26062CFF6E5624EF260330A44C0F22C
:10F7000016039A4202D24FF4305132E74DF20032E2
:10F71000CFF6CE6247F240730A44C0F21B039A420E
:10F7200002D24FF4205124E745F6C032CFF6B3623F
:10F7300049F2C0130A44C0F221039A42FFF417AF02
:10F74000A1F1B77247F22053A2F55852C0F2380324
:10F750009A4202D24FF400510BE745F2E042CFF655
:10F76000596249F6E0430A44C0F241034FF4C051E4
:10F770009A4238BF4FF4E051FBE600004AF22850AD
:10F78000C2F201000178012918BF7047002141F23F
:10F79000040C4AF224520170CEF2000CC2F20102B3
:10F7A00042F67023DCF800101268C1F200031868FA
:10F7B000891A08441860DCF8000042F67421C1F28E
:10F7C000000108607047000081B000204CF6641111
:10F7D0000090C2F201010A686FF004011160136C1D
:10F7E0009FED723A00939DED002A00901160D36B5B
:10F7F00000939DED000A00901160536C0093009BF4
:10F8000000901160926C0092009A49F25C62009044
:10F81000C1F2000212681160136C0093009B00900B
:10F820001160D06B4AF24C3100909DED001A42F607
:10F830002C20B8EE411AC1F2000021EE031A90ED1F
:10F84000063AC2F2010191ED004A21EE031A34EEAC
:10F85000413A9FED574AB0EEC33AB4EE443AB8EE9F
:10F86000423A9FED542AF1EE10FAC8BF81ED001A1A
:10F870009FED511A23EE023AB4EE413AF1EE10FA3E
:10F8800013DA4BF6DC70C2F201000021016047F28E
:10F89000DC70C1F2000001604CF20800C2F201000D
:10F8A0004FF07E51016001B07047B8EE400A9FED05
:10F8B000434A90ED055A4BF6DC7020EE020AC2F284
:10F8C000010033EE043A30EE042AB4EE410A90ED22
:10F8D000000A47F2DC7125EE033A25EE022A9FED7D
:10F8E000384AC1F20001F1EE10FAB8BFB0EE442A76
:10F8F00033EE401AB6EE003A91ED004A21EE031ABB
:10F9000031EE001A32EE440A20EE030A30EE040A09
:10F9100030EE012A31EE403A82EE032A80ED001AE1
:10F920004CF2080081ED000AC2F20100B4EE410A77
:10F930000021F1EE10FAC4F22011B2EE043A21EEE9
:10F94000011A20EE000A80ED002AC8BF016090ED88
:10F95000002AB4EE432A9FED1B2AF1EE10FAC8BF2D
:10F9600001604CF2000021EE021AC2F2010080EDAB
:10F97000001A90ED001A20EE020AB5EE401AF1EEE0
:10F9800010FABCBF0021016047F69010C1F20000E0
:10F9900080ED000A90ED000AB5EE400AF1EE10FA93
:10F9A000BCBF0021016001B0704700BF3333533A40
:10F9B000CDCC4C3EC836533A0AD7233C3D0A573E7D
:10F9C0006F12833A0AD7A33C2DE9F04F81B02DED99
:10F9D000028B82B047F2F07AC1F2000A9AF8010075
:10F9E0000AF12C0B002858460AF1100308BF1846EC
:10F9F000056848F6E4570020C0F60307002D08BF4D
:10FA000040F68C25019303E02430B0F54F7F16D0EB
:10FA1000395C012903D13E1871898D4222D03918F1
:10FA20000A7B012A02D1CA8A954219D00A7E012A8C
:10FA3000EAD14A8C9542E7D101F1180612E041F271
:10FA40007920C0F6040018F0CDF9012018F040FA32
:10FA5000A8B218F03DFA48F6E456C0F6030601E0F5
:10FA600001F10C064BF6CD72C2F20102307A7168D8
:10FA70009146127847F294684BF68C64C1F2000804
:10FA8000C2F2010488F80000C8F808102AB1C100C9
:10FA90002046F1F774FE307A7168C8F8044099F88E
:10FAA00000204BF6047447F2A068C2F20104C1F2D0
:10FAB00000082070A1602AB1C1004046F1F75FFE46
:10FAC000307A7168C4F8048099F8002047F29C7479
:10FAD0004BF61C76C1F20004C2F201062070A16050
:10FAE00032B1C1004BF61C70C2F20100F1F747FEC3
:10FAF0004FF6FE70C7F6FF7000210222666005E037
:10FB00002431B1F54F7F02F103021DD07B5C022B43
:10FB100003D1931E03402C2B11D07B181E7B022E89
:10FB200003D1561E06402C2E0BD01E7E022EE7D18E
:10FB300002EA00062C2EE3D103F1180015E0781834
:10FB400013E003F10C0010E041F27920C0F604004C
:10FB500018F048F9022018F0BBF94FF47A7018F049
:10FB6000B7F948F6E450C0F603009AF801100AF11C
:10FB70002402002908BF0AF10802116821F00101DE
:10FB800002292DD1002103E02431B1F54F7F15D09A
:10FB9000785C022803D178184289954220D07818E1
:10FBA000027B022A02D1C28A954218D0027E022A22
:10FBB000EAD1428C9542E7D1183011E041F2792028
:10FBC000C0F6040018F00EF9022018F081F9A8B26E
:10FBD00018F07EF948F6E450C0F6030000E00C305F
:10FBE000017A406899F800204BF6905447F210656E
:10FBF000C2F20104C1F200052170A06032B147F2E7
:10FC00001060C900C1F20000F1F7B9FD9AF80100D7
:10FC10000AF128016560002808BF0AF10C010C6890
:10FC20000020002C08BF4FF4967403E02430B0F598
:10FC30004F7F14D0395C19B93D1869898C4221D0A5
:10FC400039180A7B12B9CA8A944219D00A7E002A4E
:10FC5000ECD14A8C9442E9D101F1180512E041F24D
:10FC60007920C0F6040018F0BDF8002018F030F933
:10FC7000A0B218F02DF948F6E455C0F6030501E0EE
:10FC800001F10C05287A696899F8002047F2886626
:10FC90004BF69C54C1F20006C2F201043070B16010
:10FCA0002AB1C1002046F1F76AFD287A69687460BC
:10FCB00099F800204BF6107447F22475C2F2010443
:10FCC000C1F200052070A16032B1C10047F224707A
:10FCD000C1F20000F1F753FD9AF8010065600028B9
:10FCE000019808BF8346DBF8000043F697210138EE
:10FCF000884219D900200022B0F54C7F35D011463A
:10FD00003A1892F82430002B08BF04293FD092F80B
:10FD100030300A1D002B00F13000EDD141F003011D
:10FD20004329E9D138443AE00020B0F54C7F10D0A7
:10FD300039180A7E002A08BF30282BD091F82420D9
:10FD4000002A08BFB0F5407F27D03030B0F54C7F97
:10FD5000EED141F27920C0F6040018F043F80020FB
:10FD600018F0B6F843F698200AE041F27920C0F680
:10FD7000040018F037F8002018F0AAF844F62060C4
:10FD800018F0A6F848F6E450C0F6030007E002F1C8
:10FD9000240004E001F1180001E001F12400017ADF
:10FDA000406899F8002047F218744BF61465C1F2C8
:10FDB0000004C2F201052170A06032B14BF614605C
:10FDC000C900C2F20100F1F7DAFC9AF960619FED17
:10FDD000F48A00EE106AB8EEC00AB0EEC00A20EE57
:10FDE000080A10EE100A65601BF0C8F9002E00EE3C
:10FDF000100A0ED49FEDEB1A9FEDEB2A20EE014A7C
:10FE00009FEDEA1A9FEDEA3A34EE020A32EE442AF6
:10FE10001BE09FEDE81A9FEDE83A20EE014A34EE30
:10FE2000030AB7EE001A81EE005A9FEDE40A9FED37
:10FE3000E41A9FEDE42A33EE443A25EE000A25EE5B
:10FE4000011A25EE022A25EE033A42F630609AF9AD
:10FE50006141C1F2000080ED000A00EE104AB8EEE8
:10FE6000C00AB0EEC00AB1EE414AB1EE433A20EE0C
:10FE7000080A80ED011A80ED022A80ED034A80ED28
:10FE8000043A10EE100A1BF079F9002C00EE100A6B
:10FE90000ED49FEDCD1A9FEDCD2A20EE014A9FEDA5
:10FEA000CC1A9FEDCC3A34EE020A32EE442A1BE023
:10FEB0009FEDC91A9FEDC93A20EE014A34EE030ABC
:10FEC000B7EE001A81EE005A9FEDC50A9FEDC51AE4
:10FED0009FEDC52A33EE443A25EE000A25EE011ABD
:10FEE00025EE022A25EE033A4AF2B4509AF962410D
:10FEF000C2F2010080ED000A00EE104AB8EEC00A1E
:10FF0000B0EEC00AB1EE414AB1EE433A20EE080A23
:10FF100080ED011A80ED022A80ED034A80ED043A5B
:10FF200010EE100A1BF02AF9002C00EE100A0ED475
:10FF30009FEDAE1A9FEDAE2A20EE014A9FEDAD1A5D
:10FF40009FEDAD3A34EE020A32EE442A1BE09FEDFB
:10FF5000AB1A9FEDAB3A20EE014A34EE030AB7EE3E
:10FF6000001A81EE005A9FEDA70A9FEDA71A9FED98
:10FF7000A72A33EE443A25EE000A25EE011A25EEB3
:10FF8000022A25EE033A42F614609AF96341C1F25F
:10FF9000000080ED000A00EE104AB8EEC00AB0EE94
:10FFA000C00AB1EE414AB1EE433A20EE080A80EDB4
:10FFB000011A80ED022A80ED034A80ED043A10EE2A
:10FFC000100A1BF0DBF8002C00EE100A0ED49FED97
:10FFD000751A9FED752A20EE014A9FED741A9FED68
:10FFE000743A34EE020A32EE442A1BE09FED711A95
:10FFF0009FED713A20EE014A34EE030AB7EE001A83
:020000040801F1
:1000000081EE005A9FED6D0A9FED6D1A9FED6D2AEE
:1000100033EE443A25EE000A25EE011A25EE022AB7
:1000200025EE033A4AF290509AF96441C2F2010077
:1000300080ED000A00EE104AB8EEC00AB0EEC00A29
:10004000B1EE414AB1EE433A20EE080A80ED011AC2
:1000500080ED022A80ED034A80ED043A10EE100A8A
:100060001BF08CF8002C00EE100A0ED49FED561AEF
:100070009FED562A20EE014A9FED551A9FED553A05
:1000800034EE020A32EE442A1BE09FED531A9FED34
:10009000533A20EE014A34EE030AB7EE001A81EE1D
:1000A000005A9FED4F0A9FED4F1A9FED4F2A33EEF6
:1000B000443A25EE000A25EE011A25EE022A25EE25
:1000C000033A42F6F8509AF96541C1F2000080ED1A
:1000D000000A00EE104AB8EEC00AB0EEC00AB1EE57
:1000E000414AB1EE433A20EE080A80ED011A80ED54
:1000F000022A80ED034A80ED043A10EE100A1BF04C
:100100003DF8002C00EE100A0ED49FED381A9FED3A
:10011000382A20EE014A9FED371A9FED373A34EE28
:10012000020A32EE442A1BE09FED341A9FED343A66
:1001300020EE014A34EE030AB7EE001A81EE005AAF
:100140009FED300A9FED301A9FED302A33EE443A8E
:1001500025EE000A25EE011A25EE022A25EE033AC5
:100160004AF27450C2F20100B1EE414AB1EE433A94
:1001700080ED000A80ED011A80ED022A80ED034A2D
:1001800080ED043A4BF6CC70C2F201000021017000
:1001900089F8001002B0BDEC028B01B0BDE8F08F11
:1001A0002D152A3EF7B44B3DB044733F58EFF2BFD4
:1001B0006189663FDC83563D7816803F97CA863F4B
:1001C00010D3FFBFB2C4723FC5F07A3DF450703F08
:1001D000A242EEBFE8A1603FA73B863DC58C803FB1
:1001E0007FF0883F76E6FEBF1552703F8AA7A23D9A
:1001F0000FAB6B3F54A3E3BF1E56573FE3BFB33D66
:10020000F337823FF1738D3F1B90FBBFEAF76D3FE1
:100210004AF22850C2F20100017801291BD10021C5
:1002200041F2040C4AF224520170CEF2000CC2F2E8
:10023000010242F67023DCF800101268C1F20003DC
:100240001868891A08441860DCF8000042F6742126
:10025000C1F2000108604CF68C30C2F20100416B23
:10026000084700002DE9F04F87B047F2E174C1F272
:10027000000492462278012A38D148F21864C1F26B
:100280000004218848F2185A4CF2782800270FF20F
:10029000C879C1F2000AC2F2010800250FE000BFD0
:1002A000F1F7B8FD218801283BD088B2B0F5807FF6
:1002B00005F1010524BF00212180082D31D019F856
:1002C00005008AB20AF802000131B8F800008AB2CB
:1002D00082422180E9D10026F1F79CFDB7EB562F31
:1002E000DED1012806F10106F6D0D9E749F6840BE4
:1002F000C1F2000B8046DBF81C00109F1D460E4625
:10030000102800F0A68010204FF00009CBF81C0048
:10031000CBF828909BF8511041B3BE46AC46002163
:1003200067E088B20A220AF80020481CB8F80010DA
:1003300082B28A42208011D100250026F1F76AFDA1
:10034000B5EB562F03D1012806F10106F6D0F1F7DF
:1003500061FD012801D10021FFE1208880B2B0F5C4
:10036000807F4FF0000128BF2180F6E143F60000B6
:10037000DBF80010C4F2000081428BF85090CDF8F9
:100380001890CDE90499CDF80C90CDF8089002D0E2
:10039000102000212BE0002143F630020191C4F22D
:1003A0000202136900F5E63043F4804313611369D8
:1003B00003F480430193019B0191136843F002030E
:1003C0001360126802F002020192019A4FF4604237
:1003D0000292022203920122CDE904210521069115
:1003E00002A9F7F799F8DBF81C00DBF82810BE46E5
:1003F000AC4602228BF851209BE83C00234317684F
:100400002B4327F040071760DBF8107047F2E174C8
:100410003B43DBE90575C1F200043B4305F400777B
:100420003B43DBF820701843384308431060042036
:10043000DBF8241000EA154008435060D069654697
:1004400020F40060D06101207746CBF854908BF8FF
:100450005100DDF84490012020703804A86146B1B5
:1004600030465146F0F7EFFFB8F1000F6CD0404630
:1004700076E09BF8500001287BD04FF0010E49F642
:10048000EC628BF850E0C1F2000213689BF8510057
:10049000012840F08980B8F1000F4FF0010018BF2B
:1004A000BAF1000F00F04881032000218BF85100C1
:1004B000CBF85410CBF83080ABF834A0ABF836A0B2
:1004C000CBF83810ABF83C10ABF83E10DBF80870F6
:1004D000DBF80000B7F5004FCBF840100097CBF8E1
:1004E000441003D1016841F4804101600168AC46C9
:1004F000490603D4016841F040010160DBF8046063
:10050000AAF10107DBF80C10B6FA86F5B7FA87F7FF
:100510006D097F09B1F5006F47EA050140F0AF8032
:1005200049B138F8021BC160CBF83080BBF83610F7
:100530000139ABF83610BBF83610002900F0D28034
:10054000DBF80070002126E0DBF80430B3F5827F91
:100550000BD1DBF8080040B904208BF8510030467D
:1005600031465246F7F78CFCEBE09BF8500001282F
:100570001CD10220E5E038F8025BC560CBF8308082
:10058000BBF836000138ABF83600BBF8360000285F
:10059000384600F0A7808568AD07ECD41068C01A13
:1005A000B1EB502FF1D099E00220C5E04FF0010CE3
:1005B00049F6EC6E8BF850C0C1F2000EDEF8002058
:1005C0009BF85110012956D1BAF1000F00F0EF80CD
:1005D00004218BF851100021CBF85410CBF838606F
:1005E000ABF83CA0ABF83EA0CBF83010ABF8341021
:1005F000ABF83610DBF80870CBF84010B7F5004FB9
:10060000DBF80070CBF8441003D1396821F4804145
:1006100039603968A846490603D4396841F0400179
:100620003960DBF80C50BBF83E10002D00F0C5809F
:10063000002900F0C080DBF8005000210FE0F868CE
:1006400026F8020BCBF83860BBF83E000138ABF857
:100650003E00BBF83E002F46002800F0AC80B86892
:10066000C007ECD1DEF80000801AB1EB502FF0D0BB
:1006700003204546ECE102208BF851C05EE069B1F1
:1006800098F800100173DBF8300000F10108CBF896
:100690003080BBF836000138ABF83600BBF83600C6
:1006A00000B3DBF80000002110E098F8005005735B
:1006B000DBF8305005F10108CBF83080BBF836503C
:1006C000013DABF83650BBF836505DB18568AD07DB
:1006D000EBD41568ED1AB1EB552FF4D0109F032021
:1006E000654629E04AF24830C2F20100006849F646
:1006F0008171C1F25E61A0FB0101480D4FF47A7176
:1007000048430290DBF80070B6F5827F29D1B868C3
:100710006546000672D40099109F41B900200290EE
:10072000DBF80000C1680291806802900298DBF853
:100730005400002818BF01208BF851E000218BF8ED
:100740005010B9F1000F4FF0000140F0020008BF57
:10075000AF610328217018BF0121084607B0BDE82A
:10076000F08F654602980028D5D002980138029093
:10077000B8680006CFD502980028CCD0029801387E
:100780000290B8680006C6D502980028C3D0029827
:1007900001380290B8680006BDD502980028BAD08A
:1007A000029801380290B8680006DBD4B3E7012054
:1007B0008BF851C0C2E7454673E00029454670D02A
:1007C0000023B868C00706D1DEF80000801AB3EB3A
:1007D000502F0CD006E1387B3070DBF83800461C17
:1007E000CBF83860BBF83E000138ABF83E00BBF8F0
:1007F0003E00002853D0DBF80070E2E700201168CB
:10080000C91AB1F5007F1ED2B96809067FF583AF1A
:100810001168C91AB0EB512F15D1B96809067FF5D7
:100820007AAF1168C91AB0EB512F0CD1B96809061B
:100830007FF571AF1168C91AB0EB512F03D1B968B8
:100840000906DCD467E77868009920F0E000B1F58C
:10085000004F786002D0B1F5806F03D1386820F086
:1008600040003860DBF82800B0F5005F07D1386839
:1008700020F400503860386840F40050386001209F
:100880008BF8510000208BF85000DBF8540040F04A
:100890002000CBF854002020CBF854003CE7DBF8D4
:1008A0000430B3F5827F41D1DBF80870B7F5004F13
:1008B00002D0B7F5806F65D1DBF80000B7F5806F27
:1008C000016821F0400101605CD1DBF800309868DC
:1008D000C00700F0B8800027DEF80000801AB0F5ED
:1008E000007F80F08C809868C00700F0AC80DEF854
:1008F0000000801AB7EB502F40F081809868C00745
:1009000000F0A180DEF80000801AB7EB502F76D1FE
:100910009868C00700F09780DEF80000801AB7EBF7
:10092000502F6CD19868C007D6D18CE0DBF800302E
:100930009868C00700F087800027DEF80000801A62
:10094000B0F5007F49D29868C0077CD0DEF800007F
:10095000801AB7EB502F40D19868C00773D0DEF8EB
:100960000000801AB7EB502F37D19868C0076AD0C3
:10097000DEF80000801AB7EB502F2ED19868C00720
:10098000DBD160E0DBF80030986800065BD500261C
:10099000DEF80000801AB0F5007F25D298680006C6
:1009A00051D5DEF80000801AB6EB502F1CD19868A4
:1009B000000648D5DEF80000801AB6EB502F13D1A0
:1009C000986800063FD5DEF80000801AB6EB502F7D
:1009D0000AD198680006DBD435E0586820F0E000C2
:1009E000586014E0032033E05868B7F5004F20F05A
:1009F000E000586007D0B7F5806F04D007E0586872
:100A000020F0E0005860186820F040001860DBF823
:100A10002800B0F5005F07D1186820F40050186076
:100A2000186840F40050186001208BF85100002035
:100A30008BF85000DBF8540040F02000CBF8540055
:100A40002020CBF85400DBF85400002818BF012008
:100A5000109F8BF851C071E653504920427573794D
:100A6000000000004AF22850C2F20100017801297A
:100A700018BF7047002141F2040C4AF22452017061
:100A8000CEF2000CC2F2010242F67023DCF8001034
:100A90001268C1F200031868891A08441860DCF86B
:100AA000000042F67421C1F20001086070470000A6
:100AB0002DE9F04381B004464008E02800F2EC80C4
:100AC00000296DD004F11A07BDB200262846052181
:100AD0002A4640F22B1300964FF00508F8F796FBD4
:100AE00000214FF0C0404FF02A0C2A0AC6F208013C
:100AF000FDB24FF02B094FF02C0E47F6EF37402395
:100B0000A0F800C00A800D800A800D80A0F8009037
:100B10000E80A1F800800E80A1F80080A0F800E00F
:100B20000F80A0F800C00A800D800A800D80A0F818
:100B300000900E800B800E800B807B23A0F800E0DD
:100B40000F80A0F800C00A800D800A800D80A0F8F8
:100B500000900E800B800E800B80B623A0F800E082
:100B60000F80A0F800C00A800D800A800D80A0F8D8
:100B700000900E800B800E800B80A0F800E00F80AC
:100B8000A0F800C00A800D800A80F1220D80A0F834
:100B900000900E800A800E800A80A0F800E00F808E
:100BA000002C43D0611E47F6106289B2C1F20002E8
:100BB00002EB810191ED000A9FED391A9FED392A70
:100BC00020EE010A32EE400ABDEEC00A10EE101A05
:100BD0004F1D002948BF052702EB840240F22B116C
:100BE000B7F5957FC8BF0F4692ED000A04F11900D2
:100BF00020EE010A32EE400ABDEEC00A10EE103AB5
:100C00005E1D04F11A02002B48BF0526B6F5957F3C
:100C1000C8BF0E464FF47845B3B2B9B280B292B2B3
:100C20000095F8F7C3FF01B0BDE8F08347F6106008
:100C3000C1F2000090ED000A9FED1B1A9FED192AEA
:100C400020EE010A30EE020ABDEEC00A10EE100AD4
:100C5000411D002848BF05214FF0C0422A23B1F5AD
:100C6000957FC8BF40F22B111380002388B2C6F2D3
:100C7000080300271A261F801E801F802B27000ACA
:100C8000C9B21E8017801880198018802C20198006
:100C900010804FF47840188001B0BDE8F08300BFA9
:100CA000721C03428EE3A343721C03C22DE9F04F72
:100CB00093B047F2B472C1F20002117811B113B0CF
:100CC000BDE8F08F4FF001094AF2B63682F8009085
:100CD000C2F20106044630880121FFF7E9FEB4F1B3
:100CE000FF3F05DC30880021013080B2FFF7E0FED5
:100CF00030880DF10C0B051928B200240028D8BF4C
:100D00002546A8B2B0F5E07F58464FF0400188BFB5
:100D100040F2C1153580F0F732FD4DF2D04049F276
:100D20003461C2F20100C1F20001006809684BF6AB
:100D3000B942091AC9F2F51252FB01110A1202EB6B
:100D4000D171AAB201FB020044F6D351C1F2620193
:100D500050FB01F147F61060C1F2000050F822008C
:100D60008B1103EBD1751BF02BFA41EC100B41F208
:100D7000F311C0F6040158462A468DED000BEFF73B
:100D800023FBAA2040F22F114FF4B97240F2351321
:100D90000094AA25F8F73AFA49F6DE67C1F200078F
:100DA00000214FF00008002620E000BF002A49D0B3
:100DB000A8EB060000EB400005EB400080B240F2DB
:100DC0002F114FF4FC630094CDF80490F8F73AFD2E
:100DD00008F10100811B01EB410105EB41011FFA04
:100DE00088F2398081B27F2A80462BD21BF80120FD
:100DF0005E2ADBD101EB0B0040786F28D8D108F1D7
:100E000001096FEA060A0136A9EB06011FFA89F00B
:100E100001EB410100231BF8002005EB41000124F8
:100E2000009380B24FF496714FF4FC630194F8F78D
:100E300009FD08F1020000EB0A01C84600244FF04A
:100E40000109C8E74AF2B630C2F2010000884FF447
:100E5000FC671A3080B20521024640F22B1300973E
:100E6000F8F7D4F947F2B4710020C1F2000108701C
:100E700013B0BDE8F08F00002DE9F04FA5B047F2A8
:100E8000B4724DF2D045C1F200024FF0010AC2F235
:100E9000010582F800A0286049F23460C1F2000028
:100EA000016047F2F071C1F2000148780A1D20315B
:100EB000002808460491039208BF104600684BF6CC
:100EC000C071C2F2010108604BF6FC70C2F2010071
:100ED00000784BF6BC71C2F20101087000204FF09F
:100EE0000008F8F767F84FF6FF741920052119225A
:100EF00040F22B130094F8F789F919204FF49671FA
:100F000040F2DB124FF496730094F8F77FF90DF17D
:100F1000140948464021F0F732FC286844F6D351C2
:100F2000C1F26201A0FB01018A0941F25161C0F6E0
:100F300004014846EFF748FA49F6DE651B24C1F282
:100F400000050021002600271EE000BF002A49D02E
:100F5000F01B00EB400004EB400080B240F22F1188
:100F60004FF4FC63CDF80080CDF804A0F8F76AFCDC
:100F7000701CC11B01EB410104EB4101B2B229809D
:100F800081B27F2A06462DD219F801205E2ADDD1D2
:100F900001EB090040786F28DAD106F1010B6FEA06
:100FA000070A0137ABEB07011FFA8BF001EB410198
:100FB00019F8002004EB4100012580B24FF496712E
:100FC0004FF4FC63CDF800800195F8F73BFCB01CB2
:100FD00049F6DE6500EB0A014FF0010A5E46C1F2F8
:100FE0000005C7E749F23460C1F20000006844F62A
:100FF000D351C1F26201A0FB01018A0941F25161A2
:10100000C0F604014846EFF7DFF94FF0000840F260
:10101000B71B4FF0010A00210027002422E000BF87
:10102000002A42D0381B00EB40000BEB400080B29E
:1010300040F22F114FF4FC63CDF80080CDF804A0EE
:10104000F8F700FC781C011B01EB410149F6DE6258
:101050000BEB4101C1F200021180BAB281B27F2ACA
:10106000074622D219F801205E2AD9D101EB0900E6
:1010700040786F28D6D17D1CE6430134291BA8B2E5
:1010800001EB410119F800200BEB410080B24FF455
:1010900096714FF4FC63CDF80080CDF804A0F8F70A
:1010A000D1FBB81C81192F46CEE715AE3046402142
:1010B000F0F765FB4DF2D04049F23461C2F2010015
:1010C000C1F20001006809684BF6B942091AC9F279
:1010D000F51252FB01114AF2B633C2F201030A12B1
:1010E000B3F9003002EBD17101FB030044F6D35198
:1010F000C1F2620150FB01F147F61060C1F200003D
:1011000050F823008A1102EBD1771BF059F841EC1B
:10111000100B41F2F311C0F6040130463A468DED52
:10112000000BEFF751F90025AA2040F22F114FF4E0
:10113000B97240F235130095AA24F8F767F849F61A
:10114000DE6B012700214FF000084FF0000AC1F2CA
:10115000000B20E0002A48D0A8EB0A0000EB40007A
:1011600004EB400080B240F22F114FF4FC63009575
:101170000197F8F767FB08F10100A0EB0A0101EB0A
:10118000410104EB41011FFA88F2ABF8001081B273
:101190007F2A804629D2725C5E2ADBD1881940788A
:1011A0006F28D9D108F101056FEA0A0B0AF1010A8B
:1011B000A5EB0A01A8B201EB41010023325C04EB6C
:1011C0004100009380B24FF496714FF4FC63019795
:1011D000F8F738FB08F1020000EB0B0149F6DE6B73
:1011E000C1F2000BA8460025C9E74AF2B630C2F2A8
:1011F000010000884FF4FC671A3080B205210246D6
:1012000040F22B130097F8F701F89FEDEB0B41F23A
:10121000022153EC102BC0F604014846EFF7D4F836
:101220004FF000084FF0010A0021002400271AE0C7
:10123000D2B3E01B00EB4000400080B205214FF428
:10124000FC63CDF80080CDF804A0F8F7FBFA601C31
:10125000C11B01EB41014900A2B2ABF8001081B201
:101260007F2A044620D219F801205E2AE0D101EB42
:10127000090040786F28DCD1651CFE430137E91B6B
:10128000A8B201EB410119F80020480080B2022108
:101290004FF4FC63CDF80080CDF804A0F8F7D2FA43
:1012A000A01C81192C46D4E747F6EF3719200521F9
:1012B00040F2DB1205230097F7F7A8FF9FEDC00B64
:1012C00041F2022153EC102BC0F604014846EFF71F
:1012D0007BF84FF000084FF0010A0021002400279E
:1012E0001BE000BFD2B3E01B00EB4000400080B227
:1012F00040214FF4FC63CDF80080CDF804A0F8F74E
:10130000A1FA601CC11B01EB41014900A2B2ABF87C
:10131000001081B27F2A044620D219F801205E2AEB
:10132000E0D101EB090040786F28DCD1651CFE4359
:101330000137E91BA8B201EB410119F80020480070
:1013400080B23D214FF4FC63CDF80080CDF804A0BD
:10135000F8F778FAA01C81192C46D4E747F6EF3746
:101360001920402140F2DB1240230097F7F74EFF8F
:101370009FEDEF0B41F2022153EC102BC0F604015C
:101380004846EFF721F84FF000084FF0010A00211E
:10139000002400271BE000BFD2B3E01B00EB40009D
:1013A000400080B27B214FF4FC63CDF80080CDF883
:1013B00004A0F8F747FA601CC11B01EB410149008A
:1013C000A2B2ABF8001081B27F2A044620D219F8ED
:1013D00001205E2AE0D101EB090040786F28DCD1C2
:1013E000651CFE430137E91BA8B201EB410119F866
:1013F0000020480080B278214FF4FC63CDF80080D3
:10140000CDF804A0F8F71EFAA01C81192C46D4E7E9
:1014100047F6EF3719207B2140F2DB127B23009740
:10142000F7F7F4FE9FEDC40B41F2022153EC102BB1
:10143000C0F604014846EEF7C7FF4FF000084FF032
:10144000010A0021002400271BE000BFD2B3E01BEB
:1014500000EB4000400080B2B6214FF4FC63CDF8B1
:101460000080CDF804A0F8F7EDF9601CC11B01EB7A
:1014700041014900A2B2ABF8001081B27F2A0446B4
:1014800020D219F801205E2AE0D101EB0900407852
:101490006F28DCD1651CFE430137E91BA8B201EBC4
:1014A000410119F80020480080B2B3214FF4FC63D9
:1014B000CDF80080CDF804A0F8F7C4F9A01C81197C
:1014C0002C46D4E747F6EF371920B62140F2DB125D
:1014D000B6230097F7F79AFE9FED990B41F2022190
:1014E00053EC102BC0F604014846EEF76DFF4FF0A9
:1014F00000084FF0010A0021002400271BE000BF74
:10150000D2B3E01B00EB4000400080B2F1214FF469
:10151000FC63CDF80080CDF804A0F8F793F9601CC7
:10152000C11B01EB41014900A2B2ABF8001081B22E
:101530007F2A044620D219F801205E2AE0D101EB6F
:10154000090040786F28DCD1651CFE430137E91B98
:10155000A8B201EB410119F80020480080B2EE2149
:101560004FF4FC63CDF80080CDF804A0F8F76AF9D9
:10157000A01C81192C46D4E747F6EF371920F1213A
:1015800040F2DB12F1230097F7F740FE9FED6E0B60
:1015900041F2022153EC102BC0F604014846EEF74D
:1015A00013FF4FF000084FF0010A0021002400272C
:1015B00026E000BF00BF00BF000000000000244084
:1015C0000000006066662040E2B3E01B00EB4000D4
:1015D000400080B24FF496714FF4FC63CDF8008068
:1015E000CDF804A0F8F72EF9601CC11B01EB4101F6
:1015F0004900A2B2ABF8001081B27F2A044621D282
:1016000019F801205E2ADFD101EB090040786F282C
:10161000DBD1651CFE430137E91BA8B201EB410198
:1016200019F80020480080B240F229114FF4FC6301
:10163000CDF80080CDF804A0F8F704F9A01C8119BA
:101640002C46D3E747F6EF3719204FF4967140F256
:10165000DB124FF496730097F7F7D8FD47F2F0705E
:10166000C1F200004DF2D0454178C2F20105286870
:101670000029DDE9032108BF11460CF0F9FB4BF608
:10168000FC700124C2F20100047047F69D10C1F203
:101690000000047000784CF21B01C2F201010870D6
:1016A0000BF084FE4BF27450C2F2010049F2346137
:1016B0000470C1F20001286809684BF2C532091AAA
:1016C000C9F2A21200EE100A49F6F850A1FB02126C
:1016D000B8EE400AC1F2000080ED000A100A00EEE8
:1016E000100A4CF23C60B8EE400AC2F2010080EDF4
:1016F000000A49F23860C1F200000021018049F679
:10170000EC60C1F20000006849F6E062C1F200023C
:10171000106047F2B470C1F2000001704BF6947093
:10172000C2F20100C47225B0BDE8F08F00BF00BF57
:10173000000000A0999919400000008066661240E0
:101740000000008066660640000000000000F03FD8
:101750004AF2144041F29C61C2F20100C0F6040159
:10176000016042F66C1041F2BC61C1F20000C0F6AB
:10177000040101604DF2D540C2F201000121017067
:1017800049F6DB60C1F20000002202704BF6947053
:10179000C2F2010001737047B0B547F2F074C1F2B4
:1017A000000420B1C043C0B2C00984F88E01607843
:1017B00004F12001002808BF211D0868012101252E
:1017C00012F064F9012809DBC1B2890094F88E2176
:1017D00051FA80F004EB800080F84D204BF27450F9
:1017E000C2F201000570B0BD40B1C043C0B247F2C3
:1017F000F071C009C1F2000181F88F014BF2745001
:10180000C2F2010001210170704700004AF2144049
:1018100041F2C061C2F20100C0F60401016042F66B
:101820006C1041F64001C1F20000C0F604010160F5
:101830004DF2D540C2F201000121017049F6DB6092
:10184000C1F20000002202704BF69470C2F2010057
:101850000173704747F2F071C1F2000191F85E2107
:10186000104442B212F1500FD8BF6FF04F0042B295
:1018700012F10A0FA8BF6FF0090081F85E017047EE
:101880002DE9F04147F2F078C1F20008B8F8741180
:1018900001281DDBB1F5616F36DB41F287308142F3
:1018A0005FDD41F65730814240F39E8041F658306B
:1018B000814200F0FA8042F22830B1F5FA5F00F080
:1018C000F980814204BF42F21070A8F874013DE132
:1018D00040F6D76081422DDD41F26F70814261DDBB
:1018E000B1F5FA5FC0F2AE8000F0048142F2283018
:1018F000814200F0048142F21070814204BF42F242
:101900002830A8F8740121E140F65330814238DCD8
:1019100040F6C310814274DC40F63400814200F08E
:10192000CC8040F6FC00814204BF40F6C410A8F809
:1019300074010BE140F6B730814244DC40F68B2065
:10194000814200F38C8040F6FC00814200F0DC8094
:1019500040F6C410814204BF40F6FC00A8F87401B0
:10196000F4E0B1F57A6F59DA40F6D860B1F5616FFD
:1019700000F0A880814204BF4FF47A60A8F8740197
:10198000E4E0B1F5486F53DA40F65430814200F09C
:101990009C8040F6B830814204BF4FF44860A8F8FC
:1019A0007401D3E041F29310814265DC40F6D860C7
:1019B000814200F0AE80B1F57A6F04BF40F6D86086
:1019C000A8F87401C2E040F64750814261DC40F65D
:1019D000B830814200F0A280B1F5486F04BF40F6F4
:1019E000B830A8F87401B1E041F28830814271D07A
:1019F00041F27070814204BF41F65830A8F874017A
:101A0000A4E040F6C410814269D040F68C208142A7
:101A100004BF40F65430A8F8740197E041F29410E6
:101A200062D0814204BF41F28830A8F874018DE091
:101A300040F648505BD0814204BF4FF46160A8F883
:101A4000740183E041F2707081426CD041F65830ED
:101A5000814204BF41F27070A8F8740176E040F64C
:101A60008C20814264D040F65430814204BF40F65D
:101A70008C20A8F8740169E041F2941081425CD096
:101A800041F28830814204BF41F29410A8F87401F9
:101A90005CE040F64850814254D0B1F5616F04BF1C
:101AA00040F64850A8F8740150E04FF4FA50A8F8F6
:101AB00074014BE0A8F8740148E040F6FC00A8F877
:101AC000740143E0A8F8740140E040F6B830A8F88B
:101AD00074013BE041F27070A8F8740136E040F602
:101AE0008C20A8F8740131E0A8F874012EE0A8F861
:101AF00074012BE041F65830A8F8740126E04FF449
:101B0000FA50A8F8740121E040F63400A8F87401F6
:101B10001CE040F64850A8F8740117E040F6543035
:101B2000A8F8740112E041F28830A8F874010DE0C1
:101B300040F6C410A8F8740108E040F6D860A8F890
:101B4000740103E04FF44860A8F8740198F80100AC
:101B500008F108050028284608F1240608BF304689
:101B600008F104070068394608F1200408BF21463F
:101B70000CF086FB98F80100002808BF2E4630685C
:101B800008BF3C462146BDE8F0410CF079BB00009F
:101B9000002808BF7047C043C0B247F2F071C009C7
:101BA000C1F2000181F87901704700002DE9F04190
:101BB00047F2F078C1F20008B8F86E11012806DB90
:101BC0003C290CD091B93C20A8F86E010EE06429A4
:101BD00009D03C290AD10020A8F86E0106E0642053
:101BE000A8F86E0102E03C20A8F86E0198F8010008
:101BF00008F108050028284608F1240608BF3046E9
